Archive member included because of file (symbol)

e:/logiciels/freescale/kinetis design studio v2.0.0/toolchain/bin/../lib/gcc/arm-none-eabi/4.8.0\libgcc.a(_udivsi3.o)
                              ./Tools/StringTools/StringTools.o (__aeabi_uidiv)
e:/logiciels/freescale/kinetis design studio v2.0.0/toolchain/bin/../lib/gcc/arm-none-eabi/4.8.0\libgcc.a(_dvmd_tls.o)
                              e:/logiciels/freescale/kinetis design studio v2.0.0/toolchain/bin/../lib/gcc/arm-none-eabi/4.8.0\libgcc.a(_udivsi3.o) (__aeabi_idiv0)
e:/logiciels/freescale/kinetis design studio v2.0.0/toolchain/bin/../lib/gcc/arm-none-eabi/4.8.0/../../../../arm-none-eabi/lib\libg_s.a(lib_a-atexit.o)
                              e:/logiciels/freescale/kinetis design studio v2.0.0/toolchain/bin/../lib/gcc/arm-none-eabi/4.8.0/../../../../arm-none-eabi/lib/crt0.o (atexit)
e:/logiciels/freescale/kinetis design studio v2.0.0/toolchain/bin/../lib/gcc/arm-none-eabi/4.8.0/../../../../arm-none-eabi/lib\libg_s.a(lib_a-exit.o)
                              e:/logiciels/freescale/kinetis design studio v2.0.0/toolchain/bin/../lib/gcc/arm-none-eabi/4.8.0/../../../../arm-none-eabi/lib/crt0.o (exit)
e:/logiciels/freescale/kinetis design studio v2.0.0/toolchain/bin/../lib/gcc/arm-none-eabi/4.8.0/../../../../arm-none-eabi/lib\libg_s.a(lib_a-fini.o)
                              e:/logiciels/freescale/kinetis design studio v2.0.0/toolchain/bin/../lib/gcc/arm-none-eabi/4.8.0/../../../../arm-none-eabi/lib\libg_s.a(lib_a-exit.o) (__libc_fini_array)
e:/logiciels/freescale/kinetis design studio v2.0.0/toolchain/bin/../lib/gcc/arm-none-eabi/4.8.0/../../../../arm-none-eabi/lib\libg_s.a(lib_a-impure.o)
                              e:/logiciels/freescale/kinetis design studio v2.0.0/toolchain/bin/../lib/gcc/arm-none-eabi/4.8.0/../../../../arm-none-eabi/lib\libg_s.a(lib_a-exit.o) (_global_impure_ptr)
e:/logiciels/freescale/kinetis design studio v2.0.0/toolchain/bin/../lib/gcc/arm-none-eabi/4.8.0/../../../../arm-none-eabi/lib\libg_s.a(lib_a-memcpy.o)
                              ./BSP/FRAM/FM25V20MemTest.o (memcpy)
e:/logiciels/freescale/kinetis design studio v2.0.0/toolchain/bin/../lib/gcc/arm-none-eabi/4.8.0/../../../../arm-none-eabi/lib\libg_s.a(lib_a-memset.o)
                              e:/logiciels/freescale/kinetis design studio v2.0.0/toolchain/bin/../lib/gcc/arm-none-eabi/4.8.0/../../../../arm-none-eabi/lib/crt0.o (memset)
e:/logiciels/freescale/kinetis design studio v2.0.0/toolchain/bin/../lib/gcc/arm-none-eabi/4.8.0/../../../../arm-none-eabi/lib\libg_s.a(lib_a-syscalls.o)
                              e:/logiciels/freescale/kinetis design studio v2.0.0/toolchain/bin/../lib/gcc/arm-none-eabi/4.8.0/../../../../arm-none-eabi/lib\libg_s.a(lib_a-exit.o) (_exit)
e:/logiciels/freescale/kinetis design studio v2.0.0/toolchain/bin/../lib/gcc/arm-none-eabi/4.8.0/../../../../arm-none-eabi/lib\libg_s.a(lib_a-__atexit.o)
                              e:/logiciels/freescale/kinetis design studio v2.0.0/toolchain/bin/../lib/gcc/arm-none-eabi/4.8.0/../../../../arm-none-eabi/lib\libg_s.a(lib_a-atexit.o) (__do_register_exitproc)
e:/logiciels/freescale/kinetis design studio v2.0.0/toolchain/bin/../lib/gcc/arm-none-eabi/4.8.0/../../../../arm-none-eabi/lib\libg_s.a(lib_a-__call_atexit.o)
                              e:/logiciels/freescale/kinetis design studio v2.0.0/toolchain/bin/../lib/gcc/arm-none-eabi/4.8.0/../../../../arm-none-eabi/lib\libg_s.a(lib_a-__atexit.o) (__call_exitprocs)
e:/logiciels/freescale/kinetis design studio v2.0.0/toolchain/bin/../lib/gcc/arm-none-eabi/4.8.0/../../../../arm-none-eabi/lib\libg_s.a(lib_a-errno.o)
                              e:/logiciels/freescale/kinetis design studio v2.0.0/toolchain/bin/../lib/gcc/arm-none-eabi/4.8.0/../../../../arm-none-eabi/lib\libg_s.a(lib_a-syscalls.o) (__errno)
e:/logiciels/freescale/kinetis design studio v2.0.0/toolchain/bin/../lib/gcc/arm-none-eabi/4.8.0/../../../../arm-none-eabi/lib\libg_s.a(lib_a-malloc.o)
                              e:/logiciels/freescale/kinetis design studio v2.0.0/toolchain/bin/../lib/gcc/arm-none-eabi/4.8.0/../../../../arm-none-eabi/lib\libg_s.a(lib_a-__atexit.o) (malloc)
e:/logiciels/freescale/kinetis design studio v2.0.0/toolchain/bin/../lib/gcc/arm-none-eabi/4.8.0/../../../../arm-none-eabi/lib\libg_s.a(lib_a-mallocr.o)
                              e:/logiciels/freescale/kinetis design studio v2.0.0/toolchain/bin/../lib/gcc/arm-none-eabi/4.8.0/../../../../arm-none-eabi/lib\libg_s.a(lib_a-malloc.o) (_malloc_r)
e:/logiciels/freescale/kinetis design studio v2.0.0/toolchain/bin/../lib/gcc/arm-none-eabi/4.8.0/../../../../arm-none-eabi/lib\libg_s.a(lib_a-sbrkr.o)
                              e:/logiciels/freescale/kinetis design studio v2.0.0/toolchain/bin/../lib/gcc/arm-none-eabi/4.8.0/../../../../arm-none-eabi/lib\libg_s.a(lib_a-mallocr.o) (_sbrk_r)
e:/logiciels/freescale/kinetis design studio v2.0.0/toolchain/bin/../lib/gcc/arm-none-eabi/4.8.0/../../../../arm-none-eabi/lib\libg_s.a(lib_a-strlen.o)
                              e:/logiciels/freescale/kinetis design studio v2.0.0/toolchain/bin/../lib/gcc/arm-none-eabi/4.8.0/../../../../arm-none-eabi/lib\libg_s.a(lib_a-syscalls.o) (strlen)
e:/logiciels/freescale/kinetis design studio v2.0.0/toolchain/bin/../lib/gcc/arm-none-eabi/4.8.0/../../../../arm-none-eabi/lib\libg_s.a(lib_a-freer.o)
                              e:/logiciels/freescale/kinetis design studio v2.0.0/toolchain/bin/../lib/gcc/arm-none-eabi/4.8.0/../../../../arm-none-eabi/lib\libg_s.a(lib_a-malloc.o) (_free_r)
e:/logiciels/freescale/kinetis design studio v2.0.0/toolchain/bin/../lib/gcc/arm-none-eabi/4.8.0/../../../../arm-none-eabi/lib\libg_s.a(lib_a-reent.o)
                              e:/logiciels/freescale/kinetis design studio v2.0.0/toolchain/bin/../lib/gcc/arm-none-eabi/4.8.0/../../../../arm-none-eabi/lib\libg_s.a(lib_a-sbrkr.o) (errno)

Allocating common symbols
Common symbol       size              file

BQBatteryStatus     0x28              ./BSP/BatteryManagement/BQ27510DRZRG2.o
CR95HFCtrl          0x128             ./BSP/RFID_CR95HF/CR95HF.o
SRDEeprom           0x40              ./Application/RFIDManager/RFIDManager.o
errno               0x4               e:/logiciels/freescale/kinetis design studio v2.0.0/toolchain/bin/../lib/gcc/arm-none-eabi/4.8.0/../../../../arm-none-eabi/lib\libg_s.a(lib_a-reent.o)
RFIDCtrl            0x50              ./Application/RFIDManager/RFIDManager.o
Uart2Ctrl           0x1c              ./DSP/UART/uart2.o
txBuf               0x80              ./DSP/UART/uart1.o
PowerManagerCtrl    0x2               ./Application/PowerManager/PowerManager.o
SerialParameters    0x10              ./Application/MemoryManager/MemoryManager.o
rxBuf               0x80              ./DSP/UART/uart1.o
Spi1Baudrate        0x4               ./DSP/SPI/spi1.o
DeviceClock         0x2c              ./DSP/DSP/DSP_mkl16z256vlh4.o
Spi0Baudrate        0x4               ./DSP/SPI/spi0.o
TickCtrl            0x14              ./BSP/Tick/tick.o
ButtonManagerCtrl   0x4               ./Application/ButtonManager/ButtonManager.o
DivingParameters    0x4               ./Application/MemoryManager/MemoryManager.o
UsbCtrl             0x90              ./Application/UsbManager/UsbManager.o
Uart1Ctrl           0x1c              ./DSP/UART/uart1.o
MemoryManagerCtrl   0x8               ./Application/MemoryManager/MemoryManager.o
Uart0Ctrl           0x1c              ./DSP/UART/uart0.o

Discarded input sections

 .text          0x00000000        0x0 e:/logiciels/freescale/kinetis design studio v2.0.0/toolchain/bin/../lib/gcc/arm-none-eabi/4.8.0/crti.o
 .data          0x00000000        0x0 e:/logiciels/freescale/kinetis design studio v2.0.0/toolchain/bin/../lib/gcc/arm-none-eabi/4.8.0/crti.o
 .bss           0x00000000        0x0 e:/logiciels/freescale/kinetis design studio v2.0.0/toolchain/bin/../lib/gcc/arm-none-eabi/4.8.0/crti.o
 .text          0x00000000        0x0 e:/logiciels/freescale/kinetis design studio v2.0.0/toolchain/bin/../lib/gcc/arm-none-eabi/4.8.0/crtbegin.o
 .data          0x00000000        0x0 e:/logiciels/freescale/kinetis design studio v2.0.0/toolchain/bin/../lib/gcc/arm-none-eabi/4.8.0/crtbegin.o
 .bss           0x00000000        0x0 e:/logiciels/freescale/kinetis design studio v2.0.0/toolchain/bin/../lib/gcc/arm-none-eabi/4.8.0/crtbegin.o
 .data.__dso_handle
                0x00000000        0x4 e:/logiciels/freescale/kinetis design studio v2.0.0/toolchain/bin/../lib/gcc/arm-none-eabi/4.8.0/crtbegin.o
 .data          0x00000000        0x0 e:/logiciels/freescale/kinetis design studio v2.0.0/toolchain/bin/../lib/gcc/arm-none-eabi/4.8.0/../../../../arm-none-eabi/lib/crt0.o
 .bss           0x00000000        0x0 e:/logiciels/freescale/kinetis design studio v2.0.0/toolchain/bin/../lib/gcc/arm-none-eabi/4.8.0/../../../../arm-none-eabi/lib/crt0.o
 .group         0x00000000        0x8 ./Tools/StringTools/StringTools.o
 .text          0x00000000        0x0 ./Tools/StringTools/StringTools.o
 .data          0x00000000        0x0 ./Tools/StringTools/StringTools.o
 .bss           0x00000000        0x0 ./Tools/StringTools/StringTools.o
 .text.StrTool_StringLength
                0x00000000       0x40 ./Tools/StringTools/StringTools.o
 .text.StrTool_StringCopy
                0x00000000       0x70 ./Tools/StringTools/StringTools.o
 .text.StrTool_UnsignedLongToStringHex
                0x00000000       0xf8 ./Tools/StringTools/StringTools.o
 .text.StrTool_UnsignedLongToString
                0x00000000       0xe8 ./Tools/StringTools/StringTools.o
 .text.StrTool_SignedLongToString
                0x00000000       0x44 ./Tools/StringTools/StringTools.o
 .text.StrTool_StringToUnsignedLong
                0x00000000       0x78 ./Tools/StringTools/StringTools.o
 .group         0x00000000        0x8 ./Tools/Decoder7Seg/decoder7Seg.o
 .group         0x00000000        0x8 ./Tools/Decoder7Seg/decoder7Seg.o
 .text          0x00000000        0x0 ./Tools/Decoder7Seg/decoder7Seg.o
 .data          0x00000000        0x0 ./Tools/Decoder7Seg/decoder7Seg.o
 .bss           0x00000000        0x0 ./Tools/Decoder7Seg/decoder7Seg.o
 .text.Decode7segDigitASCIIDot
                0x00000000       0x4c ./Tools/Decoder7Seg/decoder7Seg.o
 .debug_macro   0x00000000      0x802 ./Tools/Decoder7Seg/decoder7Seg.o
 .group         0x00000000        0x8 ./Tools/Decoder16Seg/decoder16Seg.o
 .group         0x00000000        0x8 ./Tools/Decoder16Seg/decoder16Seg.o
 .text          0x00000000        0x0 ./Tools/Decoder16Seg/decoder16Seg.o
 .data          0x00000000        0x0 ./Tools/Decoder16Seg/decoder16Seg.o
 .bss           0x00000000        0x0 ./Tools/Decoder16Seg/decoder16Seg.o
 .debug_macro   0x00000000      0x802 ./Tools/Decoder16Seg/decoder16Seg.o
 .group         0x00000000        0x8 ./Tools/Checksum/checksum.o
 .text          0x00000000        0x0 ./Tools/Checksum/checksum.o
 .data          0x00000000        0x0 ./Tools/Checksum/checksum.o
 .bss           0x00000000        0x0 ./Tools/Checksum/checksum.o
 .text.ChecksumShortCompute
                0x00000000       0x40 ./Tools/Checksum/checksum.o
 .text.ChecksumLongCompute
                0x00000000       0x3c ./Tools/Checksum/checksum.o
 .debug_macro   0x00000000      0x802 ./Tools/Checksum/checksum.o
 .data          0x00000000        0x0 ./Project_Settings/Startup_Code/startup_MKL16Z4.o
 .bss           0x00000000        0x0 ./Project_Settings/Startup_Code/startup_MKL16Z4.o
 .group         0x00000000        0x8 ./Project_Settings/Startup_Code/system_MKL16Z4.o
 .group         0x00000000        0x8 ./Project_Settings/Startup_Code/system_MKL16Z4.o
 .group         0x00000000        0x8 ./Project_Settings/Startup_Code/system_MKL16Z4.o
 .group         0x00000000        0x8 ./Project_Settings/Startup_Code/system_MKL16Z4.o
 .group         0x00000000        0x8 ./Project_Settings/Startup_Code/system_MKL16Z4.o
 .group         0x00000000        0x8 ./Project_Settings/Startup_Code/system_MKL16Z4.o
 .group         0x00000000        0x8 ./Project_Settings/Startup_Code/system_MKL16Z4.o
 .group         0x00000000        0x8 ./Project_Settings/Startup_Code/system_MKL16Z4.o
 .text          0x00000000        0x0 ./Project_Settings/Startup_Code/system_MKL16Z4.o
 .data          0x00000000        0x0 ./Project_Settings/Startup_Code/system_MKL16Z4.o
 .bss           0x00000000        0x0 ./Project_Settings/Startup_Code/system_MKL16Z4.o
 .data.SystemCoreClock
                0x00000000        0x4 ./Project_Settings/Startup_Code/system_MKL16Z4.o
 .text.SystemCoreClockUpdate
                0x00000000      0x278 ./Project_Settings/Startup_Code/system_MKL16Z4.o
 .debug_macro   0x00000000      0x802 ./Project_Settings/Startup_Code/system_MKL16Z4.o
 .group         0x00000000        0x8 ./DSP/Watchdog/watchdog.o
 .group         0x00000000        0x8 ./DSP/Watchdog/watchdog.o
 .group         0x00000000        0x8 ./DSP/Watchdog/watchdog.o
 .group         0x00000000        0x8 ./DSP/Watchdog/watchdog.o
 .group         0x00000000        0x8 ./DSP/Watchdog/watchdog.o
 .group         0x00000000        0x8 ./DSP/Watchdog/watchdog.o
 .group         0x00000000        0x8 ./DSP/Watchdog/watchdog.o
 .group         0x00000000        0x8 ./DSP/Watchdog/watchdog.o
 .group         0x00000000        0x8 ./DSP/Watchdog/watchdog.o
 .group         0x00000000        0x8 ./DSP/Watchdog/watchdog.o
 .text          0x00000000        0x0 ./DSP/Watchdog/watchdog.o
 .data          0x00000000        0x0 ./DSP/Watchdog/watchdog.o
 .bss           0x00000000        0x0 ./DSP/Watchdog/watchdog.o
 .text.WatchdogStop
                0x00000000       0x18 ./DSP/Watchdog/watchdog.o
 .debug_macro   0x00000000      0x802 ./DSP/Watchdog/watchdog.o
 .debug_macro   0x00000000      0x214 ./DSP/Watchdog/watchdog.o
 .debug_macro   0x00000000       0x3a ./DSP/Watchdog/watchdog.o
 .debug_macro   0x00000000       0x1f ./DSP/Watchdog/watchdog.o
 .debug_macro   0x00000000      0x250 ./DSP/Watchdog/watchdog.o
 .debug_macro   0x00000000       0xc5 ./DSP/Watchdog/watchdog.o
 .debug_macro   0x00000000     0x5642 ./DSP/Watchdog/watchdog.o
 .group         0x00000000        0x8 ./DSP/UART/uart0.o
 .group         0x00000000        0x8 ./DSP/UART/uart0.o
 .group         0x00000000        0x8 ./DSP/UART/uart0.o
 .group         0x00000000        0x8 ./DSP/UART/uart0.o
 .group         0x00000000        0x8 ./DSP/UART/uart0.o
 .group         0x00000000        0x8 ./DSP/UART/uart0.o
 .group         0x00000000        0x8 ./DSP/UART/uart0.o
 .group         0x00000000        0x8 ./DSP/UART/uart0.o
 .group         0x00000000        0x8 ./DSP/UART/uart0.o
 .group         0x00000000        0x8 ./DSP/UART/uart0.o
 .group         0x00000000        0x8 ./DSP/UART/uart0.o
 .text          0x00000000        0x0 ./DSP/UART/uart0.o
 .data          0x00000000        0x0 ./DSP/UART/uart0.o
 .bss           0x00000000        0x0 ./DSP/UART/uart0.o
 .text.Uart0SendString
                0x00000000       0xbc ./DSP/UART/uart0.o
 .debug_macro   0x00000000      0x802 ./DSP/UART/uart0.o
 .debug_macro   0x00000000       0x16 ./DSP/UART/uart0.o
 .debug_macro   0x00000000      0x214 ./DSP/UART/uart0.o
 .debug_macro   0x00000000       0x39 ./DSP/UART/uart0.o
 .debug_macro   0x00000000       0x3a ./DSP/UART/uart0.o
 .debug_macro   0x00000000       0x1f ./DSP/UART/uart0.o
 .debug_macro   0x00000000      0x250 ./DSP/UART/uart0.o
 .debug_macro   0x00000000       0xc5 ./DSP/UART/uart0.o
 .debug_macro   0x00000000     0x5642 ./DSP/UART/uart0.o
 .debug_macro   0x00000000      0x1fb ./DSP/UART/uart0.o
 .group         0x00000000        0x8 ./DSP/UART/uart1.o
 .group         0x00000000        0x8 ./DSP/UART/uart1.o
 .group         0x00000000        0x8 ./DSP/UART/uart1.o
 .group         0x00000000        0x8 ./DSP/UART/uart1.o
 .group         0x00000000        0x8 ./DSP/UART/uart1.o
 .group         0x00000000        0x8 ./DSP/UART/uart1.o
 .group         0x00000000        0x8 ./DSP/UART/uart1.o
 .group         0x00000000        0x8 ./DSP/UART/uart1.o
 .group         0x00000000        0x8 ./DSP/UART/uart1.o
 .group         0x00000000        0x8 ./DSP/UART/uart1.o
 .group         0x00000000        0x8 ./DSP/UART/uart1.o
 .text          0x00000000        0x0 ./DSP/UART/uart1.o
 .data          0x00000000        0x0 ./DSP/UART/uart1.o
 .bss           0x00000000        0x0 ./DSP/UART/uart1.o
 .debug_macro   0x00000000      0x802 ./DSP/UART/uart1.o
 .debug_macro   0x00000000       0x16 ./DSP/UART/uart1.o
 .debug_macro   0x00000000      0x214 ./DSP/UART/uart1.o
 .debug_macro   0x00000000       0x39 ./DSP/UART/uart1.o
 .debug_macro   0x00000000       0x3a ./DSP/UART/uart1.o
 .debug_macro   0x00000000       0x1f ./DSP/UART/uart1.o
 .debug_macro   0x00000000      0x250 ./DSP/UART/uart1.o
 .debug_macro   0x00000000       0xc5 ./DSP/UART/uart1.o
 .debug_macro   0x00000000     0x5642 ./DSP/UART/uart1.o
 .debug_macro   0x00000000      0x1fb ./DSP/UART/uart1.o
 .group         0x00000000        0x8 ./DSP/UART/uart2.o
 .group         0x00000000        0x8 ./DSP/UART/uart2.o
 .group         0x00000000        0x8 ./DSP/UART/uart2.o
 .group         0x00000000        0x8 ./DSP/UART/uart2.o
 .group         0x00000000        0x8 ./DSP/UART/uart2.o
 .group         0x00000000        0x8 ./DSP/UART/uart2.o
 .group         0x00000000        0x8 ./DSP/UART/uart2.o
 .group         0x00000000        0x8 ./DSP/UART/uart2.o
 .group         0x00000000        0x8 ./DSP/UART/uart2.o
 .group         0x00000000        0x8 ./DSP/UART/uart2.o
 .group         0x00000000        0x8 ./DSP/UART/uart2.o
 .text          0x00000000        0x0 ./DSP/UART/uart2.o
 .data          0x00000000        0x0 ./DSP/UART/uart2.o
 .bss           0x00000000        0x0 ./DSP/UART/uart2.o
 .text.Uart2SendString
                0x00000000       0xbc ./DSP/UART/uart2.o
 .debug_macro   0x00000000      0x802 ./DSP/UART/uart2.o
 .debug_macro   0x00000000       0x16 ./DSP/UART/uart2.o
 .debug_macro   0x00000000      0x214 ./DSP/UART/uart2.o
 .debug_macro   0x00000000       0x39 ./DSP/UART/uart2.o
 .debug_macro   0x00000000       0x3a ./DSP/UART/uart2.o
 .debug_macro   0x00000000       0x1f ./DSP/UART/uart2.o
 .debug_macro   0x00000000      0x250 ./DSP/UART/uart2.o
 .debug_macro   0x00000000       0xc5 ./DSP/UART/uart2.o
 .debug_macro   0x00000000     0x5642 ./DSP/UART/uart2.o
 .debug_macro   0x00000000      0x1fb ./DSP/UART/uart2.o
 .group         0x00000000        0x8 ./DSP/SPI/spi0.o
 .group         0x00000000        0x8 ./DSP/SPI/spi0.o
 .group         0x00000000        0x8 ./DSP/SPI/spi0.o
 .group         0x00000000        0x8 ./DSP/SPI/spi0.o
 .group         0x00000000        0x8 ./DSP/SPI/spi0.o
 .group         0x00000000        0x8 ./DSP/SPI/spi0.o
 .group         0x00000000        0x8 ./DSP/SPI/spi0.o
 .group         0x00000000        0x8 ./DSP/SPI/spi0.o
 .group         0x00000000        0x8 ./DSP/SPI/spi0.o
 .group         0x00000000        0x8 ./DSP/SPI/spi0.o
 .group         0x00000000        0x8 ./DSP/SPI/spi0.o
 .text          0x00000000        0x0 ./DSP/SPI/spi0.o
 .data          0x00000000        0x0 ./DSP/SPI/spi0.o
 .bss           0x00000000        0x0 ./DSP/SPI/spi0.o
 .text.Spi0GetBaudrate
                0x00000000       0x14 ./DSP/SPI/spi0.o
 .text.Spi0Read
                0x00000000       0x9c ./DSP/SPI/spi0.o
 .debug_macro   0x00000000      0x802 ./DSP/SPI/spi0.o
 .debug_macro   0x00000000       0x16 ./DSP/SPI/spi0.o
 .debug_macro   0x00000000      0x214 ./DSP/SPI/spi0.o
 .debug_macro   0x00000000       0x39 ./DSP/SPI/spi0.o
 .debug_macro   0x00000000       0x3a ./DSP/SPI/spi0.o
 .debug_macro   0x00000000       0x1f ./DSP/SPI/spi0.o
 .debug_macro   0x00000000      0x250 ./DSP/SPI/spi0.o
 .debug_macro   0x00000000       0xc5 ./DSP/SPI/spi0.o
 .debug_macro   0x00000000     0x5642 ./DSP/SPI/spi0.o
 .debug_macro   0x00000000      0x1fb ./DSP/SPI/spi0.o
 .group         0x00000000        0x8 ./DSP/SPI/spi1.o
 .group         0x00000000        0x8 ./DSP/SPI/spi1.o
 .group         0x00000000        0x8 ./DSP/SPI/spi1.o
 .group         0x00000000        0x8 ./DSP/SPI/spi1.o
 .group         0x00000000        0x8 ./DSP/SPI/spi1.o
 .group         0x00000000        0x8 ./DSP/SPI/spi1.o
 .group         0x00000000        0x8 ./DSP/SPI/spi1.o
 .group         0x00000000        0x8 ./DSP/SPI/spi1.o
 .group         0x00000000        0x8 ./DSP/SPI/spi1.o
 .group         0x00000000        0x8 ./DSP/SPI/spi1.o
 .group         0x00000000        0x8 ./DSP/SPI/spi1.o
 .text          0x00000000        0x0 ./DSP/SPI/spi1.o
 .data          0x00000000        0x0 ./DSP/SPI/spi1.o
 .bss           0x00000000        0x0 ./DSP/SPI/spi1.o
 .text.Spi1GetBaudrate
                0x00000000       0x14 ./DSP/SPI/spi1.o
 .debug_macro   0x00000000      0x802 ./DSP/SPI/spi1.o
 .debug_macro   0x00000000       0x16 ./DSP/SPI/spi1.o
 .debug_macro   0x00000000      0x214 ./DSP/SPI/spi1.o
 .debug_macro   0x00000000       0x39 ./DSP/SPI/spi1.o
 .debug_macro   0x00000000       0x3a ./DSP/SPI/spi1.o
 .debug_macro   0x00000000       0x1f ./DSP/SPI/spi1.o
 .debug_macro   0x00000000      0x250 ./DSP/SPI/spi1.o
 .debug_macro   0x00000000       0xc5 ./DSP/SPI/spi1.o
 .debug_macro   0x00000000     0x5642 ./DSP/SPI/spi1.o
 .debug_macro   0x00000000      0x1fb ./DSP/SPI/spi1.o
 .group         0x00000000        0x8 ./DSP/RTC/rtc.o
 .group         0x00000000        0x8 ./DSP/RTC/rtc.o
 .group         0x00000000        0x8 ./DSP/RTC/rtc.o
 .group         0x00000000        0x8 ./DSP/RTC/rtc.o
 .group         0x00000000        0x8 ./DSP/RTC/rtc.o
 .group         0x00000000        0x8 ./DSP/RTC/rtc.o
 .group         0x00000000        0x8 ./DSP/RTC/rtc.o
 .group         0x00000000        0x8 ./DSP/RTC/rtc.o
 .group         0x00000000        0x8 ./DSP/RTC/rtc.o
 .group         0x00000000        0x8 ./DSP/RTC/rtc.o
 .group         0x00000000        0x8 ./DSP/RTC/rtc.o
 .text          0x00000000        0x0 ./DSP/RTC/rtc.o
 .data          0x00000000        0x0 ./DSP/RTC/rtc.o
 .bss           0x00000000        0x0 ./DSP/RTC/rtc.o
 .debug_macro   0x00000000      0x802 ./DSP/RTC/rtc.o
 .debug_macro   0x00000000       0x16 ./DSP/RTC/rtc.o
 .debug_macro   0x00000000      0x214 ./DSP/RTC/rtc.o
 .debug_macro   0x00000000       0x39 ./DSP/RTC/rtc.o
 .debug_macro   0x00000000       0x3a ./DSP/RTC/rtc.o
 .debug_macro   0x00000000       0x1f ./DSP/RTC/rtc.o
 .debug_macro   0x00000000      0x250 ./DSP/RTC/rtc.o
 .debug_macro   0x00000000       0xc5 ./DSP/RTC/rtc.o
 .debug_macro   0x00000000     0x5642 ./DSP/RTC/rtc.o
 .debug_macro   0x00000000      0x1fb ./DSP/RTC/rtc.o
 .group         0x00000000        0x8 ./DSP/PIT/pit.o
 .group         0x00000000        0x8 ./DSP/PIT/pit.o
 .group         0x00000000        0x8 ./DSP/PIT/pit.o
 .group         0x00000000        0x8 ./DSP/PIT/pit.o
 .group         0x00000000        0x8 ./DSP/PIT/pit.o
 .group         0x00000000        0x8 ./DSP/PIT/pit.o
 .group         0x00000000        0x8 ./DSP/PIT/pit.o
 .group         0x00000000        0x8 ./DSP/PIT/pit.o
 .group         0x00000000        0x8 ./DSP/PIT/pit.o
 .group         0x00000000        0x8 ./DSP/PIT/pit.o
 .group         0x00000000        0x8 ./DSP/PIT/pit.o
 .text          0x00000000        0x0 ./DSP/PIT/pit.o
 .data          0x00000000        0x0 ./DSP/PIT/pit.o
 .bss           0x00000000        0x0 ./DSP/PIT/pit.o
 .debug_macro   0x00000000      0x802 ./DSP/PIT/pit.o
 .debug_macro   0x00000000       0x16 ./DSP/PIT/pit.o
 .debug_macro   0x00000000      0x214 ./DSP/PIT/pit.o
 .debug_macro   0x00000000       0x39 ./DSP/PIT/pit.o
 .debug_macro   0x00000000       0x3a ./DSP/PIT/pit.o
 .debug_macro   0x00000000       0x1f ./DSP/PIT/pit.o
 .debug_macro   0x00000000      0x250 ./DSP/PIT/pit.o
 .debug_macro   0x00000000       0xc5 ./DSP/PIT/pit.o
 .debug_macro   0x00000000     0x5642 ./DSP/PIT/pit.o
 .debug_macro   0x00000000      0x1fb ./DSP/PIT/pit.o
 .group         0x00000000        0x8 ./DSP/I2C/i2c0.o
 .group         0x00000000        0x8 ./DSP/I2C/i2c0.o
 .group         0x00000000        0x8 ./DSP/I2C/i2c0.o
 .group         0x00000000        0x8 ./DSP/I2C/i2c0.o
 .group         0x00000000        0x8 ./DSP/I2C/i2c0.o
 .group         0x00000000        0x8 ./DSP/I2C/i2c0.o
 .group         0x00000000        0x8 ./DSP/I2C/i2c0.o
 .group         0x00000000        0x8 ./DSP/I2C/i2c0.o
 .group         0x00000000        0x8 ./DSP/I2C/i2c0.o
 .group         0x00000000        0x8 ./DSP/I2C/i2c0.o
 .group         0x00000000        0x8 ./DSP/I2C/i2c0.o
 .text          0x00000000        0x0 ./DSP/I2C/i2c0.o
 .data          0x00000000        0x0 ./DSP/I2C/i2c0.o
 .bss           0x00000000        0x0 ./DSP/I2C/i2c0.o
 .text.I2C0GetBaudrate
                0x00000000       0x14 ./DSP/I2C/i2c0.o
 .debug_macro   0x00000000      0x802 ./DSP/I2C/i2c0.o
 .debug_macro   0x00000000       0x16 ./DSP/I2C/i2c0.o
 .debug_macro   0x00000000      0x214 ./DSP/I2C/i2c0.o
 .debug_macro   0x00000000       0x39 ./DSP/I2C/i2c0.o
 .debug_macro   0x00000000       0x3a ./DSP/I2C/i2c0.o
 .debug_macro   0x00000000       0x1f ./DSP/I2C/i2c0.o
 .debug_macro   0x00000000      0x250 ./DSP/I2C/i2c0.o
 .debug_macro   0x00000000       0xc5 ./DSP/I2C/i2c0.o
 .debug_macro   0x00000000     0x5642 ./DSP/I2C/i2c0.o
 .debug_macro   0x00000000      0x1fb ./DSP/I2C/i2c0.o
 .group         0x00000000        0x8 ./DSP/Device/device.o
 .group         0x00000000        0x8 ./DSP/Device/device.o
 .group         0x00000000        0x8 ./DSP/Device/device.o
 .group         0x00000000        0x8 ./DSP/Device/device.o
 .group         0x00000000        0x8 ./DSP/Device/device.o
 .group         0x00000000        0x8 ./DSP/Device/device.o
 .group         0x00000000        0x8 ./DSP/Device/device.o
 .group         0x00000000        0x8 ./DSP/Device/device.o
 .group         0x00000000        0x8 ./DSP/Device/device.o
 .group         0x00000000        0x8 ./DSP/Device/device.o
 .group         0x00000000        0x8 ./DSP/Device/device.o
 .text          0x00000000        0x0 ./DSP/Device/device.o
 .data          0x00000000        0x0 ./DSP/Device/device.o
 .bss           0x00000000        0x0 ./DSP/Device/device.o
 .text.LPM_Sleep
                0x00000000       0x1c ./DSP/Device/device.o
 .debug_macro   0x00000000      0x802 ./DSP/Device/device.o
 .debug_macro   0x00000000       0x16 ./DSP/Device/device.o
 .debug_macro   0x00000000      0x214 ./DSP/Device/device.o
 .debug_macro   0x00000000       0x39 ./DSP/Device/device.o
 .debug_macro   0x00000000       0x3a ./DSP/Device/device.o
 .debug_macro   0x00000000       0x1f ./DSP/Device/device.o
 .debug_macro   0x00000000      0x250 ./DSP/Device/device.o
 .debug_macro   0x00000000       0xc5 ./DSP/Device/device.o
 .debug_macro   0x00000000     0x5642 ./DSP/Device/device.o
 .debug_macro   0x00000000      0x1fb ./DSP/Device/device.o
 .group         0x00000000        0x8 ./DSP/DSP/DSP_mkl16z256vlh4.o
 .group         0x00000000        0x8 ./DSP/DSP/DSP_mkl16z256vlh4.o
 .group         0x00000000        0x8 ./DSP/DSP/DSP_mkl16z256vlh4.o
 .group         0x00000000        0x8 ./DSP/DSP/DSP_mkl16z256vlh4.o
 .group         0x00000000        0x8 ./DSP/DSP/DSP_mkl16z256vlh4.o
 .group         0x00000000        0x8 ./DSP/DSP/DSP_mkl16z256vlh4.o
 .group         0x00000000        0x8 ./DSP/DSP/DSP_mkl16z256vlh4.o
 .group         0x00000000        0x8 ./DSP/DSP/DSP_mkl16z256vlh4.o
 .group         0x00000000        0x8 ./DSP/DSP/DSP_mkl16z256vlh4.o
 .group         0x00000000        0x8 ./DSP/DSP/DSP_mkl16z256vlh4.o
 .text          0x00000000        0x0 ./DSP/DSP/DSP_mkl16z256vlh4.o
 .data          0x00000000        0x0 ./DSP/DSP/DSP_mkl16z256vlh4.o
 .bss           0x00000000        0x0 ./DSP/DSP/DSP_mkl16z256vlh4.o
 .text.I2C1ClockGate
                0x00000000       0x48 ./DSP/DSP/DSP_mkl16z256vlh4.o
 .text.I2C1PinMappingPeripheral
                0x00000000        0x8 ./DSP/DSP/DSP_mkl16z256vlh4.o
 .debug_macro   0x00000000      0x802 ./DSP/DSP/DSP_mkl16z256vlh4.o
 .debug_macro   0x00000000       0x16 ./DSP/DSP/DSP_mkl16z256vlh4.o
 .debug_macro   0x00000000      0x214 ./DSP/DSP/DSP_mkl16z256vlh4.o
 .debug_macro   0x00000000       0x39 ./DSP/DSP/DSP_mkl16z256vlh4.o
 .debug_macro   0x00000000       0x3a ./DSP/DSP/DSP_mkl16z256vlh4.o
 .debug_macro   0x00000000       0x1f ./DSP/DSP/DSP_mkl16z256vlh4.o
 .debug_macro   0x00000000      0x250 ./DSP/DSP/DSP_mkl16z256vlh4.o
 .debug_macro   0x00000000       0xc5 ./DSP/DSP/DSP_mkl16z256vlh4.o
 .debug_macro   0x00000000     0x5642 ./DSP/DSP/DSP_mkl16z256vlh4.o
 .debug_macro   0x00000000      0x1fb ./DSP/DSP/DSP_mkl16z256vlh4.o
 .group         0x00000000        0x8 ./BSP/Tick/tick.o
 .group         0x00000000        0x8 ./BSP/Tick/tick.o
 .group         0x00000000        0x8 ./BSP/Tick/tick.o
 .group         0x00000000        0x8 ./BSP/Tick/tick.o
 .group         0x00000000        0x8 ./BSP/Tick/tick.o
 .group         0x00000000        0x8 ./BSP/Tick/tick.o
 .group         0x00000000        0x8 ./BSP/Tick/tick.o
 .group         0x00000000        0x8 ./BSP/Tick/tick.o
 .group         0x00000000        0x8 ./BSP/Tick/tick.o
 .group         0x00000000        0x8 ./BSP/Tick/tick.o
 .group         0x00000000        0x8 ./BSP/Tick/tick.o
 .group         0x00000000        0x8 ./BSP/Tick/tick.o
 .text          0x00000000        0x0 ./BSP/Tick/tick.o
 .data          0x00000000        0x0 ./BSP/Tick/tick.o
 .bss           0x00000000        0x0 ./BSP/Tick/tick.o
 .debug_macro   0x00000000      0x802 ./BSP/Tick/tick.o
 .debug_macro   0x00000000       0x16 ./BSP/Tick/tick.o
 .debug_macro   0x00000000      0x214 ./BSP/Tick/tick.o
 .debug_macro   0x00000000       0x39 ./BSP/Tick/tick.o
 .debug_macro   0x00000000       0x3a ./BSP/Tick/tick.o
 .debug_macro   0x00000000       0x1f ./BSP/Tick/tick.o
 .debug_macro   0x00000000      0x250 ./BSP/Tick/tick.o
 .debug_macro   0x00000000       0xc5 ./BSP/Tick/tick.o
 .debug_macro   0x00000000     0x5642 ./BSP/Tick/tick.o
 .debug_macro   0x00000000      0x1fb ./BSP/Tick/tick.o
 .debug_macro   0x00000000       0x2e ./BSP/Tick/tick.o
 .group         0x00000000        0x8 ./BSP/RFID_CR95HF/CR95HF.o
 .group         0x00000000        0x8 ./BSP/RFID_CR95HF/CR95HF.o
 .group         0x00000000        0x8 ./BSP/RFID_CR95HF/CR95HF.o
 .group         0x00000000        0x8 ./BSP/RFID_CR95HF/CR95HF.o
 .group         0x00000000        0x8 ./BSP/RFID_CR95HF/CR95HF.o
 .group         0x00000000        0x8 ./BSP/RFID_CR95HF/CR95HF.o
 .group         0x00000000        0x8 ./BSP/RFID_CR95HF/CR95HF.o
 .group         0x00000000        0x8 ./BSP/RFID_CR95HF/CR95HF.o
 .group         0x00000000        0x8 ./BSP/RFID_CR95HF/CR95HF.o
 .group         0x00000000        0x8 ./BSP/RFID_CR95HF/CR95HF.o
 .group         0x00000000        0x8 ./BSP/RFID_CR95HF/CR95HF.o
 .group         0x00000000        0x8 ./BSP/RFID_CR95HF/CR95HF.o
 .group         0x00000000        0x8 ./BSP/RFID_CR95HF/CR95HF.o
 .group         0x00000000        0x8 ./BSP/RFID_CR95HF/CR95HF.o
 .group         0x00000000        0x8 ./BSP/RFID_CR95HF/CR95HF.o
 .group         0x00000000        0x8 ./BSP/RFID_CR95HF/CR95HF.o
 .text          0x00000000        0x0 ./BSP/RFID_CR95HF/CR95HF.o
 .data          0x00000000        0x0 ./BSP/RFID_CR95HF/CR95HF.o
 .bss           0x00000000        0x0 ./BSP/RFID_CR95HF/CR95HF.o
 .debug_macro   0x00000000      0x802 ./BSP/RFID_CR95HF/CR95HF.o
 .debug_macro   0x00000000       0x16 ./BSP/RFID_CR95HF/CR95HF.o
 .debug_macro   0x00000000      0x214 ./BSP/RFID_CR95HF/CR95HF.o
 .debug_macro   0x00000000       0x39 ./BSP/RFID_CR95HF/CR95HF.o
 .debug_macro   0x00000000       0x3a ./BSP/RFID_CR95HF/CR95HF.o
 .debug_macro   0x00000000       0x1f ./BSP/RFID_CR95HF/CR95HF.o
 .debug_macro   0x00000000      0x250 ./BSP/RFID_CR95HF/CR95HF.o
 .debug_macro   0x00000000       0xc5 ./BSP/RFID_CR95HF/CR95HF.o
 .debug_macro   0x00000000     0x5642 ./BSP/RFID_CR95HF/CR95HF.o
 .debug_macro   0x00000000      0x1fb ./BSP/RFID_CR95HF/CR95HF.o
 .group         0x00000000        0x8 ./BSP/RFID_CR95HF/CR95UartMapper.o
 .group         0x00000000        0x8 ./BSP/RFID_CR95HF/CR95UartMapper.o
 .group         0x00000000        0x8 ./BSP/RFID_CR95HF/CR95UartMapper.o
 .group         0x00000000        0x8 ./BSP/RFID_CR95HF/CR95UartMapper.o
 .group         0x00000000        0x8 ./BSP/RFID_CR95HF/CR95UartMapper.o
 .group         0x00000000        0x8 ./BSP/RFID_CR95HF/CR95UartMapper.o
 .group         0x00000000        0x8 ./BSP/RFID_CR95HF/CR95UartMapper.o
 .group         0x00000000        0x8 ./BSP/RFID_CR95HF/CR95UartMapper.o
 .group         0x00000000        0x8 ./BSP/RFID_CR95HF/CR95UartMapper.o
 .group         0x00000000        0x8 ./BSP/RFID_CR95HF/CR95UartMapper.o
 .group         0x00000000        0x8 ./BSP/RFID_CR95HF/CR95UartMapper.o
 .group         0x00000000        0x8 ./BSP/RFID_CR95HF/CR95UartMapper.o
 .group         0x00000000        0x8 ./BSP/RFID_CR95HF/CR95UartMapper.o
 .text          0x00000000        0x0 ./BSP/RFID_CR95HF/CR95UartMapper.o
 .data          0x00000000        0x0 ./BSP/RFID_CR95HF/CR95UartMapper.o
 .bss           0x00000000        0x0 ./BSP/RFID_CR95HF/CR95UartMapper.o
 .text.CR95UartEnableTransmitter
                0x00000000       0x54 ./BSP/RFID_CR95HF/CR95UartMapper.o
 .text.CR95UartDisableTransmitter
                0x00000000       0x40 ./BSP/RFID_CR95HF/CR95UartMapper.o
 .text.CR95UartClearAllErrorFlag
                0x00000000       0x20 ./BSP/RFID_CR95HF/CR95UartMapper.o
 .text.CR95UartSendString
                0x00000000       0x2c ./BSP/RFID_CR95HF/CR95UartMapper.o
 .debug_macro   0x00000000      0x802 ./BSP/RFID_CR95HF/CR95UartMapper.o
 .debug_macro   0x00000000       0x16 ./BSP/RFID_CR95HF/CR95UartMapper.o
 .debug_macro   0x00000000      0x214 ./BSP/RFID_CR95HF/CR95UartMapper.o
 .debug_macro   0x00000000       0x39 ./BSP/RFID_CR95HF/CR95UartMapper.o
 .debug_macro   0x00000000       0x3a ./BSP/RFID_CR95HF/CR95UartMapper.o
 .debug_macro   0x00000000       0x1f ./BSP/RFID_CR95HF/CR95UartMapper.o
 .debug_macro   0x00000000      0x250 ./BSP/RFID_CR95HF/CR95UartMapper.o
 .debug_macro   0x00000000       0xc5 ./BSP/RFID_CR95HF/CR95UartMapper.o
 .debug_macro   0x00000000     0x5642 ./BSP/RFID_CR95HF/CR95UartMapper.o
 .debug_macro   0x00000000      0x1fb ./BSP/RFID_CR95HF/CR95UartMapper.o
 .debug_macro   0x00000000       0x65 ./BSP/RFID_CR95HF/CR95UartMapper.o
 .debug_macro   0x00000000       0x5d ./BSP/RFID_CR95HF/CR95UartMapper.o
 .debug_macro   0x00000000       0x10 ./BSP/RFID_CR95HF/CR95UartMapper.o
 .group         0x00000000        0x8 ./BSP/Led/led.o
 .group         0x00000000        0x8 ./BSP/Led/led.o
 .group         0x00000000        0x8 ./BSP/Led/led.o
 .group         0x00000000        0x8 ./BSP/Led/led.o
 .group         0x00000000        0x8 ./BSP/Led/led.o
 .group         0x00000000        0x8 ./BSP/Led/led.o
 .group         0x00000000        0x8 ./BSP/Led/led.o
 .group         0x00000000        0x8 ./BSP/Led/led.o
 .group         0x00000000        0x8 ./BSP/Led/led.o
 .group         0x00000000        0x8 ./BSP/Led/led.o
 .group         0x00000000        0x8 ./BSP/Led/led.o
 .text          0x00000000        0x0 ./BSP/Led/led.o
 .data          0x00000000        0x0 ./BSP/Led/led.o
 .bss           0x00000000        0x0 ./BSP/Led/led.o
 .debug_macro   0x00000000      0x802 ./BSP/Led/led.o
 .debug_macro   0x00000000       0x16 ./BSP/Led/led.o
 .debug_macro   0x00000000      0x214 ./BSP/Led/led.o
 .debug_macro   0x00000000       0x39 ./BSP/Led/led.o
 .debug_macro   0x00000000       0x3a ./BSP/Led/led.o
 .debug_macro   0x00000000       0x1f ./BSP/Led/led.o
 .debug_macro   0x00000000      0x250 ./BSP/Led/led.o
 .debug_macro   0x00000000       0xc5 ./BSP/Led/led.o
 .debug_macro   0x00000000     0x5642 ./BSP/Led/led.o
 .debug_macro   0x00000000      0x1fb ./BSP/Led/led.o
 .group         0x00000000        0x8 ./BSP/FRAM/FM25V20.o
 .group         0x00000000        0x8 ./BSP/FRAM/FM25V20.o
 .group         0x00000000        0x8 ./BSP/FRAM/FM25V20.o
 .group         0x00000000        0x8 ./BSP/FRAM/FM25V20.o
 .group         0x00000000        0x8 ./BSP/FRAM/FM25V20.o
 .group         0x00000000        0x8 ./BSP/FRAM/FM25V20.o
 .group         0x00000000        0x8 ./BSP/FRAM/FM25V20.o
 .group         0x00000000        0x8 ./BSP/FRAM/FM25V20.o
 .group         0x00000000        0x8 ./BSP/FRAM/FM25V20.o
 .group         0x00000000        0x8 ./BSP/FRAM/FM25V20.o
 .group         0x00000000        0x8 ./BSP/FRAM/FM25V20.o
 .group         0x00000000        0x8 ./BSP/FRAM/FM25V20.o
 .text          0x00000000        0x0 ./BSP/FRAM/FM25V20.o
 .data          0x00000000        0x0 ./BSP/FRAM/FM25V20.o
 .bss           0x00000000        0x0 ./BSP/FRAM/FM25V20.o
 .text.FM25V20ReadStatusReg
                0x00000000       0x70 ./BSP/FRAM/FM25V20.o
 .text.FM25V20ReadDeviceId
                0x00000000       0x74 ./BSP/FRAM/FM25V20.o
 .debug_macro   0x00000000      0x802 ./BSP/FRAM/FM25V20.o
 .debug_macro   0x00000000       0x16 ./BSP/FRAM/FM25V20.o
 .debug_macro   0x00000000      0x214 ./BSP/FRAM/FM25V20.o
 .debug_macro   0x00000000       0x39 ./BSP/FRAM/FM25V20.o
 .debug_macro   0x00000000       0x3a ./BSP/FRAM/FM25V20.o
 .debug_macro   0x00000000       0x1f ./BSP/FRAM/FM25V20.o
 .debug_macro   0x00000000      0x250 ./BSP/FRAM/FM25V20.o
 .debug_macro   0x00000000       0xc5 ./BSP/FRAM/FM25V20.o
 .debug_macro   0x00000000     0x5642 ./BSP/FRAM/FM25V20.o
 .debug_macro   0x00000000      0x1fb ./BSP/FRAM/FM25V20.o
 .debug_macro   0x00000000       0x44 ./BSP/FRAM/FM25V20.o
 .group         0x00000000        0x8 ./BSP/FRAM/FM25V20MemTest.o
 .group         0x00000000        0x8 ./BSP/FRAM/FM25V20MemTest.o
 .group         0x00000000        0x8 ./BSP/FRAM/FM25V20MemTest.o
 .group         0x00000000        0x8 ./BSP/FRAM/FM25V20MemTest.o
 .group         0x00000000        0x8 ./BSP/FRAM/FM25V20MemTest.o
 .group         0x00000000        0x8 ./BSP/FRAM/FM25V20MemTest.o
 .group         0x00000000        0x8 ./BSP/FRAM/FM25V20MemTest.o
 .group         0x00000000        0x8 ./BSP/FRAM/FM25V20MemTest.o
 .group         0x00000000        0x8 ./BSP/FRAM/FM25V20MemTest.o
 .group         0x00000000        0x8 ./BSP/FRAM/FM25V20MemTest.o
 .group         0x00000000        0x8 ./BSP/FRAM/FM25V20MemTest.o
 .group         0x00000000        0x8 ./BSP/FRAM/FM25V20MemTest.o
 .text          0x00000000        0x0 ./BSP/FRAM/FM25V20MemTest.o
 .data          0x00000000        0x0 ./BSP/FRAM/FM25V20MemTest.o
 .bss           0x00000000        0x0 ./BSP/FRAM/FM25V20MemTest.o
 .text.FM25V20MemTest_Main
                0x00000000       0xcc ./BSP/FRAM/FM25V20MemTest.o
 .rodata        0x00000000       0x30 ./BSP/FRAM/FM25V20MemTest.o
 .text.FM25V20MemTest_Set
                0x00000000       0xd4 ./BSP/FRAM/FM25V20MemTest.o
 .text.FM25V20MemTest_Clear
                0x00000000       0xd0 ./BSP/FRAM/FM25V20MemTest.o
 .text.FM25V20MemTest_HighFreqUp
                0x00000000       0xd4 ./BSP/FRAM/FM25V20MemTest.o
 .text.FM25V20MemTest_HighFreqDown
                0x00000000       0xd4 ./BSP/FRAM/FM25V20MemTest.o
 .text.FM25V20MemTest_PulseP
                0x00000000      0x154 ./BSP/FRAM/FM25V20MemTest.o
 .text.FM25V20MemTest_PulseN
                0x00000000      0x154 ./BSP/FRAM/FM25V20MemTest.o
 .debug_info    0x00000000      0x410 ./BSP/FRAM/FM25V20MemTest.o
 .debug_abbrev  0x00000000       0xe9 ./BSP/FRAM/FM25V20MemTest.o
 .debug_aranges
                0x00000000       0x50 ./BSP/FRAM/FM25V20MemTest.o
 .debug_ranges  0x00000000       0x40 ./BSP/FRAM/FM25V20MemTest.o
 .debug_macro   0x00000000       0xb6 ./BSP/FRAM/FM25V20MemTest.o
 .debug_macro   0x00000000      0x802 ./BSP/FRAM/FM25V20MemTest.o
 .debug_macro   0x00000000       0x16 ./BSP/FRAM/FM25V20MemTest.o
 .debug_macro   0x00000000      0x214 ./BSP/FRAM/FM25V20MemTest.o
 .debug_macro   0x00000000       0x39 ./BSP/FRAM/FM25V20MemTest.o
 .debug_macro   0x00000000       0x3a ./BSP/FRAM/FM25V20MemTest.o
 .debug_macro   0x00000000       0x1f ./BSP/FRAM/FM25V20MemTest.o
 .debug_macro   0x00000000      0x250 ./BSP/FRAM/FM25V20MemTest.o
 .debug_macro   0x00000000       0xc5 ./BSP/FRAM/FM25V20MemTest.o
 .debug_macro   0x00000000     0x5642 ./BSP/FRAM/FM25V20MemTest.o
 .debug_macro   0x00000000      0x1fb ./BSP/FRAM/FM25V20MemTest.o
 .debug_macro   0x00000000       0x44 ./BSP/FRAM/FM25V20MemTest.o
 .debug_macro   0x00000000       0x84 ./BSP/FRAM/FM25V20MemTest.o
 .debug_line    0x00000000      0x36c ./BSP/FRAM/FM25V20MemTest.o
 .debug_str     0x00000000    0x1efbc ./BSP/FRAM/FM25V20MemTest.o
 .comment       0x00000000       0x2b ./BSP/FRAM/FM25V20MemTest.o
 .ARM.attributes
                0x00000000       0x32 ./BSP/FRAM/FM25V20MemTest.o
 .debug_frame   0x00000000       0xf0 ./BSP/FRAM/FM25V20MemTest.o
 .group         0x00000000        0x8 ./BSP/Display/display.o
 .group         0x00000000        0x8 ./BSP/Display/display.o
 .group         0x00000000        0x8 ./BSP/Display/display.o
 .group         0x00000000        0x8 ./BSP/Display/display.o
 .group         0x00000000        0x8 ./BSP/Display/display.o
 .group         0x00000000        0x8 ./BSP/Display/display.o
 .group         0x00000000        0x8 ./BSP/Display/display.o
 .group         0x00000000        0x8 ./BSP/Display/display.o
 .group         0x00000000        0x8 ./BSP/Display/display.o
 .group         0x00000000        0x8 ./BSP/Display/display.o
 .group         0x00000000        0x8 ./BSP/Display/display.o
 .group         0x00000000        0x8 ./BSP/Display/display.o
 .group         0x00000000        0x8 ./BSP/Display/display.o
 .group         0x00000000        0x8 ./BSP/Display/display.o
 .text          0x00000000        0x0 ./BSP/Display/display.o
 .data          0x00000000        0x0 ./BSP/Display/display.o
 .bss           0x00000000        0x0 ./BSP/Display/display.o
 .debug_macro   0x00000000      0x802 ./BSP/Display/display.o
 .debug_macro   0x00000000       0x16 ./BSP/Display/display.o
 .debug_macro   0x00000000      0x214 ./BSP/Display/display.o
 .debug_macro   0x00000000       0x39 ./BSP/Display/display.o
 .debug_macro   0x00000000       0x3a ./BSP/Display/display.o
 .debug_macro   0x00000000       0x1f ./BSP/Display/display.o
 .debug_macro   0x00000000      0x250 ./BSP/Display/display.o
 .debug_macro   0x00000000       0xc5 ./BSP/Display/display.o
 .debug_macro   0x00000000     0x5642 ./BSP/Display/display.o
 .debug_macro   0x00000000      0x1fb ./BSP/Display/display.o
 .debug_macro   0x00000000       0x44 ./BSP/Display/display.o
 .debug_macro   0x00000000       0x6a ./BSP/Display/display.o
 .debug_macro   0x00000000       0xca ./BSP/Display/display.o
 .group         0x00000000        0x8 ./BSP/Button/button.o
 .group         0x00000000        0x8 ./BSP/Button/button.o
 .group         0x00000000        0x8 ./BSP/Button/button.o
 .group         0x00000000        0x8 ./BSP/Button/button.o
 .group         0x00000000        0x8 ./BSP/Button/button.o
 .group         0x00000000        0x8 ./BSP/Button/button.o
 .group         0x00000000        0x8 ./BSP/Button/button.o
 .group         0x00000000        0x8 ./BSP/Button/button.o
 .group         0x00000000        0x8 ./BSP/Button/button.o
 .group         0x00000000        0x8 ./BSP/Button/button.o
 .group         0x00000000        0x8 ./BSP/Button/button.o
 .text          0x00000000        0x0 ./BSP/Button/button.o
 .data          0x00000000        0x0 ./BSP/Button/button.o
 .bss           0x00000000        0x0 ./BSP/Button/button.o
 .debug_macro   0x00000000      0x802 ./BSP/Button/button.o
 .debug_macro   0x00000000       0x16 ./BSP/Button/button.o
 .debug_macro   0x00000000      0x214 ./BSP/Button/button.o
 .debug_macro   0x00000000       0x39 ./BSP/Button/button.o
 .debug_macro   0x00000000       0x3a ./BSP/Button/button.o
 .debug_macro   0x00000000       0x1f ./BSP/Button/button.o
 .debug_macro   0x00000000      0x250 ./BSP/Button/button.o
 .debug_macro   0x00000000       0xc5 ./BSP/Button/button.o
 .debug_macro   0x00000000     0x5642 ./BSP/Button/button.o
 .debug_macro   0x00000000      0x1fb ./BSP/Button/button.o
 .group         0x00000000        0x8 ./BSP/BatteryManagement/BQ27510DRZRG2.o
 .group         0x00000000        0x8 ./BSP/BatteryManagement/BQ27510DRZRG2.o
 .group         0x00000000        0x8 ./BSP/BatteryManagement/BQ27510DRZRG2.o
 .group         0x00000000        0x8 ./BSP/BatteryManagement/BQ27510DRZRG2.o
 .group         0x00000000        0x8 ./BSP/BatteryManagement/BQ27510DRZRG2.o
 .group         0x00000000        0x8 ./BSP/BatteryManagement/BQ27510DRZRG2.o
 .group         0x00000000        0x8 ./BSP/BatteryManagement/BQ27510DRZRG2.o
 .group         0x00000000        0x8 ./BSP/BatteryManagement/BQ27510DRZRG2.o
 .group         0x00000000        0x8 ./BSP/BatteryManagement/BQ27510DRZRG2.o
 .group         0x00000000        0x8 ./BSP/BatteryManagement/BQ27510DRZRG2.o
 .group         0x00000000        0x8 ./BSP/BatteryManagement/BQ27510DRZRG2.o
 .group         0x00000000        0x8 ./BSP/BatteryManagement/BQ27510DRZRG2.o
 .text          0x00000000        0x0 ./BSP/BatteryManagement/BQ27510DRZRG2.o
 .data          0x00000000        0x0 ./BSP/BatteryManagement/BQ27510DRZRG2.o
 .bss           0x00000000        0x0 ./BSP/BatteryManagement/BQ27510DRZRG2.o
 .text.BQ_getStandbyCurrent
                0x00000000       0x74 ./BSP/BatteryManagement/BQ27510DRZRG2.o
 .debug_macro   0x00000000      0x802 ./BSP/BatteryManagement/BQ27510DRZRG2.o
 .debug_macro   0x00000000       0x16 ./BSP/BatteryManagement/BQ27510DRZRG2.o
 .debug_macro   0x00000000      0x214 ./BSP/BatteryManagement/BQ27510DRZRG2.o
 .debug_macro   0x00000000       0x39 ./BSP/BatteryManagement/BQ27510DRZRG2.o
 .debug_macro   0x00000000       0x3a ./BSP/BatteryManagement/BQ27510DRZRG2.o
 .debug_macro   0x00000000       0x1f ./BSP/BatteryManagement/BQ27510DRZRG2.o
 .debug_macro   0x00000000      0x250 ./BSP/BatteryManagement/BQ27510DRZRG2.o
 .debug_macro   0x00000000       0xc5 ./BSP/BatteryManagement/BQ27510DRZRG2.o
 .debug_macro   0x00000000     0x5642 ./BSP/BatteryManagement/BQ27510DRZRG2.o
 .debug_macro   0x00000000      0x1fb ./BSP/BatteryManagement/BQ27510DRZRG2.o
 .debug_macro   0x00000000       0x3a ./BSP/BatteryManagement/BQ27510DRZRG2.o
 .group         0x00000000        0x8 ./BSP/BatteryManagement/LTC4160.o
 .group         0x00000000        0x8 ./BSP/BatteryManagement/LTC4160.o
 .group         0x00000000        0x8 ./BSP/BatteryManagement/LTC4160.o
 .group         0x00000000        0x8 ./BSP/BatteryManagement/LTC4160.o
 .group         0x00000000        0x8 ./BSP/BatteryManagement/LTC4160.o
 .group         0x00000000        0x8 ./BSP/BatteryManagement/LTC4160.o
 .group         0x00000000        0x8 ./BSP/BatteryManagement/LTC4160.o
 .group         0x00000000        0x8 ./BSP/BatteryManagement/LTC4160.o
 .group         0x00000000        0x8 ./BSP/BatteryManagement/LTC4160.o
 .group         0x00000000        0x8 ./BSP/BatteryManagement/LTC4160.o
 .group         0x00000000        0x8 ./BSP/BatteryManagement/LTC4160.o
 .text          0x00000000        0x0 ./BSP/BatteryManagement/LTC4160.o
 .data          0x00000000        0x0 ./BSP/BatteryManagement/LTC4160.o
 .bss           0x00000000        0x0 ./BSP/BatteryManagement/LTC4160.o
 .debug_macro   0x00000000      0x802 ./BSP/BatteryManagement/LTC4160.o
 .debug_macro   0x00000000       0x16 ./BSP/BatteryManagement/LTC4160.o
 .debug_macro   0x00000000      0x214 ./BSP/BatteryManagement/LTC4160.o
 .debug_macro   0x00000000       0x39 ./BSP/BatteryManagement/LTC4160.o
 .debug_macro   0x00000000       0x3a ./BSP/BatteryManagement/LTC4160.o
 .debug_macro   0x00000000       0x1f ./BSP/BatteryManagement/LTC4160.o
 .debug_macro   0x00000000      0x250 ./BSP/BatteryManagement/LTC4160.o
 .debug_macro   0x00000000       0xc5 ./BSP/BatteryManagement/LTC4160.o
 .debug_macro   0x00000000     0x5642 ./BSP/BatteryManagement/LTC4160.o
 .debug_macro   0x00000000      0x1fb ./BSP/BatteryManagement/LTC4160.o
 .group         0x00000000        0x8 ./Application/UsbManager/UsbManager.o
 .group         0x00000000        0x8 ./Application/UsbManager/UsbManager.o
 .group         0x00000000        0x8 ./Application/UsbManager/UsbManager.o
 .group         0x00000000        0x8 ./Application/UsbManager/UsbManager.o
 .group         0x00000000        0x8 ./Application/UsbManager/UsbManager.o
 .group         0x00000000        0x8 ./Application/UsbManager/UsbManager.o
 .group         0x00000000        0x8 ./Application/UsbManager/UsbManager.o
 .group         0x00000000        0x8 ./Application/UsbManager/UsbManager.o
 .group         0x00000000        0x8 ./Application/UsbManager/UsbManager.o
 .group         0x00000000        0x8 ./Application/UsbManager/UsbManager.o
 .group         0x00000000        0x8 ./Application/UsbManager/UsbManager.o
 .group         0x00000000        0x8 ./Application/UsbManager/UsbManager.o
 .group         0x00000000        0x8 ./Application/UsbManager/UsbManager.o
 .group         0x00000000        0x8 ./Application/UsbManager/UsbManager.o
 .group         0x00000000        0x8 ./Application/UsbManager/UsbManager.o
 .group         0x00000000        0x8 ./Application/UsbManager/UsbManager.o
 .group         0x00000000        0x8 ./Application/UsbManager/UsbManager.o
 .group         0x00000000        0x8 ./Application/UsbManager/UsbManager.o
 .group         0x00000000        0x8 ./Application/UsbManager/UsbManager.o
 .group         0x00000000        0x8 ./Application/UsbManager/UsbManager.o
 .group         0x00000000        0x8 ./Application/UsbManager/UsbManager.o
 .group         0x00000000        0x8 ./Application/UsbManager/UsbManager.o
 .group         0x00000000        0x8 ./Application/UsbManager/UsbManager.o
 .group         0x00000000        0x8 ./Application/UsbManager/UsbManager.o
 .group         0x00000000        0x8 ./Application/UsbManager/UsbManager.o
 .group         0x00000000        0x8 ./Application/UsbManager/UsbManager.o
 .group         0x00000000        0x8 ./Application/UsbManager/UsbManager.o
 .group         0x00000000        0x8 ./Application/UsbManager/UsbManager.o
 .group         0x00000000        0x8 ./Application/UsbManager/UsbManager.o
 .group         0x00000000        0x8 ./Application/UsbManager/UsbManager.o
 .group         0x00000000        0x8 ./Application/UsbManager/UsbManager.o
 .group         0x00000000        0x8 ./Application/UsbManager/UsbManager.o
 .group         0x00000000        0x8 ./Application/UsbManager/UsbManager.o
 .group         0x00000000        0x8 ./Application/UsbManager/UsbManager.o
 .group         0x00000000        0x8 ./Application/UsbManager/UsbManager.o
 .group         0x00000000        0x8 ./Application/UsbManager/UsbManager.o
 .text          0x00000000        0x0 ./Application/UsbManager/UsbManager.o
 .data          0x00000000        0x0 ./Application/UsbManager/UsbManager.o
 .bss           0x00000000        0x0 ./Application/UsbManager/UsbManager.o
 .text.UsbManagerInit
                0x00000000       0x4c ./Application/UsbManager/UsbManager.o
 .debug_macro   0x00000000      0x802 ./Application/UsbManager/UsbManager.o
 .debug_macro   0x00000000       0x16 ./Application/UsbManager/UsbManager.o
 .debug_macro   0x00000000      0x214 ./Application/UsbManager/UsbManager.o
 .debug_macro   0x00000000       0x39 ./Application/UsbManager/UsbManager.o
 .debug_macro   0x00000000       0x3a ./Application/UsbManager/UsbManager.o
 .debug_macro   0x00000000       0x1f ./Application/UsbManager/UsbManager.o
 .debug_macro   0x00000000      0x250 ./Application/UsbManager/UsbManager.o
 .debug_macro   0x00000000       0xc5 ./Application/UsbManager/UsbManager.o
 .debug_macro   0x00000000     0x5642 ./Application/UsbManager/UsbManager.o
 .debug_macro   0x00000000      0x1fb ./Application/UsbManager/UsbManager.o
 .debug_macro   0x00000000       0x34 ./Application/UsbManager/UsbManager.o
 .debug_macro   0x00000000       0x48 ./Application/UsbManager/UsbManager.o
 .debug_macro   0x00000000       0x3a ./Application/UsbManager/UsbManager.o
 .debug_macro   0x00000000       0x8e ./Application/UsbManager/UsbManager.o
 .debug_macro   0x00000000       0x84 ./Application/UsbManager/UsbManager.o
 .debug_macro   0x00000000       0x5d ./Application/UsbManager/UsbManager.o
 .debug_macro   0x00000000       0x10 ./Application/UsbManager/UsbManager.o
 .debug_macro   0x00000000       0x1c ./Application/UsbManager/UsbManager.o
 .debug_macro   0x00000000       0x6a ./Application/UsbManager/UsbManager.o
 .debug_macro   0x00000000       0xca ./Application/UsbManager/UsbManager.o
 .debug_macro   0x00000000       0x3b ./Application/UsbManager/UsbManager.o
 .group         0x00000000        0x8 ./Application/RFIDManager/RFIDManager.o
 .group         0x00000000        0x8 ./Application/RFIDManager/RFIDManager.o
 .group         0x00000000        0x8 ./Application/RFIDManager/RFIDManager.o
 .group         0x00000000        0x8 ./Application/RFIDManager/RFIDManager.o
 .group         0x00000000        0x8 ./Application/RFIDManager/RFIDManager.o
 .group         0x00000000        0x8 ./Application/RFIDManager/RFIDManager.o
 .group         0x00000000        0x8 ./Application/RFIDManager/RFIDManager.o
 .group         0x00000000        0x8 ./Application/RFIDManager/RFIDManager.o
 .group         0x00000000        0x8 ./Application/RFIDManager/RFIDManager.o
 .group         0x00000000        0x8 ./Application/RFIDManager/RFIDManager.o
 .group         0x00000000        0x8 ./Application/RFIDManager/RFIDManager.o
 .group         0x00000000        0x8 ./Application/RFIDManager/RFIDManager.o
 .group         0x00000000        0x8 ./Application/RFIDManager/RFIDManager.o
 .group         0x00000000        0x8 ./Application/RFIDManager/RFIDManager.o
 .group         0x00000000        0x8 ./Application/RFIDManager/RFIDManager.o
 .group         0x00000000        0x8 ./Application/RFIDManager/RFIDManager.o
 .group         0x00000000        0x8 ./Application/RFIDManager/RFIDManager.o
 .group         0x00000000        0x8 ./Application/RFIDManager/RFIDManager.o
 .group         0x00000000        0x8 ./Application/RFIDManager/RFIDManager.o
 .group         0x00000000        0x8 ./Application/RFIDManager/RFIDManager.o
 .group         0x00000000        0x8 ./Application/RFIDManager/RFIDManager.o
 .group         0x00000000        0x8 ./Application/RFIDManager/RFIDManager.o
 .group         0x00000000        0x8 ./Application/RFIDManager/RFIDManager.o
 .group         0x00000000        0x8 ./Application/RFIDManager/RFIDManager.o
 .group         0x00000000        0x8 ./Application/RFIDManager/RFIDManager.o
 .group         0x00000000        0x8 ./Application/RFIDManager/RFIDManager.o
 .group         0x00000000        0x8 ./Application/RFIDManager/RFIDManager.o
 .group         0x00000000        0x8 ./Application/RFIDManager/RFIDManager.o
 .group         0x00000000        0x8 ./Application/RFIDManager/RFIDManager.o
 .group         0x00000000        0x8 ./Application/RFIDManager/RFIDManager.o
 .group         0x00000000        0x8 ./Application/RFIDManager/RFIDManager.o
 .group         0x00000000        0x8 ./Application/RFIDManager/RFIDManager.o
 .group         0x00000000        0x8 ./Application/RFIDManager/RFIDManager.o
 .group         0x00000000        0x8 ./Application/RFIDManager/RFIDManager.o
 .group         0x00000000        0x8 ./Application/RFIDManager/RFIDManager.o
 .group         0x00000000        0x8 ./Application/RFIDManager/RFIDManager.o
 .text          0x00000000        0x0 ./Application/RFIDManager/RFIDManager.o
 .data          0x00000000        0x0 ./Application/RFIDManager/RFIDManager.o
 .bss           0x00000000        0x0 ./Application/RFIDManager/RFIDManager.o
 .debug_macro   0x00000000      0x802 ./Application/RFIDManager/RFIDManager.o
 .debug_macro   0x00000000       0x16 ./Application/RFIDManager/RFIDManager.o
 .debug_macro   0x00000000      0x214 ./Application/RFIDManager/RFIDManager.o
 .debug_macro   0x00000000       0x39 ./Application/RFIDManager/RFIDManager.o
 .debug_macro   0x00000000       0x3a ./Application/RFIDManager/RFIDManager.o
 .debug_macro   0x00000000       0x1f ./Application/RFIDManager/RFIDManager.o
 .debug_macro   0x00000000      0x250 ./Application/RFIDManager/RFIDManager.o
 .debug_macro   0x00000000       0xc5 ./Application/RFIDManager/RFIDManager.o
 .debug_macro   0x00000000     0x5642 ./Application/RFIDManager/RFIDManager.o
 .debug_macro   0x00000000      0x1fb ./Application/RFIDManager/RFIDManager.o
 .debug_macro   0x00000000       0x65 ./Application/RFIDManager/RFIDManager.o
 .debug_macro   0x00000000       0x5d ./Application/RFIDManager/RFIDManager.o
 .debug_macro   0x00000000       0x10 ./Application/RFIDManager/RFIDManager.o
 .debug_macro   0x00000000       0x34 ./Application/RFIDManager/RFIDManager.o
 .debug_macro   0x00000000       0x48 ./Application/RFIDManager/RFIDManager.o
 .debug_macro   0x00000000       0x1c ./Application/RFIDManager/RFIDManager.o
 .debug_macro   0x00000000       0x3a ./Application/RFIDManager/RFIDManager.o
 .debug_macro   0x00000000       0x8e ./Application/RFIDManager/RFIDManager.o
 .debug_macro   0x00000000       0x81 ./Application/RFIDManager/RFIDManager.o
 .debug_macro   0x00000000       0x4a ./Application/RFIDManager/RFIDManager.o
 .debug_macro   0x00000000       0x6a ./Application/RFIDManager/RFIDManager.o
 .debug_macro   0x00000000       0xca ./Application/RFIDManager/RFIDManager.o
 .debug_macro   0x00000000       0x3b ./Application/RFIDManager/RFIDManager.o
 .debug_macro   0x00000000       0x52 ./Application/RFIDManager/RFIDManager.o
 .debug_macro   0x00000000       0x28 ./Application/RFIDManager/RFIDManager.o
 .debug_macro   0x00000000       0x4a ./Application/RFIDManager/RFIDManager.o
 .debug_macro   0x00000000       0x84 ./Application/RFIDManager/RFIDManager.o
 .debug_macro   0x00000000       0x2e ./Application/RFIDManager/RFIDManager.o
 .debug_macro   0x00000000       0x3a ./Application/RFIDManager/RFIDManager.o
 .debug_macro   0x00000000      0x196 ./Application/RFIDManager/RFIDManager.o
 .debug_macro   0x00000000       0x7c ./Application/RFIDManager/RFIDManager.o
 .debug_macro   0x00000000       0x16 ./Application/RFIDManager/RFIDManager.o
 .debug_macro   0x00000000       0x10 ./Application/RFIDManager/RFIDManager.o
 .debug_macro   0x00000000       0x16 ./Application/RFIDManager/RFIDManager.o
 .debug_macro   0x00000000       0x8e ./Application/RFIDManager/RFIDManager.o
 .group         0x00000000        0x8 ./Application/PowerManager/PowerManager.o
 .group         0x00000000        0x8 ./Application/PowerManager/PowerManager.o
 .group         0x00000000        0x8 ./Application/PowerManager/PowerManager.o
 .group         0x00000000        0x8 ./Application/PowerManager/PowerManager.o
 .group         0x00000000        0x8 ./Application/PowerManager/PowerManager.o
 .group         0x00000000        0x8 ./Application/PowerManager/PowerManager.o
 .group         0x00000000        0x8 ./Application/PowerManager/PowerManager.o
 .group         0x00000000        0x8 ./Application/PowerManager/PowerManager.o
 .group         0x00000000        0x8 ./Application/PowerManager/PowerManager.o
 .group         0x00000000        0x8 ./Application/PowerManager/PowerManager.o
 .group         0x00000000        0x8 ./Application/PowerManager/PowerManager.o
 .group         0x00000000        0x8 ./Application/PowerManager/PowerManager.o
 .group         0x00000000        0x8 ./Application/PowerManager/PowerManager.o
 .group         0x00000000        0x8 ./Application/PowerManager/PowerManager.o
 .group         0x00000000        0x8 ./Application/PowerManager/PowerManager.o
 .group         0x00000000        0x8 ./Application/PowerManager/PowerManager.o
 .group         0x00000000        0x8 ./Application/PowerManager/PowerManager.o
 .group         0x00000000        0x8 ./Application/PowerManager/PowerManager.o
 .group         0x00000000        0x8 ./Application/PowerManager/PowerManager.o
 .group         0x00000000        0x8 ./Application/PowerManager/PowerManager.o
 .group         0x00000000        0x8 ./Application/PowerManager/PowerManager.o
 .group         0x00000000        0x8 ./Application/PowerManager/PowerManager.o
 .group         0x00000000        0x8 ./Application/PowerManager/PowerManager.o
 .group         0x00000000        0x8 ./Application/PowerManager/PowerManager.o
 .group         0x00000000        0x8 ./Application/PowerManager/PowerManager.o
 .group         0x00000000        0x8 ./Application/PowerManager/PowerManager.o
 .group         0x00000000        0x8 ./Application/PowerManager/PowerManager.o
 .group         0x00000000        0x8 ./Application/PowerManager/PowerManager.o
 .group         0x00000000        0x8 ./Application/PowerManager/PowerManager.o
 .group         0x00000000        0x8 ./Application/PowerManager/PowerManager.o
 .group         0x00000000        0x8 ./Application/PowerManager/PowerManager.o
 .group         0x00000000        0x8 ./Application/PowerManager/PowerManager.o
 .group         0x00000000        0x8 ./Application/PowerManager/PowerManager.o
 .group         0x00000000        0x8 ./Application/PowerManager/PowerManager.o
 .group         0x00000000        0x8 ./Application/PowerManager/PowerManager.o
 .group         0x00000000        0x8 ./Application/PowerManager/PowerManager.o
 .text          0x00000000        0x0 ./Application/PowerManager/PowerManager.o
 .data          0x00000000        0x0 ./Application/PowerManager/PowerManager.o
 .bss           0x00000000        0x0 ./Application/PowerManager/PowerManager.o
 .text.PowerManagerSendBatteryInfo
                0x00000000      0x1a0 ./Application/PowerManager/PowerManager.o
 .debug_macro   0x00000000      0x802 ./Application/PowerManager/PowerManager.o
 .debug_macro   0x00000000       0x16 ./Application/PowerManager/PowerManager.o
 .debug_macro   0x00000000      0x214 ./Application/PowerManager/PowerManager.o
 .debug_macro   0x00000000       0x39 ./Application/PowerManager/PowerManager.o
 .debug_macro   0x00000000       0x3a ./Application/PowerManager/PowerManager.o
 .debug_macro   0x00000000       0x1f ./Application/PowerManager/PowerManager.o
 .debug_macro   0x00000000      0x250 ./Application/PowerManager/PowerManager.o
 .debug_macro   0x00000000       0xc5 ./Application/PowerManager/PowerManager.o
 .debug_macro   0x00000000     0x5642 ./Application/PowerManager/PowerManager.o
 .debug_macro   0x00000000      0x1fb ./Application/PowerManager/PowerManager.o
 .debug_macro   0x00000000       0x3a ./Application/PowerManager/PowerManager.o
 .debug_macro   0x00000000       0x8e ./Application/PowerManager/PowerManager.o
 .debug_macro   0x00000000       0x81 ./Application/PowerManager/PowerManager.o
 .debug_macro   0x00000000       0x4a ./Application/PowerManager/PowerManager.o
 .debug_macro   0x00000000       0x6a ./Application/PowerManager/PowerManager.o
 .debug_macro   0x00000000       0xca ./Application/PowerManager/PowerManager.o
 .debug_macro   0x00000000       0x3b ./Application/PowerManager/PowerManager.o
 .debug_macro   0x00000000       0x57 ./Application/PowerManager/PowerManager.o
 .debug_macro   0x00000000       0x52 ./Application/PowerManager/PowerManager.o
 .debug_macro   0x00000000       0x28 ./Application/PowerManager/PowerManager.o
 .debug_macro   0x00000000       0x4a ./Application/PowerManager/PowerManager.o
 .debug_macro   0x00000000       0x84 ./Application/PowerManager/PowerManager.o
 .debug_macro   0x00000000       0x2e ./Application/PowerManager/PowerManager.o
 .debug_macro   0x00000000       0x3a ./Application/PowerManager/PowerManager.o
 .debug_macro   0x00000000       0x34 ./Application/PowerManager/PowerManager.o
 .debug_macro   0x00000000       0x48 ./Application/PowerManager/PowerManager.o
 .debug_macro   0x00000000      0x196 ./Application/PowerManager/PowerManager.o
 .debug_macro   0x00000000       0x7c ./Application/PowerManager/PowerManager.o
 .debug_macro   0x00000000       0x16 ./Application/PowerManager/PowerManager.o
 .debug_macro   0x00000000       0x6b ./Application/PowerManager/PowerManager.o
 .debug_macro   0x00000000       0x5d ./Application/PowerManager/PowerManager.o
 .debug_macro   0x00000000       0x10 ./Application/PowerManager/PowerManager.o
 .debug_macro   0x00000000       0x1c ./Application/PowerManager/PowerManager.o
 .debug_macro   0x00000000       0x16 ./Application/PowerManager/PowerManager.o
 .debug_macro   0x00000000       0x8e ./Application/PowerManager/PowerManager.o
 .debug_macro   0x00000000       0x10 ./Application/PowerManager/PowerManager.o
 .group         0x00000000        0x8 ./Application/MemoryManager/MemoryManager.o
 .group         0x00000000        0x8 ./Application/MemoryManager/MemoryManager.o
 .group         0x00000000        0x8 ./Application/MemoryManager/MemoryManager.o
 .group         0x00000000        0x8 ./Application/MemoryManager/MemoryManager.o
 .group         0x00000000        0x8 ./Application/MemoryManager/MemoryManager.o
 .group         0x00000000        0x8 ./Application/MemoryManager/MemoryManager.o
 .group         0x00000000        0x8 ./Application/MemoryManager/MemoryManager.o
 .group         0x00000000        0x8 ./Application/MemoryManager/MemoryManager.o
 .group         0x00000000        0x8 ./Application/MemoryManager/MemoryManager.o
 .group         0x00000000        0x8 ./Application/MemoryManager/MemoryManager.o
 .group         0x00000000        0x8 ./Application/MemoryManager/MemoryManager.o
 .group         0x00000000        0x8 ./Application/MemoryManager/MemoryManager.o
 .group         0x00000000        0x8 ./Application/MemoryManager/MemoryManager.o
 .group         0x00000000        0x8 ./Application/MemoryManager/MemoryManager.o
 .text          0x00000000        0x0 ./Application/MemoryManager/MemoryManager.o
 .data          0x00000000        0x0 ./Application/MemoryManager/MemoryManager.o
 .bss           0x00000000        0x0 ./Application/MemoryManager/MemoryManager.o
 .debug_macro   0x00000000      0x802 ./Application/MemoryManager/MemoryManager.o
 .debug_macro   0x00000000       0x16 ./Application/MemoryManager/MemoryManager.o
 .debug_macro   0x00000000      0x214 ./Application/MemoryManager/MemoryManager.o
 .debug_macro   0x00000000       0x39 ./Application/MemoryManager/MemoryManager.o
 .debug_macro   0x00000000       0x3a ./Application/MemoryManager/MemoryManager.o
 .debug_macro   0x00000000       0x1f ./Application/MemoryManager/MemoryManager.o
 .debug_macro   0x00000000      0x250 ./Application/MemoryManager/MemoryManager.o
 .debug_macro   0x00000000       0xc5 ./Application/MemoryManager/MemoryManager.o
 .debug_macro   0x00000000     0x5642 ./Application/MemoryManager/MemoryManager.o
 .debug_macro   0x00000000      0x1fb ./Application/MemoryManager/MemoryManager.o
 .debug_macro   0x00000000       0x44 ./Application/MemoryManager/MemoryManager.o
 .debug_macro   0x00000000       0x84 ./Application/MemoryManager/MemoryManager.o
 .debug_macro   0x00000000      0x196 ./Application/MemoryManager/MemoryManager.o
 .debug_macro   0x00000000       0x7c ./Application/MemoryManager/MemoryManager.o
 .group         0x00000000        0x8 ./Application/Global/globalParameters.o
 .text          0x00000000        0x0 ./Application/Global/globalParameters.o
 .data          0x00000000        0x0 ./Application/Global/globalParameters.o
 .bss           0x00000000        0x0 ./Application/Global/globalParameters.o
 .debug_info    0x00000000       0x21 ./Application/Global/globalParameters.o
 .debug_abbrev  0x00000000       0x13 ./Application/Global/globalParameters.o
 .debug_aranges
                0x00000000       0x18 ./Application/Global/globalParameters.o
 .debug_macro   0x00000000       0x11 ./Application/Global/globalParameters.o
 .debug_macro   0x00000000      0x802 ./Application/Global/globalParameters.o
 .debug_line    0x00000000       0x49 ./Application/Global/globalParameters.o
 .debug_str     0x00000000     0x2263 ./Application/Global/globalParameters.o
 .comment       0x00000000       0x2b ./Application/Global/globalParameters.o
 .ARM.attributes
                0x00000000       0x32 ./Application/Global/globalParameters.o
 .group         0x00000000        0x8 ./Application/ButtonManager/ButtonManager.o
 .group         0x00000000        0x8 ./Application/ButtonManager/ButtonManager.o
 .group         0x00000000        0x8 ./Application/ButtonManager/ButtonManager.o
 .group         0x00000000        0x8 ./Application/ButtonManager/ButtonManager.o
 .group         0x00000000        0x8 ./Application/ButtonManager/ButtonManager.o
 .group         0x00000000        0x8 ./Application/ButtonManager/ButtonManager.o
 .group         0x00000000        0x8 ./Application/ButtonManager/ButtonManager.o
 .group         0x00000000        0x8 ./Application/ButtonManager/ButtonManager.o
 .group         0x00000000        0x8 ./Application/ButtonManager/ButtonManager.o
 .group         0x00000000        0x8 ./Application/ButtonManager/ButtonManager.o
 .group         0x00000000        0x8 ./Application/ButtonManager/ButtonManager.o
 .group         0x00000000        0x8 ./Application/ButtonManager/ButtonManager.o
 .group         0x00000000        0x8 ./Application/ButtonManager/ButtonManager.o
 .group         0x00000000        0x8 ./Application/ButtonManager/ButtonManager.o
 .group         0x00000000        0x8 ./Application/ButtonManager/ButtonManager.o
 .group         0x00000000        0x8 ./Application/ButtonManager/ButtonManager.o
 .group         0x00000000        0x8 ./Application/ButtonManager/ButtonManager.o
 .group         0x00000000        0x8 ./Application/ButtonManager/ButtonManager.o
 .group         0x00000000        0x8 ./Application/ButtonManager/ButtonManager.o
 .group         0x00000000        0x8 ./Application/ButtonManager/ButtonManager.o
 .group         0x00000000        0x8 ./Application/ButtonManager/ButtonManager.o
 .group         0x00000000        0x8 ./Application/ButtonManager/ButtonManager.o
 .group         0x00000000        0x8 ./Application/ButtonManager/ButtonManager.o
 .group         0x00000000        0x8 ./Application/ButtonManager/ButtonManager.o
 .group         0x00000000        0x8 ./Application/ButtonManager/ButtonManager.o
 .group         0x00000000        0x8 ./Application/ButtonManager/ButtonManager.o
 .group         0x00000000        0x8 ./Application/ButtonManager/ButtonManager.o
 .group         0x00000000        0x8 ./Application/ButtonManager/ButtonManager.o
 .group         0x00000000        0x8 ./Application/ButtonManager/ButtonManager.o
 .group         0x00000000        0x8 ./Application/ButtonManager/ButtonManager.o
 .group         0x00000000        0x8 ./Application/ButtonManager/ButtonManager.o
 .group         0x00000000        0x8 ./Application/ButtonManager/ButtonManager.o
 .group         0x00000000        0x8 ./Application/ButtonManager/ButtonManager.o
 .group         0x00000000        0x8 ./Application/ButtonManager/ButtonManager.o
 .group         0x00000000        0x8 ./Application/ButtonManager/ButtonManager.o
 .group         0x00000000        0x8 ./Application/ButtonManager/ButtonManager.o
 .text          0x00000000        0x0 ./Application/ButtonManager/ButtonManager.o
 .data          0x00000000        0x0 ./Application/ButtonManager/ButtonManager.o
 .bss           0x00000000        0x0 ./Application/ButtonManager/ButtonManager.o
 .debug_macro   0x00000000      0x802 ./Application/ButtonManager/ButtonManager.o
 .debug_macro   0x00000000       0x16 ./Application/ButtonManager/ButtonManager.o
 .debug_macro   0x00000000      0x214 ./Application/ButtonManager/ButtonManager.o
 .debug_macro   0x00000000       0x39 ./Application/ButtonManager/ButtonManager.o
 .debug_macro   0x00000000       0x3a ./Application/ButtonManager/ButtonManager.o
 .debug_macro   0x00000000       0x1f ./Application/ButtonManager/ButtonManager.o
 .debug_macro   0x00000000      0x250 ./Application/ButtonManager/ButtonManager.o
 .debug_macro   0x00000000       0xc5 ./Application/ButtonManager/ButtonManager.o
 .debug_macro   0x00000000     0x5642 ./Application/ButtonManager/ButtonManager.o
 .debug_macro   0x00000000      0x1fb ./Application/ButtonManager/ButtonManager.o
 .debug_macro   0x00000000       0x3a ./Application/ButtonManager/ButtonManager.o
 .debug_macro   0x00000000       0x8e ./Application/ButtonManager/ButtonManager.o
 .debug_macro   0x00000000       0x81 ./Application/ButtonManager/ButtonManager.o
 .debug_macro   0x00000000       0x4a ./Application/ButtonManager/ButtonManager.o
 .debug_macro   0x00000000       0x6a ./Application/ButtonManager/ButtonManager.o
 .debug_macro   0x00000000       0xca ./Application/ButtonManager/ButtonManager.o
 .debug_macro   0x00000000       0x3b ./Application/ButtonManager/ButtonManager.o
 .debug_macro   0x00000000       0x57 ./Application/ButtonManager/ButtonManager.o
 .debug_macro   0x00000000       0x52 ./Application/ButtonManager/ButtonManager.o
 .debug_macro   0x00000000       0x28 ./Application/ButtonManager/ButtonManager.o
 .debug_macro   0x00000000       0x4a ./Application/ButtonManager/ButtonManager.o
 .debug_macro   0x00000000       0x84 ./Application/ButtonManager/ButtonManager.o
 .debug_macro   0x00000000       0x3a ./Application/ButtonManager/ButtonManager.o
 .debug_macro   0x00000000       0x34 ./Application/ButtonManager/ButtonManager.o
 .debug_macro   0x00000000       0x48 ./Application/ButtonManager/ButtonManager.o
 .debug_macro   0x00000000      0x196 ./Application/ButtonManager/ButtonManager.o
 .debug_macro   0x00000000       0x7c ./Application/ButtonManager/ButtonManager.o
 .debug_macro   0x00000000       0x16 ./Application/ButtonManager/ButtonManager.o
 .debug_macro   0x00000000       0x6b ./Application/ButtonManager/ButtonManager.o
 .debug_macro   0x00000000       0x5d ./Application/ButtonManager/ButtonManager.o
 .debug_macro   0x00000000       0x10 ./Application/ButtonManager/ButtonManager.o
 .debug_macro   0x00000000       0x1c ./Application/ButtonManager/ButtonManager.o
 .debug_macro   0x00000000       0x16 ./Application/ButtonManager/ButtonManager.o
 .debug_macro   0x00000000       0x8e ./Application/ButtonManager/ButtonManager.o
 .debug_macro   0x00000000       0x10 ./Application/ButtonManager/ButtonManager.o
 .group         0x00000000        0x8 ./Application/main.o
 .group         0x00000000        0x8 ./Application/main.o
 .group         0x00000000        0x8 ./Application/main.o
 .group         0x00000000        0x8 ./Application/main.o
 .group         0x00000000        0x8 ./Application/main.o
 .group         0x00000000        0x8 ./Application/main.o
 .group         0x00000000        0x8 ./Application/main.o
 .group         0x00000000        0x8 ./Application/main.o
 .group         0x00000000        0x8 ./Application/main.o
 .group         0x00000000        0x8 ./Application/main.o
 .group         0x00000000        0x8 ./Application/main.o
 .group         0x00000000        0x8 ./Application/main.o
 .group         0x00000000        0x8 ./Application/main.o
 .group         0x00000000        0x8 ./Application/main.o
 .group         0x00000000        0x8 ./Application/main.o
 .group         0x00000000        0x8 ./Application/main.o
 .group         0x00000000        0x8 ./Application/main.o
 .group         0x00000000        0x8 ./Application/main.o
 .group         0x00000000        0x8 ./Application/main.o
 .group         0x00000000        0x8 ./Application/main.o
 .group         0x00000000        0x8 ./Application/main.o
 .group         0x00000000        0x8 ./Application/main.o
 .group         0x00000000        0x8 ./Application/main.o
 .group         0x00000000        0x8 ./Application/main.o
 .group         0x00000000        0x8 ./Application/main.o
 .group         0x00000000        0x8 ./Application/main.o
 .group         0x00000000        0x8 ./Application/main.o
 .group         0x00000000        0x8 ./Application/main.o
 .group         0x00000000        0x8 ./Application/main.o
 .group         0x00000000        0x8 ./Application/main.o
 .group         0x00000000        0x8 ./Application/main.o
 .group         0x00000000        0x8 ./Application/main.o
 .group         0x00000000        0x8 ./Application/main.o
 .group         0x00000000        0x8 ./Application/main.o
 .group         0x00000000        0x8 ./Application/main.o
 .group         0x00000000        0x8 ./Application/main.o
 .text          0x00000000        0x0 ./Application/main.o
 .data          0x00000000        0x0 ./Application/main.o
 .bss           0x00000000        0x0 ./Application/main.o
 .debug_macro   0x00000000      0x802 ./Application/main.o
 .debug_macro   0x00000000       0x16 ./Application/main.o
 .debug_macro   0x00000000      0x214 ./Application/main.o
 .debug_macro   0x00000000       0x39 ./Application/main.o
 .debug_macro   0x00000000       0x3a ./Application/main.o
 .debug_macro   0x00000000       0x1f ./Application/main.o
 .debug_macro   0x00000000      0x250 ./Application/main.o
 .debug_macro   0x00000000       0xc5 ./Application/main.o
 .debug_macro   0x00000000     0x5642 ./Application/main.o
 .debug_macro   0x00000000      0x1fb ./Application/main.o
 .debug_macro   0x00000000       0x22 ./Application/main.o
 .debug_macro   0x00000000       0x34 ./Application/main.o
 .debug_macro   0x00000000       0x48 ./Application/main.o
 .debug_macro   0x00000000       0x65 ./Application/main.o
 .debug_macro   0x00000000       0x5d ./Application/main.o
 .debug_macro   0x00000000       0x52 ./Application/main.o
 .debug_macro   0x00000000       0x4a ./Application/main.o
 .debug_macro   0x00000000       0x4a ./Application/main.o
 .debug_macro   0x00000000       0x84 ./Application/main.o
 .debug_macro   0x00000000       0x6a ./Application/main.o
 .debug_macro   0x00000000       0xca ./Application/main.o
 .debug_macro   0x00000000       0x3b ./Application/main.o
 .debug_macro   0x00000000       0x16 ./Application/main.o
 .debug_macro   0x00000000       0x3a ./Application/main.o
 .debug_macro   0x00000000       0x8e ./Application/main.o
 .debug_macro   0x00000000       0x81 ./Application/main.o
 .debug_macro   0x00000000      0x196 ./Application/main.o
 .debug_macro   0x00000000       0x7c ./Application/main.o
 .debug_macro   0x00000000       0x10 ./Application/main.o
 .debug_macro   0x00000000       0x1c ./Application/main.o
 .debug_macro   0x00000000       0x16 ./Application/main.o
 .debug_macro   0x00000000       0x8e ./Application/main.o
 .debug_macro   0x00000000       0x10 ./Application/main.o
 .data          0x00000000        0x0 e:/logiciels/freescale/kinetis design studio v2.0.0/toolchain/bin/../lib/gcc/arm-none-eabi/4.8.0\libgcc.a(_udivsi3.o)
 .bss           0x00000000        0x0 e:/logiciels/freescale/kinetis design studio v2.0.0/toolchain/bin/../lib/gcc/arm-none-eabi/4.8.0\libgcc.a(_udivsi3.o)
 .data          0x00000000        0x0 e:/logiciels/freescale/kinetis design studio v2.0.0/toolchain/bin/../lib/gcc/arm-none-eabi/4.8.0\libgcc.a(_dvmd_tls.o)
 .bss           0x00000000        0x0 e:/logiciels/freescale/kinetis design studio v2.0.0/toolchain/bin/../lib/gcc/arm-none-eabi/4.8.0\libgcc.a(_dvmd_tls.o)
 .text          0x00000000        0x0 e:/logiciels/freescale/kinetis design studio v2.0.0/toolchain/bin/../lib/gcc/arm-none-eabi/4.8.0/../../../../arm-none-eabi/lib\libg_s.a(lib_a-atexit.o)
 .data          0x00000000        0x0 e:/logiciels/freescale/kinetis design studio v2.0.0/toolchain/bin/../lib/gcc/arm-none-eabi/4.8.0/../../../../arm-none-eabi/lib\libg_s.a(lib_a-atexit.o)
 .bss           0x00000000        0x0 e:/logiciels/freescale/kinetis design studio v2.0.0/toolchain/bin/../lib/gcc/arm-none-eabi/4.8.0/../../../../arm-none-eabi/lib\libg_s.a(lib_a-atexit.o)
 .text          0x00000000        0x0 e:/logiciels/freescale/kinetis design studio v2.0.0/toolchain/bin/../lib/gcc/arm-none-eabi/4.8.0/../../../../arm-none-eabi/lib\libg_s.a(lib_a-exit.o)
 .data          0x00000000        0x0 e:/logiciels/freescale/kinetis design studio v2.0.0/toolchain/bin/../lib/gcc/arm-none-eabi/4.8.0/../../../../arm-none-eabi/lib\libg_s.a(lib_a-exit.o)
 .bss           0x00000000        0x0 e:/logiciels/freescale/kinetis design studio v2.0.0/toolchain/bin/../lib/gcc/arm-none-eabi/4.8.0/../../../../arm-none-eabi/lib\libg_s.a(lib_a-exit.o)
 .text          0x00000000        0x0 e:/logiciels/freescale/kinetis design studio v2.0.0/toolchain/bin/../lib/gcc/arm-none-eabi/4.8.0/../../../../arm-none-eabi/lib\libg_s.a(lib_a-fini.o)
 .data          0x00000000        0x0 e:/logiciels/freescale/kinetis design studio v2.0.0/toolchain/bin/../lib/gcc/arm-none-eabi/4.8.0/../../../../arm-none-eabi/lib\libg_s.a(lib_a-fini.o)
 .bss           0x00000000        0x0 e:/logiciels/freescale/kinetis design studio v2.0.0/toolchain/bin/../lib/gcc/arm-none-eabi/4.8.0/../../../../arm-none-eabi/lib\libg_s.a(lib_a-fini.o)
 .text          0x00000000        0x0 e:/logiciels/freescale/kinetis design studio v2.0.0/toolchain/bin/../lib/gcc/arm-none-eabi/4.8.0/../../../../arm-none-eabi/lib\libg_s.a(lib_a-impure.o)
 .data          0x00000000        0x0 e:/logiciels/freescale/kinetis design studio v2.0.0/toolchain/bin/../lib/gcc/arm-none-eabi/4.8.0/../../../../arm-none-eabi/lib\libg_s.a(lib_a-impure.o)
 .bss           0x00000000        0x0 e:/logiciels/freescale/kinetis design studio v2.0.0/toolchain/bin/../lib/gcc/arm-none-eabi/4.8.0/../../../../arm-none-eabi/lib\libg_s.a(lib_a-impure.o)
 .text          0x00000000        0x0 e:/logiciels/freescale/kinetis design studio v2.0.0/toolchain/bin/../lib/gcc/arm-none-eabi/4.8.0/../../../../arm-none-eabi/lib\libg_s.a(lib_a-memcpy.o)
 .data          0x00000000        0x0 e:/logiciels/freescale/kinetis design studio v2.0.0/toolchain/bin/../lib/gcc/arm-none-eabi/4.8.0/../../../../arm-none-eabi/lib\libg_s.a(lib_a-memcpy.o)
 .bss           0x00000000        0x0 e:/logiciels/freescale/kinetis design studio v2.0.0/toolchain/bin/../lib/gcc/arm-none-eabi/4.8.0/../../../../arm-none-eabi/lib\libg_s.a(lib_a-memcpy.o)
 .text          0x00000000        0x0 e:/logiciels/freescale/kinetis design studio v2.0.0/toolchain/bin/../lib/gcc/arm-none-eabi/4.8.0/../../../../arm-none-eabi/lib\libg_s.a(lib_a-memset.o)
 .data          0x00000000        0x0 e:/logiciels/freescale/kinetis design studio v2.0.0/toolchain/bin/../lib/gcc/arm-none-eabi/4.8.0/../../../../arm-none-eabi/lib\libg_s.a(lib_a-memset.o)
 .bss           0x00000000        0x0 e:/logiciels/freescale/kinetis design studio v2.0.0/toolchain/bin/../lib/gcc/arm-none-eabi/4.8.0/../../../../arm-none-eabi/lib\libg_s.a(lib_a-memset.o)
 .text          0x00000000        0x0 e:/logiciels/freescale/kinetis design studio v2.0.0/toolchain/bin/../lib/gcc/arm-none-eabi/4.8.0/../../../../arm-none-eabi/lib\libg_s.a(lib_a-syscalls.o)
 .data          0x00000000        0x0 e:/logiciels/freescale/kinetis design studio v2.0.0/toolchain/bin/../lib/gcc/arm-none-eabi/4.8.0/../../../../arm-none-eabi/lib\libg_s.a(lib_a-syscalls.o)
 .bss           0x00000000        0x0 e:/logiciels/freescale/kinetis design studio v2.0.0/toolchain/bin/../lib/gcc/arm-none-eabi/4.8.0/../../../../arm-none-eabi/lib\libg_s.a(lib_a-syscalls.o)
 .text.invalid_fd
                0x00000000       0x1c e:/logiciels/freescale/kinetis design studio v2.0.0/toolchain/bin/../lib/gcc/arm-none-eabi/4.8.0/../../../../arm-none-eabi/lib\libg_s.a(lib_a-syscalls.o)
 .text.error    0x00000000       0x1c e:/logiciels/freescale/kinetis design studio v2.0.0/toolchain/bin/../lib/gcc/arm-none-eabi/4.8.0/../../../../arm-none-eabi/lib\libg_s.a(lib_a-syscalls.o)
 .text.findslot.part.0
                0x00000000       0x1c e:/logiciels/freescale/kinetis design studio v2.0.0/toolchain/bin/../lib/gcc/arm-none-eabi/4.8.0/../../../../arm-none-eabi/lib\libg_s.a(lib_a-syscalls.o)
 .text.initialise_monitor_handles
                0x00000000       0x78 e:/logiciels/freescale/kinetis design studio v2.0.0/toolchain/bin/../lib/gcc/arm-none-eabi/4.8.0/../../../../arm-none-eabi/lib\libg_s.a(lib_a-syscalls.o)
 .text._swiread
                0x00000000       0x26 e:/logiciels/freescale/kinetis design studio v2.0.0/toolchain/bin/../lib/gcc/arm-none-eabi/4.8.0/../../../../arm-none-eabi/lib\libg_s.a(lib_a-syscalls.o)
 .text._read    0x00000000       0x64 e:/logiciels/freescale/kinetis design studio v2.0.0/toolchain/bin/../lib/gcc/arm-none-eabi/4.8.0/../../../../arm-none-eabi/lib\libg_s.a(lib_a-syscalls.o)
 .text._swilseek
                0x00000000       0xa4 e:/logiciels/freescale/kinetis design studio v2.0.0/toolchain/bin/../lib/gcc/arm-none-eabi/4.8.0/../../../../arm-none-eabi/lib\libg_s.a(lib_a-syscalls.o)
 .text._lseek   0x00000000       0x10 e:/logiciels/freescale/kinetis design studio v2.0.0/toolchain/bin/../lib/gcc/arm-none-eabi/4.8.0/../../../../arm-none-eabi/lib\libg_s.a(lib_a-syscalls.o)
 .text._swiwrite
                0x00000000       0x26 e:/logiciels/freescale/kinetis design studio v2.0.0/toolchain/bin/../lib/gcc/arm-none-eabi/4.8.0/../../../../arm-none-eabi/lib\libg_s.a(lib_a-syscalls.o)
 .text._write   0x00000000       0x68 e:/logiciels/freescale/kinetis design studio v2.0.0/toolchain/bin/../lib/gcc/arm-none-eabi/4.8.0/../../../../arm-none-eabi/lib\libg_s.a(lib_a-syscalls.o)
 .text._swiopen
                0x00000000       0x84 e:/logiciels/freescale/kinetis design studio v2.0.0/toolchain/bin/../lib/gcc/arm-none-eabi/4.8.0/../../../../arm-none-eabi/lib\libg_s.a(lib_a-syscalls.o)
 .text._open    0x00000000       0x18 e:/logiciels/freescale/kinetis design studio v2.0.0/toolchain/bin/../lib/gcc/arm-none-eabi/4.8.0/../../../../arm-none-eabi/lib\libg_s.a(lib_a-syscalls.o)
 .text._swiclose
                0x00000000       0x40 e:/logiciels/freescale/kinetis design studio v2.0.0/toolchain/bin/../lib/gcc/arm-none-eabi/4.8.0/../../../../arm-none-eabi/lib\libg_s.a(lib_a-syscalls.o)
 .text._close   0x00000000       0x10 e:/logiciels/freescale/kinetis design studio v2.0.0/toolchain/bin/../lib/gcc/arm-none-eabi/4.8.0/../../../../arm-none-eabi/lib\libg_s.a(lib_a-syscalls.o)
 .text._getpid  0x00000000        0x4 e:/logiciels/freescale/kinetis design studio v2.0.0/toolchain/bin/../lib/gcc/arm-none-eabi/4.8.0/../../../../arm-none-eabi/lib\libg_s.a(lib_a-syscalls.o)
 .text._fstat   0x00000000       0x1e e:/logiciels/freescale/kinetis design studio v2.0.0/toolchain/bin/../lib/gcc/arm-none-eabi/4.8.0/../../../../arm-none-eabi/lib\libg_s.a(lib_a-syscalls.o)
 .text._stat    0x00000000       0x34 e:/logiciels/freescale/kinetis design studio v2.0.0/toolchain/bin/../lib/gcc/arm-none-eabi/4.8.0/../../../../arm-none-eabi/lib\libg_s.a(lib_a-syscalls.o)
 .text._link    0x00000000        0x6 e:/logiciels/freescale/kinetis design studio v2.0.0/toolchain/bin/../lib/gcc/arm-none-eabi/4.8.0/../../../../arm-none-eabi/lib\libg_s.a(lib_a-syscalls.o)
 .text._unlink  0x00000000       0x2a e:/logiciels/freescale/kinetis design studio v2.0.0/toolchain/bin/../lib/gcc/arm-none-eabi/4.8.0/../../../../arm-none-eabi/lib\libg_s.a(lib_a-syscalls.o)
 .text._raise   0x00000000        0x2 e:/logiciels/freescale/kinetis design studio v2.0.0/toolchain/bin/../lib/gcc/arm-none-eabi/4.8.0/../../../../arm-none-eabi/lib\libg_s.a(lib_a-syscalls.o)
 .text._gettimeofday
                0x00000000       0x2a e:/logiciels/freescale/kinetis design studio v2.0.0/toolchain/bin/../lib/gcc/arm-none-eabi/4.8.0/../../../../arm-none-eabi/lib\libg_s.a(lib_a-syscalls.o)
 .text._times   0x00000000       0x22 e:/logiciels/freescale/kinetis design studio v2.0.0/toolchain/bin/../lib/gcc/arm-none-eabi/4.8.0/../../../../arm-none-eabi/lib\libg_s.a(lib_a-syscalls.o)
 .text._isatty  0x00000000       0x44 e:/logiciels/freescale/kinetis design studio v2.0.0/toolchain/bin/../lib/gcc/arm-none-eabi/4.8.0/../../../../arm-none-eabi/lib\libg_s.a(lib_a-syscalls.o)
 .text._system  0x00000000       0x42 e:/logiciels/freescale/kinetis design studio v2.0.0/toolchain/bin/../lib/gcc/arm-none-eabi/4.8.0/../../../../arm-none-eabi/lib\libg_s.a(lib_a-syscalls.o)
 .text._rename  0x00000000       0x3a e:/logiciels/freescale/kinetis design studio v2.0.0/toolchain/bin/../lib/gcc/arm-none-eabi/4.8.0/../../../../arm-none-eabi/lib\libg_s.a(lib_a-syscalls.o)
 .bss.monitor_stdout
                0x00000000        0x4 e:/logiciels/freescale/kinetis design studio v2.0.0/toolchain/bin/../lib/gcc/arm-none-eabi/4.8.0/../../../../arm-none-eabi/lib\libg_s.a(lib_a-syscalls.o)
 .bss.monitor_stdin
                0x00000000        0x4 e:/logiciels/freescale/kinetis design studio v2.0.0/toolchain/bin/../lib/gcc/arm-none-eabi/4.8.0/../../../../arm-none-eabi/lib\libg_s.a(lib_a-syscalls.o)
 .rodata.str1.1
                0x00000000        0x4 e:/logiciels/freescale/kinetis design studio v2.0.0/toolchain/bin/../lib/gcc/arm-none-eabi/4.8.0/../../../../arm-none-eabi/lib\libg_s.a(lib_a-syscalls.o)
 .bss.monitor_stderr
                0x00000000        0x4 e:/logiciels/freescale/kinetis design studio v2.0.0/toolchain/bin/../lib/gcc/arm-none-eabi/4.8.0/../../../../arm-none-eabi/lib\libg_s.a(lib_a-syscalls.o)
 .bss.openfiles
                0x00000000       0xa0 e:/logiciels/freescale/kinetis design studio v2.0.0/toolchain/bin/../lib/gcc/arm-none-eabi/4.8.0/../../../../arm-none-eabi/lib\libg_s.a(lib_a-syscalls.o)
 .text          0x00000000        0x0 e:/logiciels/freescale/kinetis design studio v2.0.0/toolchain/bin/../lib/gcc/arm-none-eabi/4.8.0/../../../../arm-none-eabi/lib\libg_s.a(lib_a-__atexit.o)
 .data          0x00000000        0x0 e:/logiciels/freescale/kinetis design studio v2.0.0/toolchain/bin/../lib/gcc/arm-none-eabi/4.8.0/../../../../arm-none-eabi/lib\libg_s.a(lib_a-__atexit.o)
 .bss           0x00000000        0x0 e:/logiciels/freescale/kinetis design studio v2.0.0/toolchain/bin/../lib/gcc/arm-none-eabi/4.8.0/../../../../arm-none-eabi/lib\libg_s.a(lib_a-__atexit.o)
 .data.__atexit_dummy
                0x00000000        0x4 e:/logiciels/freescale/kinetis design studio v2.0.0/toolchain/bin/../lib/gcc/arm-none-eabi/4.8.0/../../../../arm-none-eabi/lib\libg_s.a(lib_a-__atexit.o)
 .text          0x00000000        0x0 e:/logiciels/freescale/kinetis design studio v2.0.0/toolchain/bin/../lib/gcc/arm-none-eabi/4.8.0/../../../../arm-none-eabi/lib\libg_s.a(lib_a-__call_atexit.o)
 .data          0x00000000        0x0 e:/logiciels/freescale/kinetis design studio v2.0.0/toolchain/bin/../lib/gcc/arm-none-eabi/4.8.0/../../../../arm-none-eabi/lib\libg_s.a(lib_a-__call_atexit.o)
 .bss           0x00000000        0x0 e:/logiciels/freescale/kinetis design studio v2.0.0/toolchain/bin/../lib/gcc/arm-none-eabi/4.8.0/../../../../arm-none-eabi/lib\libg_s.a(lib_a-__call_atexit.o)
 .text          0x00000000        0x0 e:/logiciels/freescale/kinetis design studio v2.0.0/toolchain/bin/../lib/gcc/arm-none-eabi/4.8.0/../../../../arm-none-eabi/lib\libg_s.a(lib_a-errno.o)
 .data          0x00000000        0x0 e:/logiciels/freescale/kinetis design studio v2.0.0/toolchain/bin/../lib/gcc/arm-none-eabi/4.8.0/../../../../arm-none-eabi/lib\libg_s.a(lib_a-errno.o)
 .bss           0x00000000        0x0 e:/logiciels/freescale/kinetis design studio v2.0.0/toolchain/bin/../lib/gcc/arm-none-eabi/4.8.0/../../../../arm-none-eabi/lib\libg_s.a(lib_a-errno.o)
 .text          0x00000000        0x0 e:/logiciels/freescale/kinetis design studio v2.0.0/toolchain/bin/../lib/gcc/arm-none-eabi/4.8.0/../../../../arm-none-eabi/lib\libg_s.a(lib_a-malloc.o)
 .data          0x00000000        0x0 e:/logiciels/freescale/kinetis design studio v2.0.0/toolchain/bin/../lib/gcc/arm-none-eabi/4.8.0/../../../../arm-none-eabi/lib\libg_s.a(lib_a-malloc.o)
 .bss           0x00000000        0x0 e:/logiciels/freescale/kinetis design studio v2.0.0/toolchain/bin/../lib/gcc/arm-none-eabi/4.8.0/../../../../arm-none-eabi/lib\libg_s.a(lib_a-malloc.o)
 .text          0x00000000        0x0 e:/logiciels/freescale/kinetis design studio v2.0.0/toolchain/bin/../lib/gcc/arm-none-eabi/4.8.0/../../../../arm-none-eabi/lib\libg_s.a(lib_a-mallocr.o)
 .data          0x00000000        0x0 e:/logiciels/freescale/kinetis design studio v2.0.0/toolchain/bin/../lib/gcc/arm-none-eabi/4.8.0/../../../../arm-none-eabi/lib\libg_s.a(lib_a-mallocr.o)
 .bss           0x00000000        0x0 e:/logiciels/freescale/kinetis design studio v2.0.0/toolchain/bin/../lib/gcc/arm-none-eabi/4.8.0/../../../../arm-none-eabi/lib\libg_s.a(lib_a-mallocr.o)
 .text          0x00000000        0x0 e:/logiciels/freescale/kinetis design studio v2.0.0/toolchain/bin/../lib/gcc/arm-none-eabi/4.8.0/../../../../arm-none-eabi/lib\libg_s.a(lib_a-sbrkr.o)
 .data          0x00000000        0x0 e:/logiciels/freescale/kinetis design studio v2.0.0/toolchain/bin/../lib/gcc/arm-none-eabi/4.8.0/../../../../arm-none-eabi/lib\libg_s.a(lib_a-sbrkr.o)
 .bss           0x00000000        0x0 e:/logiciels/freescale/kinetis design studio v2.0.0/toolchain/bin/../lib/gcc/arm-none-eabi/4.8.0/../../../../arm-none-eabi/lib\libg_s.a(lib_a-sbrkr.o)
 .text          0x00000000        0x0 e:/logiciels/freescale/kinetis design studio v2.0.0/toolchain/bin/../lib/gcc/arm-none-eabi/4.8.0/../../../../arm-none-eabi/lib\libg_s.a(lib_a-strlen.o)
 .data          0x00000000        0x0 e:/logiciels/freescale/kinetis design studio v2.0.0/toolchain/bin/../lib/gcc/arm-none-eabi/4.8.0/../../../../arm-none-eabi/lib\libg_s.a(lib_a-strlen.o)
 .bss           0x00000000        0x0 e:/logiciels/freescale/kinetis design studio v2.0.0/toolchain/bin/../lib/gcc/arm-none-eabi/4.8.0/../../../../arm-none-eabi/lib\libg_s.a(lib_a-strlen.o)
 .text.strlen   0x00000000        0xe e:/logiciels/freescale/kinetis design studio v2.0.0/toolchain/bin/../lib/gcc/arm-none-eabi/4.8.0/../../../../arm-none-eabi/lib\libg_s.a(lib_a-strlen.o)
 .comment       0x00000000       0x2b e:/logiciels/freescale/kinetis design studio v2.0.0/toolchain/bin/../lib/gcc/arm-none-eabi/4.8.0/../../../../arm-none-eabi/lib\libg_s.a(lib_a-strlen.o)
 .ARM.attributes
                0x00000000       0x31 e:/logiciels/freescale/kinetis design studio v2.0.0/toolchain/bin/../lib/gcc/arm-none-eabi/4.8.0/../../../../arm-none-eabi/lib\libg_s.a(lib_a-strlen.o)
 .text          0x00000000        0x0 e:/logiciels/freescale/kinetis design studio v2.0.0/toolchain/bin/../lib/gcc/arm-none-eabi/4.8.0/../../../../arm-none-eabi/lib\libg_s.a(lib_a-freer.o)
 .data          0x00000000        0x0 e:/logiciels/freescale/kinetis design studio v2.0.0/toolchain/bin/../lib/gcc/arm-none-eabi/4.8.0/../../../../arm-none-eabi/lib\libg_s.a(lib_a-freer.o)
 .bss           0x00000000        0x0 e:/logiciels/freescale/kinetis design studio v2.0.0/toolchain/bin/../lib/gcc/arm-none-eabi/4.8.0/../../../../arm-none-eabi/lib\libg_s.a(lib_a-freer.o)
 .text          0x00000000        0x0 e:/logiciels/freescale/kinetis design studio v2.0.0/toolchain/bin/../lib/gcc/arm-none-eabi/4.8.0/../../../../arm-none-eabi/lib\libg_s.a(lib_a-reent.o)
 .data          0x00000000        0x0 e:/logiciels/freescale/kinetis design studio v2.0.0/toolchain/bin/../lib/gcc/arm-none-eabi/4.8.0/../../../../arm-none-eabi/lib\libg_s.a(lib_a-reent.o)
 .bss           0x00000000        0x0 e:/logiciels/freescale/kinetis design studio v2.0.0/toolchain/bin/../lib/gcc/arm-none-eabi/4.8.0/../../../../arm-none-eabi/lib\libg_s.a(lib_a-reent.o)
 .text.cleanup_glue
                0x00000000       0x1a e:/logiciels/freescale/kinetis design studio v2.0.0/toolchain/bin/../lib/gcc/arm-none-eabi/4.8.0/../../../../arm-none-eabi/lib\libg_s.a(lib_a-reent.o)
 .text._reclaim_reent
                0x00000000       0x7c e:/logiciels/freescale/kinetis design studio v2.0.0/toolchain/bin/../lib/gcc/arm-none-eabi/4.8.0/../../../../arm-none-eabi/lib\libg_s.a(lib_a-reent.o)
 .text._wrapup_reent
                0x00000000       0x38 e:/logiciels/freescale/kinetis design studio v2.0.0/toolchain/bin/../lib/gcc/arm-none-eabi/4.8.0/../../../../arm-none-eabi/lib\libg_s.a(lib_a-reent.o)
 .text          0x00000000        0x0 e:/logiciels/freescale/kinetis design studio v2.0.0/toolchain/bin/../lib/gcc/arm-none-eabi/4.8.0/crtend.o
 .data          0x00000000        0x0 e:/logiciels/freescale/kinetis design studio v2.0.0/toolchain/bin/../lib/gcc/arm-none-eabi/4.8.0/crtend.o
 .bss           0x00000000        0x0 e:/logiciels/freescale/kinetis design studio v2.0.0/toolchain/bin/../lib/gcc/arm-none-eabi/4.8.0/crtend.o
 .eh_frame      0x00000000        0x4 e:/logiciels/freescale/kinetis design studio v2.0.0/toolchain/bin/../lib/gcc/arm-none-eabi/4.8.0/crtend.o
 .text          0x00000000        0x0 e:/logiciels/freescale/kinetis design studio v2.0.0/toolchain/bin/../lib/gcc/arm-none-eabi/4.8.0/crtn.o
 .data          0x00000000        0x0 e:/logiciels/freescale/kinetis design studio v2.0.0/toolchain/bin/../lib/gcc/arm-none-eabi/4.8.0/crtn.o
 .bss           0x00000000        0x0 e:/logiciels/freescale/kinetis design studio v2.0.0/toolchain/bin/../lib/gcc/arm-none-eabi/4.8.0/crtn.o

Memory Configuration

Name             Origin             Length             Attributes
m_interrupts     0x00000000         0x00000100         xr
m_flash_config   0x00000400         0x00000010         xr
m_text           0x00000410         0x0003fbf0         xr
m_data           0x1fffe000         0x00008000         rw
*default*        0x00000000         0xffffffff

Linker script and memory map

LOAD e:/logiciels/freescale/kinetis design studio v2.0.0/toolchain/bin/../lib/gcc/arm-none-eabi/4.8.0/crti.o
LOAD e:/logiciels/freescale/kinetis design studio v2.0.0/toolchain/bin/../lib/gcc/arm-none-eabi/4.8.0/crtbegin.o
LOAD e:/logiciels/freescale/kinetis design studio v2.0.0/toolchain/bin/../lib/gcc/arm-none-eabi/4.8.0/../../../../arm-none-eabi/lib/crt0.o
LOAD ./Tools/StringTools/StringTools.o
LOAD ./Tools/Decoder7Seg/decoder7Seg.o
LOAD ./Tools/Decoder16Seg/decoder16Seg.o
LOAD ./Tools/Checksum/checksum.o
LOAD ./Project_Settings/Startup_Code/startup_MKL16Z4.o
LOAD ./Project_Settings/Startup_Code/system_MKL16Z4.o
LOAD ./DSP/Watchdog/watchdog.o
LOAD ./DSP/UART/uart0.o
LOAD ./DSP/UART/uart1.o
LOAD ./DSP/UART/uart2.o
LOAD ./DSP/SPI/spi0.o
LOAD ./DSP/SPI/spi1.o
LOAD ./DSP/RTC/rtc.o
LOAD ./DSP/PIT/pit.o
LOAD ./DSP/I2C/i2c0.o
LOAD ./DSP/Device/device.o
LOAD ./DSP/DSP/DSP_mkl16z256vlh4.o
LOAD ./BSP/Tick/tick.o
LOAD ./BSP/RFID_CR95HF/CR95HF.o
LOAD ./BSP/RFID_CR95HF/CR95UartMapper.o
LOAD ./BSP/Led/led.o
LOAD ./BSP/FRAM/FM25V20.o
LOAD ./BSP/FRAM/FM25V20MemTest.o
LOAD ./BSP/Display/display.o
LOAD ./BSP/Button/button.o
LOAD ./BSP/BatteryManagement/BQ27510DRZRG2.o
LOAD ./BSP/BatteryManagement/LTC4160.o
LOAD ./Application/UsbManager/UsbManager.o
LOAD ./Application/RFIDManager/RFIDManager.o
LOAD ./Application/PowerManager/PowerManager.o
LOAD ./Application/MemoryManager/MemoryManager.o
LOAD ./Application/Global/globalParameters.o
LOAD ./Application/ButtonManager/ButtonManager.o
LOAD ./Application/main.o
LOAD e:/logiciels/freescale/kinetis design studio v2.0.0/toolchain/bin/../lib/gcc/arm-none-eabi/4.8.0/../../../../arm-none-eabi/lib\libstdc++.a
LOAD e:/logiciels/freescale/kinetis design studio v2.0.0/toolchain/bin/../lib/gcc/arm-none-eabi/4.8.0/../../../../arm-none-eabi/lib\libm.a
START GROUP
LOAD e:/logiciels/freescale/kinetis design studio v2.0.0/toolchain/bin/../lib/gcc/arm-none-eabi/4.8.0\libgcc.a
LOAD e:/logiciels/freescale/kinetis design studio v2.0.0/toolchain/bin/../lib/gcc/arm-none-eabi/4.8.0/../../../../arm-none-eabi/lib\libg_s.a
LOAD e:/logiciels/freescale/kinetis design studio v2.0.0/toolchain/bin/../lib/gcc/arm-none-eabi/4.8.0/../../../../arm-none-eabi/lib\libc_s.a
END GROUP
LOAD e:/logiciels/freescale/kinetis design studio v2.0.0/toolchain/bin/../lib/gcc/arm-none-eabi/4.8.0/crtend.o
LOAD e:/logiciels/freescale/kinetis design studio v2.0.0/toolchain/bin/../lib/gcc/arm-none-eabi/4.8.0/crtn.o
                0x00000400                HEAP_SIZE = DEFINED (__heap_size__)?__heap_size__:0x400
                0x00000400                STACK_SIZE = DEFINED (__stack_size__)?__stack_size__:0x400

.interrupts     0x00000000       0xc0
                0x00000000                __VECTOR_TABLE = .
                0x00000000                . = ALIGN (0x4)
 *(.isr_vector)
 .isr_vector    0x00000000       0xc0 ./Project_Settings/Startup_Code/startup_MKL16Z4.o
                0x00000000                __isr_vector
                0x000000c0                . = ALIGN (0x4)

.flash_config   0x00000400       0x10
                0x00000400                . = ALIGN (0x4)
 *(.FlashConfig)
 .FlashConfig   0x00000400       0x10 ./Project_Settings/Startup_Code/startup_MKL16Z4.o
                0x00000410                . = ALIGN (0x4)

.text           0x00000410     0x8a78
                0x00000410                . = ALIGN (0x4)
 *(.text)
 .text          0x00000410       0xf4 e:/logiciels/freescale/kinetis design studio v2.0.0/toolchain/bin/../lib/gcc/arm-none-eabi/4.8.0/../../../../arm-none-eabi/lib/crt0.o
                0x00000440                _start
 .text          0x00000504       0x44 ./Project_Settings/Startup_Code/startup_MKL16Z4.o
                0x00000504                Reset_Handler
                0x00000544                HardFault_Handler
                0x00000544                SysTick_Handler
                0x00000544                PendSV_Handler
                0x00000544                NMI_Handler
                0x00000544                PORTC_PORTD_IRQHandler
                0x00000544                I2C1_IRQHandler
                0x00000544                DMA2_IRQHandler
                0x00000544                TPM0_IRQHandler
                0x00000544                I2S0_IRQHandler
                0x00000544                TSI0_IRQHandler
                0x00000544                ADC0_IRQHandler
                0x00000544                SPI1_IRQHandler
                0x00000544                DefaultISR
                0x00000544                TPM2_IRQHandler
                0x00000544                LPTimer_IRQHandler
                0x00000544                RTC_IRQHandler
                0x00000544                I2C0_IRQHandler
                0x00000544                RTC_Seconds_IRQHandler
                0x00000544                MCG_IRQHandler
                0x00000544                Reserved20_IRQHandler
                0x00000544                Default_Handler
                0x00000544                LLW_IRQHandler
                0x00000544                SVC_Handler
                0x00000544                DMA3_IRQHandler
                0x00000544                DMA0_IRQHandler
                0x00000544                DAC0_IRQHandler
                0x00000544                Reserved45_IRQHandler
                0x00000544                TPM1_IRQHandler
                0x00000544                LVD_LVW_IRQHandler
                0x00000544                SPI0_IRQHandler
                0x00000544                FTFA_IRQHandler
                0x00000544                Reserved40_IRQHandler
                0x00000544                CMP0_IRQHandler
                0x00000544                DMA1_IRQHandler
 .text          0x00000548       0x9c e:/logiciels/freescale/kinetis design studio v2.0.0/toolchain/bin/../lib/gcc/arm-none-eabi/4.8.0\libgcc.a(_udivsi3.o)
                0x00000548                __aeabi_uidiv
                0x00000548                __udivsi3
                0x000005d0                __aeabi_uidivmod
 .text          0x000005e4        0x4 e:/logiciels/freescale/kinetis design studio v2.0.0/toolchain/bin/../lib/gcc/arm-none-eabi/4.8.0\libgcc.a(_dvmd_tls.o)
                0x000005e4                __aeabi_idiv0
                0x000005e4                __aeabi_ldiv0
 *(.text*)
 .text.deregister_tm_clones
                0x000005e8       0x24 e:/logiciels/freescale/kinetis design studio v2.0.0/toolchain/bin/../lib/gcc/arm-none-eabi/4.8.0/crtbegin.o
 .text.register_tm_clones
                0x0000060c       0x28 e:/logiciels/freescale/kinetis design studio v2.0.0/toolchain/bin/../lib/gcc/arm-none-eabi/4.8.0/crtbegin.o
 .text.__do_global_dtors_aux
                0x00000634       0x30 e:/logiciels/freescale/kinetis design studio v2.0.0/toolchain/bin/../lib/gcc/arm-none-eabi/4.8.0/crtbegin.o
 .text.frame_dummy
                0x00000664       0x3c e:/logiciels/freescale/kinetis design studio v2.0.0/toolchain/bin/../lib/gcc/arm-none-eabi/4.8.0/crtbegin.o
 .text.StrTool_ClearString
                0x000006a0       0x34 ./Tools/StringTools/StringTools.o
                0x000006a0                StrTool_ClearString
 .text.Decode7segDigitASCII
                0x000006d4      0x130 ./Tools/Decoder7Seg/decoder7Seg.o
                0x000006d4                Decode7segDigitASCII
 .text.Decode16segDigitASCII
                0x00000804      0x274 ./Tools/Decoder16Seg/decoder16Seg.o
                0x00000804                Decode16segDigitASCII
 .text.ChecksumByteCompute
                0x00000a78       0x3c ./Tools/Checksum/checksum.o
                0x00000a78                ChecksumByteCompute
 .text.ChecksumByteOnShortCompute
                0x00000ab4       0x3c ./Tools/Checksum/checksum.o
                0x00000ab4                ChecksumByteOnShortCompute
 .text.SystemInit
                0x00000af0       0xd4 ./Project_Settings/Startup_Code/system_MKL16Z4.o
                0x00000af0                SystemInit
 .text.WatchdogStart
                0x00000bc4       0x34 ./DSP/Watchdog/watchdog.o
                0x00000bc4                WatchdogStart
 .text.WatchdogKick
                0x00000bf8       0x20 ./DSP/Watchdog/watchdog.o
                0x00000bf8                WatchdogKick
 .text.UART0_IRQHandler
                0x00000c18      0x114 ./DSP/UART/uart0.o
                0x00000c18                UART0_IRQHandler
 .text.Uart0Init
                0x00000d2c       0xec ./DSP/UART/uart0.o
                0x00000d2c                Uart0Init
 .text.Uart0SendData
                0x00000e18       0xe4 ./DSP/UART/uart0.o
                0x00000e18                Uart0SendData
 .text.Uart0ReadChar
                0x00000efc       0x9c ./DSP/UART/uart0.o
                0x00000efc                Uart0ReadChar
 .text.UART1_IRQHandler
                0x00000f98      0x104 ./DSP/UART/uart1.o
                0x00000f98                UART1_IRQHandler
 .text.Uart1Init
                0x0000109c       0xec ./DSP/UART/uart1.o
                0x0000109c                Uart1Init
 .text.Uart1SendData
                0x00001188       0xd4 ./DSP/UART/uart1.o
                0x00001188                Uart1SendData
 .text.Uart1SendString
                0x0000125c       0xbc ./DSP/UART/uart1.o
                0x0000125c                Uart1SendString
 .text.Uart1ReadChar
                0x00001318       0x9c ./DSP/UART/uart1.o
                0x00001318                Uart1ReadChar
 .text.UART2_IRQHandler
                0x000013b4      0x104 ./DSP/UART/uart2.o
                0x000013b4                UART2_IRQHandler
 .text.Uart2Init
                0x000014b8       0xec ./DSP/UART/uart2.o
                0x000014b8                Uart2Init
 .text.Uart2SendData
                0x000015a4       0xd4 ./DSP/UART/uart2.o
                0x000015a4                Uart2SendData
 .text.Uart2ReadChar
                0x00001678       0x9c ./DSP/UART/uart2.o
                0x00001678                Uart2ReadChar
 .text.Spi0Init
                0x00001714      0x1dc ./DSP/SPI/spi0.o
                0x00001714                Spi0Init
 .text.Spi0Send
                0x000018f0       0x94 ./DSP/SPI/spi0.o
                0x000018f0                Spi0Send
 .text.Spi1Init
                0x00001984      0x1dc ./DSP/SPI/spi1.o
                0x00001984                Spi1Init
 .text.Spi1Send
                0x00001b60       0x94 ./DSP/SPI/spi1.o
                0x00001b60                Spi1Send
 .text.Spi1Read
                0x00001bf4       0xd8 ./DSP/SPI/spi1.o
                0x00001bf4                Spi1Read
 .text.RtcInit  0x00001ccc       0x58 ./DSP/RTC/rtc.o
                0x00001ccc                RtcInit
 .text.RtcGetTime
                0x00001d24       0x38 ./DSP/RTC/rtc.o
                0x00001d24                RtcGetTime
 .text.RtcSetTime
                0x00001d5c       0x40 ./DSP/RTC/rtc.o
                0x00001d5c                RtcSetTime
 .text.RtcUpdatedSinceLastReset
                0x00001d9c       0x14 ./DSP/RTC/rtc.o
                0x00001d9c                RtcUpdatedSinceLastReset
 .text.PIT_IRQHandler
                0x00001db0       0x60 ./DSP/PIT/pit.o
                0x00001db0                PIT_IRQHandler
 .text.PitInit  0x00001e10       0xf4 ./DSP/PIT/pit.o
                0x00001e10                PitInit
 .text.I2C0Init
                0x00001f04       0x74 ./DSP/I2C/i2c0.o
                0x00001f04                I2C0Init
 .text.I2C0Send
                0x00001f78      0x148 ./DSP/I2C/i2c0.o
                0x00001f78                I2C0Send
 .text.I2C0Read
                0x000020c0      0x208 ./DSP/I2C/i2c0.o
                0x000020c0                I2C0Read
 .text.DeviceInit
                0x000022c8        0xc ./DSP/Device/device.o
                0x000022c8                DeviceInit
 .text.DeviceClockSwitchDefaultFEI
                0x000022d4      0x154 ./DSP/Device/device.o
                0x000022d4                DeviceClockSwitchDefaultFEI
 .text.DeviceClockSwitchHighPower
                0x00002428      0x1e0 ./DSP/Device/device.o
                0x00002428                DeviceClockSwitchHighPower
 .text.LPM_DeepSleep
                0x00002608       0x1c ./DSP/Device/device.o
                0x00002608                LPM_DeepSleep
 .text.LPM_VLPS
                0x00002624       0x44 ./DSP/Device/device.o
                0x00002624                LPM_VLPS
 .text.UART0ClockGate
                0x00002668       0x78 ./DSP/DSP/DSP_mkl16z256vlh4.o
                0x00002668                UART0ClockGate
 .text.UART1ClockGate
                0x000026e0       0x4c ./DSP/DSP/DSP_mkl16z256vlh4.o
                0x000026e0                UART1ClockGate
 .text.UART2ClockGate
                0x0000272c       0x4c ./DSP/DSP/DSP_mkl16z256vlh4.o
                0x0000272c                UART2ClockGate
 .text.SPI0ClockGate
                0x00002778       0x4c ./DSP/DSP/DSP_mkl16z256vlh4.o
                0x00002778                SPI0ClockGate
 .text.SPI1ClockGate
                0x000027c4       0x4c ./DSP/DSP/DSP_mkl16z256vlh4.o
                0x000027c4                SPI1ClockGate
 .text.I2C0ClockGate
                0x00002810       0x48 ./DSP/DSP/DSP_mkl16z256vlh4.o
                0x00002810                I2C0ClockGate
 .text.UART0PinMappingPeripheral
                0x00002858       0x70 ./DSP/DSP/DSP_mkl16z256vlh4.o
                0x00002858                UART0PinMappingPeripheral
 .text.UART1PinMappingPeripheral
                0x000028c8       0x70 ./DSP/DSP/DSP_mkl16z256vlh4.o
                0x000028c8                UART1PinMappingPeripheral
 .text.UART2PinMappingPeripheral
                0x00002938       0x70 ./DSP/DSP/DSP_mkl16z256vlh4.o
                0x00002938                UART2PinMappingPeripheral
 .text.SPI0PinMappingPeripheral
                0x000029a8       0x70 ./DSP/DSP/DSP_mkl16z256vlh4.o
                0x000029a8                SPI0PinMappingPeripheral
 .text.SPI1PinMappingPeripheral
                0x00002a18       0xa0 ./DSP/DSP/DSP_mkl16z256vlh4.o
                0x00002a18                SPI1PinMappingPeripheral
 .text.I2C0PinMappingPeripheral
                0x00002ab8       0x70 ./DSP/DSP/DSP_mkl16z256vlh4.o
                0x00002ab8                I2C0PinMappingPeripheral
 .text.TickCallBack
                0x00002b28      0x110 ./BSP/Tick/tick.o
                0x00002b28                TickCallBack
 .text.TickInit
                0x00002c38       0x5c ./BSP/Tick/tick.o
                0x00002c38                TickInit
 .text.TickGetMsCounter
                0x00002c94       0x14 ./BSP/Tick/tick.o
                0x00002c94                TickGetMsCounter
 .text.TickMilliSecElapsedFrom
                0x00002ca8       0x30 ./BSP/Tick/tick.o
                0x00002ca8                TickMilliSecElapsedFrom
 .text.CR95HFWriteCommand
                0x00002cd8       0xfc ./BSP/RFID_CR95HF/CR95HF.o
                0x00002cd8                CR95HFWriteCommand
 .text.CR95HFReadAnswer
                0x00002dd4       0x48 ./BSP/RFID_CR95HF/CR95HF.o
                0x00002dd4                CR95HFReadAnswer
 .text.CR95HFBufCompare
                0x00002e1c       0xf0 ./BSP/RFID_CR95HF/CR95HF.o
                0x00002e1c                CR95HFBufCompare
 .text.CR95HFCommandManager
                0x00002f0c       0x8c ./BSP/RFID_CR95HF/CR95HF.o
                0x00002f0c                CR95HFCommandManager
 .text.CR95HFEchoStateMachine
                0x00002f98      0x110 ./BSP/RFID_CR95HF/CR95HF.o
                0x00002f98                CR95HFEchoStateMachine
 .text.CR95HFFieldOffStateMachine
                0x000030a8      0x100 ./BSP/RFID_CR95HF/CR95HF.o
                0x000030a8                CR95HFFieldOffStateMachine
 .text.CR95HFField15693StateMachine
                0x000031a8      0x100 ./BSP/RFID_CR95HF/CR95HF.o
                0x000031a8                CR95HFField15693StateMachine
 .text.CR95HFHibernateStateMachine
                0x000032a8      0x128 ./BSP/RFID_CR95HF/CR95HF.o
                0x000032a8                CR95HFHibernateStateMachine
 .text.CR95HFReadStateMachine
                0x000033d0      0x150 ./BSP/RFID_CR95HF/CR95HF.o
                0x000033d0                CR95HFReadStateMachine
 .text.CR95HFWriteStateMachine
                0x00003520      0x188 ./BSP/RFID_CR95HF/CR95HF.o
                0x00003520                CR95HFWriteStateMachine
 .text.CR95HFBridgeStateMachine
                0x000036a8       0xdc ./BSP/RFID_CR95HF/CR95HF.o
                0x000036a8                CR95HFBridgeStateMachine
 .text.CR95HFInit
                0x00003784       0x4c ./BSP/RFID_CR95HF/CR95HF.o
                0x00003784                CR95HFInit
 .text.CR95HFManager
                0x000037d0       0xbc ./BSP/RFID_CR95HF/CR95HF.o
                0x000037d0                CR95HFManager
 .text.CR95HFStartEcho
                0x0000388c       0x34 ./BSP/RFID_CR95HF/CR95HF.o
                0x0000388c                CR95HFStartEcho
 .text.CR95HFStartFieldOff
                0x000038c0       0x34 ./BSP/RFID_CR95HF/CR95HF.o
                0x000038c0                CR95HFStartFieldOff
 .text.CR95HFStartField15693
                0x000038f4       0x34 ./BSP/RFID_CR95HF/CR95HF.o
                0x000038f4                CR95HFStartField15693
 .text.CR95HFStartHibernate
                0x00003928       0x34 ./BSP/RFID_CR95HF/CR95HF.o
                0x00003928                CR95HFStartHibernate
 .text.CR95HFStartRead
                0x0000395c       0x48 ./BSP/RFID_CR95HF/CR95HF.o
                0x0000395c                CR95HFStartRead
 .text.CR95HFStartWrite
                0x000039a4       0x54 ./BSP/RFID_CR95HF/CR95HF.o
                0x000039a4                CR95HFStartWrite
 .text.CR95HFStartBridge
                0x000039f8       0x90 ./BSP/RFID_CR95HF/CR95HF.o
                0x000039f8                CR95HFStartBridge
 .text.CR95HFManagerIsReady
                0x00003a88       0x20 ./BSP/RFID_CR95HF/CR95HF.o
                0x00003a88                CR95HFManagerIsReady
 .text.CR95SelectDevice
                0x00003aa8       0x20 ./BSP/RFID_CR95HF/CR95UartMapper.o
                0x00003aa8                CR95SelectDevice
 .text.CR95UartInit
                0x00003ac8       0x60 ./BSP/RFID_CR95HF/CR95UartMapper.o
                0x00003ac8                CR95UartInit
 .text.CR95UartEnableReceiver
                0x00003b28       0x40 ./BSP/RFID_CR95HF/CR95UartMapper.o
                0x00003b28                CR95UartEnableReceiver
 .text.CR95UartDisableReceiver
                0x00003b68       0x30 ./BSP/RFID_CR95HF/CR95UartMapper.o
                0x00003b68                CR95UartDisableReceiver
 .text.CR95UartSendData
                0x00003b98       0x40 ./BSP/RFID_CR95HF/CR95UartMapper.o
                0x00003b98                CR95UartSendData
 .text.CR95UartReadChar
                0x00003bd8       0x28 ./BSP/RFID_CR95HF/CR95UartMapper.o
                0x00003bd8                CR95UartReadChar
 .text.CR95UartResetReceiver
                0x00003c00       0x5c ./BSP/RFID_CR95HF/CR95UartMapper.o
                0x00003c00                CR95UartResetReceiver
 .text.CR95UartGetUartStructCtrl
                0x00003c5c       0x24 ./BSP/RFID_CR95HF/CR95UartMapper.o
                0x00003c5c                CR95UartGetUartStructCtrl
 .text.CR95ExtGetConnectionState
                0x00003c80       0x8c ./BSP/RFID_CR95HF/CR95UartMapper.o
                0x00003c80                CR95ExtGetConnectionState
 .text.LedInit  0x00003d0c       0x54 ./BSP/Led/led.o
                0x00003d0c                LedInit
 .text.FM25V20Init
                0x00003d60       0xf4 ./BSP/FRAM/FM25V20.o
                0x00003d60                FM25V20Init
 .text.FM25V20_SetWriteEnable
                0x00003e54       0x7c ./BSP/FRAM/FM25V20.o
                0x00003e54                FM25V20_SetWriteEnable
 .text.FM25V20SetStatusReg
                0x00003ed0       0x98 ./BSP/FRAM/FM25V20.o
                0x00003ed0                FM25V20SetStatusReg
 .text.FM25V20LPM
                0x00003f68       0x60 ./BSP/FRAM/FM25V20.o
                0x00003f68                FM25V20LPM
 .text.FM25V20WakeUp
                0x00003fc8       0x58 ./BSP/FRAM/FM25V20.o
                0x00003fc8                FM25V20WakeUp
 .text.FM25V20WriteData
                0x00004020       0xd0 ./BSP/FRAM/FM25V20.o
                0x00004020                FM25V20WriteData
 .text.FM25V20ReadData
                0x000040f0       0xa4 ./BSP/FRAM/FM25V20.o
                0x000040f0                FM25V20ReadData
 .text.FM25V20IsInLowPower
                0x00004194       0x14 ./BSP/FRAM/FM25V20.o
                0x00004194                FM25V20IsInLowPower
 .text.DisplayInit
                0x000041a8       0xb8 ./BSP/Display/display.o
                0x000041a8                DisplayInit
 .text.DisplaySetDataDisplayed
                0x00004260      0x120 ./BSP/Display/display.o
                0x00004260                DisplaySetDataDisplayed
 .text.DisplayGetDataDisplayed
                0x00004380       0x4c ./BSP/Display/display.o
                0x00004380                DisplayGetDataDisplayed
 .text.DisplayDigitTo7Seg
                0x000043cc      0x2d8 ./BSP/Display/display.o
                0x000043cc                DisplayDigitTo7Seg
 .text.DisplayDigitTo16Seg
                0x000046a4      0x21c ./BSP/Display/display.o
                0x000046a4                DisplayDigitTo16Seg
 .text.DisplaySetPower
                0x000048c0       0xd0 ./BSP/Display/display.o
                0x000048c0                DisplaySetPower
 .text.ButtonInit
                0x00004990       0x48 ./BSP/Button/button.o
                0x00004990                ButtonInit
 .text.BQ27510DRZRG2_Init
                0x000049d8       0x24 ./BSP/BatteryManagement/BQ27510DRZRG2.o
                0x000049d8                BQ27510DRZRG2_Init
 .text.BQ_batteryIsConnected
                0x000049fc       0x2c ./BSP/BatteryManagement/BQ27510DRZRG2.o
                0x000049fc                BQ_batteryIsConnected
 .text.BQ_getCellTemperature
                0x00004a28       0x8c ./BSP/BatteryManagement/BQ27510DRZRG2.o
                0x00004a28                BQ_getCellTemperature
 .text.BQ_getCellVoltage
                0x00004ab4       0x70 ./BSP/BatteryManagement/BQ27510DRZRG2.o
                0x00004ab4                BQ_getCellVoltage
 .text.BQ_getNominalAvailableCapacity
                0x00004b24       0x70 ./BSP/BatteryManagement/BQ27510DRZRG2.o
                0x00004b24                BQ_getNominalAvailableCapacity
 .text.BQ_getFullAvailableCapacity
                0x00004b94       0x70 ./BSP/BatteryManagement/BQ27510DRZRG2.o
                0x00004b94                BQ_getFullAvailableCapacity
 .text.BQ_getRemainingCapacity
                0x00004c04       0x70 ./BSP/BatteryManagement/BQ27510DRZRG2.o
                0x00004c04                BQ_getRemainingCapacity
 .text.BQ_getFullChargeCapacity
                0x00004c74       0x70 ./BSP/BatteryManagement/BQ27510DRZRG2.o
                0x00004c74                BQ_getFullChargeCapacity
 .text.BQ_getAverageCurrent
                0x00004ce4       0x74 ./BSP/BatteryManagement/BQ27510DRZRG2.o
                0x00004ce4                BQ_getAverageCurrent
 .text.BQ_getTimeToEmpty
                0x00004d58       0x70 ./BSP/BatteryManagement/BQ27510DRZRG2.o
                0x00004d58                BQ_getTimeToEmpty
 .text.BQ_getTimeToFull
                0x00004dc8       0x70 ./BSP/BatteryManagement/BQ27510DRZRG2.o
                0x00004dc8                BQ_getTimeToFull
 .text.BQ_getStandbyTimeToEmpty
                0x00004e38       0x70 ./BSP/BatteryManagement/BQ27510DRZRG2.o
                0x00004e38                BQ_getStandbyTimeToEmpty
 .text.BQ_getMaxLoadCurrent
                0x00004ea8       0x74 ./BSP/BatteryManagement/BQ27510DRZRG2.o
                0x00004ea8                BQ_getMaxLoadCurrent
 .text.BQ_getMaxLoadTimeToEmpty
                0x00004f1c       0x70 ./BSP/BatteryManagement/BQ27510DRZRG2.o
                0x00004f1c                BQ_getMaxLoadTimeToEmpty
 .text.BQ_getAvailableEnergy
                0x00004f8c       0x78 ./BSP/BatteryManagement/BQ27510DRZRG2.o
                0x00004f8c                BQ_getAvailableEnergy
 .text.BQ_getAveragePower
                0x00005004       0x74 ./BSP/BatteryManagement/BQ27510DRZRG2.o
                0x00005004                BQ_getAveragePower
 .text.BQ_getTTEAtConstantPower
                0x00005078       0x70 ./BSP/BatteryManagement/BQ27510DRZRG2.o
                0x00005078                BQ_getTTEAtConstantPower
 .text.BQ_getCycleCount
                0x000050e8       0x70 ./BSP/BatteryManagement/BQ27510DRZRG2.o
                0x000050e8                BQ_getCycleCount
 .text.BQ_getStateOfCharge
                0x00005158       0x70 ./BSP/BatteryManagement/BQ27510DRZRG2.o
                0x00005158                BQ_getStateOfCharge
 .text.BQ_getFullInfo
                0x000051c8      0x168 ./BSP/BatteryManagement/BQ27510DRZRG2.o
                0x000051c8                BQ_getFullInfo
 .text.LTC4160Init
                0x00005330       0xbc ./BSP/BatteryManagement/LTC4160.o
                0x00005330                LTC4160Init
 .text.LTC4160SetILimit
                0x000053ec       0x30 ./BSP/BatteryManagement/LTC4160.o
                0x000053ec                LTC4160SetILimit
 .text.UsbManager
                0x0000541c      0x2c8 ./Application/UsbManager/UsbManager.o
                0x0000541c                UsbManager
 .text.UsbManagerCmdDealer
                0x000056e4      0x838 ./Application/UsbManager/UsbManager.o
                0x000056e4                UsbManagerCmdDealer
 .text.UsbManagerSendCR95Error
                0x00005f1c       0x40 ./Application/UsbManager/UsbManager.o
                0x00005f1c                UsbManagerSendCR95Error
 .text.UsbManagerSendCR95Result
                0x00005f5c       0x40 ./Application/UsbManager/UsbManager.o
                0x00005f5c                UsbManagerSendCR95Result
 .text.RFIDManagerInit
                0x00005f9c       0x38 ./Application/RFIDManager/RFIDManager.o
                0x00005f9c                RFIDManagerInit
 .text.RFIDManager
                0x00005fd4      0x118 ./Application/RFIDManager/RFIDManager.o
                0x00005fd4                RFIDManager
 .text.RFIDDealer
                0x000060ec       0x54 ./Application/RFIDManager/RFIDManager.o
                0x000060ec                RFIDDealer
 .text.RFIDIntLpmStateMachine
                0x00006140      0x104 ./Application/RFIDManager/RFIDManager.o
                0x00006140                RFIDIntLpmStateMachine
 .text.RFIDExtLpmStateMachine
                0x00006244      0x104 ./Application/RFIDManager/RFIDManager.o
                0x00006244                RFIDExtLpmStateMachine
 .text.RFIDBridgeStateMachine
                0x00006348      0x1c0 ./Application/RFIDManager/RFIDManager.o
                0x00006348                RFIDBridgeStateMachine
 .text.RFIDReadStateMachine
                0x00006508      0x1f4 ./Application/RFIDManager/RFIDManager.o
                0x00006508                RFIDReadStateMachine
 .text.RFIDWriteStateMachine
                0x000066fc      0x468 ./Application/RFIDManager/RFIDManager.o
                0x000066fc                RFIDWriteStateMachine
 .text.RFIDManagerSendBridgeCommand
                0x00006b64       0x74 ./Application/RFIDManager/RFIDManager.o
                0x00006b64                RFIDManagerSendBridgeCommand
 .text.PORTA_IRQHandler
                0x00006bd8        0xc ./Application/PowerManager/PowerManager.o
                0x00006bd8                PORTA_IRQHandler
 .text.PowerManagerInit
                0x00006be4       0x70 ./Application/PowerManager/PowerManager.o
                0x00006be4                PowerManagerInit
 .text.PowerManager
                0x00006c54      0x104 ./Application/PowerManager/PowerManager.o
                0x00006c54                PowerManager
 .text.PowerManagerDisplayLoading
                0x00006d58       0x88 ./Application/PowerManager/PowerManager.o
                0x00006d58                PowerManagerDisplayLoading
 .text.PowerManagerDisplayLoadingError
                0x00006de0       0x34 ./Application/PowerManager/PowerManager.o
                0x00006de0                PowerManagerDisplayLoadingError
 .text.PowerManagerDisplayLoaded
                0x00006e14       0x2c ./Application/PowerManager/PowerManager.o
                0x00006e14                PowerManagerDisplayLoaded
 .text.PowerManagerEnterLPM
                0x00006e40       0xdc ./Application/PowerManager/PowerManager.o
                0x00006e40                PowerManagerEnterLPM
 .text.PowerManagerExitLPM
                0x00006f1c       0x4c ./Application/PowerManager/PowerManager.o
                0x00006f1c                PowerManagerExitLPM
 .text.PowerManagerEnableWakeUpInterrupt
                0x00006f68       0x4c ./Application/PowerManager/PowerManager.o
                0x00006f68                PowerManagerEnableWakeUpInterrupt
 .text.PowerManagerDisableWakeUpInterrupt
                0x00006fb4       0x34 ./Application/PowerManager/PowerManager.o
                0x00006fb4                PowerManagerDisableWakeUpInterrupt
 .text.PowerManagerClearWakeUpInterruptFlag
                0x00006fe8       0x38 ./Application/PowerManager/PowerManager.o
                0x00006fe8                PowerManagerClearWakeUpInterruptFlag
 .text.PowerManagerLPMController
                0x00007020       0x68 ./Application/PowerManager/PowerManager.o
                0x00007020                PowerManagerLPMController
 .text.MemoryManagerInit
                0x00007088       0x98 ./Application/MemoryManager/MemoryManager.o
                0x00007088                MemoryManagerInit
 .text.MemoryManagerReadDiving
                0x00007120       0x6c ./Application/MemoryManager/MemoryManager.o
                0x00007120                MemoryManagerReadDiving
 .text.MemoryManagerCheckDiving
                0x0000718c       0x60 ./Application/MemoryManager/MemoryManager.o
                0x0000718c                MemoryManagerCheckDiving
 .text.MemoryManagerWriteDiving
                0x000071ec       0xac ./Application/MemoryManager/MemoryManager.o
                0x000071ec                MemoryManagerWriteDiving
 .text.MemoryManagerReadSerial
                0x00007298       0x6c ./Application/MemoryManager/MemoryManager.o
                0x00007298                MemoryManagerReadSerial
 .text.MemoryManagerCheckSerial
                0x00007304       0x54 ./Application/MemoryManager/MemoryManager.o
                0x00007304                MemoryManagerCheckSerial
 .text.MemoryManagerWriteSerial
                0x00007358       0xa0 ./Application/MemoryManager/MemoryManager.o
                0x00007358                MemoryManagerWriteSerial
 .text.MemoryManagerWriteLog
                0x000073f8      0x11c ./Application/MemoryManager/MemoryManager.o
                0x000073f8                MemoryManagerWriteLog
 .text.MemoryManagerClearLog
                0x00007514       0xcc ./Application/MemoryManager/MemoryManager.o
                0x00007514                MemoryManagerClearLog
 .text.MemoryManagerComputeNbrLog
                0x000075e0       0xb4 ./Application/MemoryManager/MemoryManager.o
                0x000075e0                MemoryManagerComputeNbrLog
 .text.MemoryManagerReadLog
                0x00007694       0xd0 ./Application/MemoryManager/MemoryManager.o
                0x00007694                MemoryManagerReadLog
 .text.ButtonManagerDealer
                0x00007764      0x2c4 ./Application/ButtonManager/ButtonManager.o
                0x00007764                ButtonManagerDealer
 .text.ButtonManagerDisplayProgrammedError
                0x00007a28       0x34 ./Application/ButtonManager/ButtonManager.o
                0x00007a28                ButtonManagerDisplayProgrammedError
 .text.ButtonManagerDisplayDateError
                0x00007a5c       0x34 ./Application/ButtonManager/ButtonManager.o
                0x00007a5c                ButtonManagerDisplayDateError
 .text.ButtonManagerDisplayRfidError
                0x00007a90       0x34 ./Application/ButtonManager/ButtonManager.o
                0x00007a90                ButtonManagerDisplayRfidError
 .text.ButtonManagerDisplayRead
                0x00007ac4      0x164 ./Application/ButtonManager/ButtonManager.o
                0x00007ac4                ButtonManagerDisplayRead
 .text.ButtonManagerDisplayWrite
                0x00007c28       0xb0 ./Application/ButtonManager/ButtonManager.o
                0x00007c28                ButtonManagerDisplayWrite
 .text.ButtonManagerDisplayWriteError
                0x00007cd8       0x34 ./Application/ButtonManager/ButtonManager.o
                0x00007cd8                ButtonManagerDisplayWriteError
 .text.ButtonManagerDisplayLogError
                0x00007d0c       0x34 ./Application/ButtonManager/ButtonManager.o
                0x00007d0c                ButtonManagerDisplayLogError
 .text.ButtonManagerDisplayNone
                0x00007d40       0x20 ./Application/ButtonManager/ButtonManager.o
                0x00007d40                ButtonManagerDisplayNone
 .text.ButtonManagerInit
                0x00007d60       0x54 ./Application/ButtonManager/ButtonManager.o
                0x00007d60                ButtonManagerInit
 .text.ButtonManager
                0x00007db4      0x6c4 ./Application/ButtonManager/ButtonManager.o
                0x00007db4                ButtonManager
 .text.main     0x00008478       0xac ./Application/main.o
                0x00008478                main
 .text.CriticalInit
                0x00008524       0x28 ./Application/main.o
                0x00008524                CriticalInit
 .text.Setup    0x0000854c       0x64 ./Application/main.o
                0x0000854c                Setup
 .text.StartScheduling
                0x000085b0       0x34 ./Application/main.o
                0x000085b0                StartScheduling
 .text.task10ms
                0x000085e4        0x8 ./Application/main.o
                0x000085e4                task10ms
 .text.task100ms
                0x000085ec        0x8 ./Application/main.o
                0x000085ec                task100ms
 .text.task1s   0x000085f4        0xc ./Application/main.o
                0x000085f4                task1s
 .text.task1min
                0x00008600        0x8 ./Application/main.o
                0x00008600                task1min
 .text.taskBackground
                0x00008608       0x18 ./Application/main.o
                0x00008608                taskBackground
 .text.taskSchedulerOverrun
                0x00008620        0x8 ./Application/main.o
                0x00008620                taskSchedulerOverrun
 .text.atexit   0x00008628       0x10 e:/logiciels/freescale/kinetis design studio v2.0.0/toolchain/bin/../lib/gcc/arm-none-eabi/4.8.0/../../../../arm-none-eabi/lib\libg_s.a(lib_a-atexit.o)
                0x00008628                atexit
 .text.exit     0x00008638       0x30 e:/logiciels/freescale/kinetis design studio v2.0.0/toolchain/bin/../lib/gcc/arm-none-eabi/4.8.0/../../../../arm-none-eabi/lib\libg_s.a(lib_a-exit.o)
                0x00008638                exit
 .text.__libc_fini_array
                0x00008668       0x28 e:/logiciels/freescale/kinetis design studio v2.0.0/toolchain/bin/../lib/gcc/arm-none-eabi/4.8.0/../../../../arm-none-eabi/lib\libg_s.a(lib_a-fini.o)
                0x00008668                __libc_fini_array
 .text.memcpy   0x00008690       0x12 e:/logiciels/freescale/kinetis design studio v2.0.0/toolchain/bin/../lib/gcc/arm-none-eabi/4.8.0/../../../../arm-none-eabi/lib\libg_s.a(lib_a-memcpy.o)
                0x00008690                memcpy
 .text.memset   0x000086a2       0x12 e:/logiciels/freescale/kinetis design studio v2.0.0/toolchain/bin/../lib/gcc/arm-none-eabi/4.8.0/../../../../arm-none-eabi/lib\libg_s.a(lib_a-memset.o)
                0x000086a2                memset
 .text._kill    0x000086b4       0x24 e:/logiciels/freescale/kinetis design studio v2.0.0/toolchain/bin/../lib/gcc/arm-none-eabi/4.8.0/../../../../arm-none-eabi/lib\libg_s.a(lib_a-syscalls.o)
                0x000086b4                _kill
 .text._exit    0x000086d8        0xc e:/logiciels/freescale/kinetis design studio v2.0.0/toolchain/bin/../lib/gcc/arm-none-eabi/4.8.0/../../../../arm-none-eabi/lib\libg_s.a(lib_a-syscalls.o)
                0x000086d8                _exit
 .text._sbrk    0x000086e4       0x38 e:/logiciels/freescale/kinetis design studio v2.0.0/toolchain/bin/../lib/gcc/arm-none-eabi/4.8.0/../../../../arm-none-eabi/lib\libg_s.a(lib_a-syscalls.o)
                0x000086e4                _sbrk
 .text.__do_register_exitproc
                0x0000871c       0x80 e:/logiciels/freescale/kinetis design studio v2.0.0/toolchain/bin/../lib/gcc/arm-none-eabi/4.8.0/../../../../arm-none-eabi/lib\libg_s.a(lib_a-__atexit.o)
                0x0000871c                __do_register_exitproc
 .text.__call_exitprocs
                0x0000879c       0xa8 e:/logiciels/freescale/kinetis design studio v2.0.0/toolchain/bin/../lib/gcc/arm-none-eabi/4.8.0/../../../../arm-none-eabi/lib\libg_s.a(lib_a-__call_atexit.o)
                0x0000879c                __call_exitprocs
 .text.__errno  0x00008844        0xc e:/logiciels/freescale/kinetis design studio v2.0.0/toolchain/bin/../lib/gcc/arm-none-eabi/4.8.0/../../../../arm-none-eabi/lib\libg_s.a(lib_a-errno.o)
                0x00008844                __errno
 .text.malloc   0x00008850       0x14 e:/logiciels/freescale/kinetis design studio v2.0.0/toolchain/bin/../lib/gcc/arm-none-eabi/4.8.0/../../../../arm-none-eabi/lib\libg_s.a(lib_a-malloc.o)
                0x00008850                malloc
 .text.free     0x00008864       0x14 e:/logiciels/freescale/kinetis design studio v2.0.0/toolchain/bin/../lib/gcc/arm-none-eabi/4.8.0/../../../../arm-none-eabi/lib\libg_s.a(lib_a-malloc.o)
                0x00008864                free
 .text._malloc_r
                0x00008878       0x98 e:/logiciels/freescale/kinetis design studio v2.0.0/toolchain/bin/../lib/gcc/arm-none-eabi/4.8.0/../../../../arm-none-eabi/lib\libg_s.a(lib_a-mallocr.o)
                0x00008878                _malloc_r
 .text._sbrk_r  0x00008910       0x24 e:/logiciels/freescale/kinetis design studio v2.0.0/toolchain/bin/../lib/gcc/arm-none-eabi/4.8.0/../../../../arm-none-eabi/lib\libg_s.a(lib_a-sbrkr.o)
                0x00008910                _sbrk_r
 .text._free_r  0x00008934       0x90 e:/logiciels/freescale/kinetis design studio v2.0.0/toolchain/bin/../lib/gcc/arm-none-eabi/4.8.0/../../../../arm-none-eabi/lib\libg_s.a(lib_a-freer.o)
                0x00008934                _free_r
 *(.rodata)
 .rodata        0x000089c4        0x4 ./Application/UsbManager/UsbManager.o
 .rodata        0x000089c8       0x68 ./Application/PowerManager/PowerManager.o
 .rodata        0x00008a30       0x14 ./Application/ButtonManager/ButtonManager.o
 *(.rodata*)
 .rodata.Decode7segDigitASCII
                0x00008a44      0x120 ./Tools/Decoder7Seg/decoder7Seg.o
 .rodata.Decode16segDigitASCII
                0x00008b64      0x148 ./Tools/Decoder16Seg/decoder16Seg.o
 .rodata.CR95HFCommandManager
                0x00008cac       0x20 ./BSP/RFID_CR95HF/CR95HF.o
 .rodata.RFIDDealer
                0x00008ccc       0x84 ./Application/RFIDManager/RFIDManager.o
 .rodata.RFIDIntLpmStateMachine
                0x00008d50       0x20 ./Application/RFIDManager/RFIDManager.o
 .rodata.RFIDExtLpmStateMachine
                0x00008d70       0x20 ./Application/RFIDManager/RFIDManager.o
 .rodata.RFIDBridgeStateMachine
                0x00008d90       0x30 ./Application/RFIDManager/RFIDManager.o
 .rodata.RFIDReadStateMachine
                0x00008dc0       0x28 ./Application/RFIDManager/RFIDManager.o
 .rodata.RFIDWriteStateMachine
                0x00008de8       0x54 ./Application/RFIDManager/RFIDManager.o
 .rodata.ButtonManagerDealer
                0x00008e3c       0x2c ./Application/ButtonManager/ButtonManager.o
 .rodata.str1.1
                0x00008e68        0x2 e:/logiciels/freescale/kinetis design studio v2.0.0/toolchain/bin/../lib/gcc/arm-none-eabi/4.8.0/../../../../arm-none-eabi/lib\libg_s.a(lib_a-impure.o)
 *fill*         0x00008e6a        0x2 
 .rodata._global_impure_ptr
                0x00008e6c        0x4 e:/logiciels/freescale/kinetis design studio v2.0.0/toolchain/bin/../lib/gcc/arm-none-eabi/4.8.0/../../../../arm-none-eabi/lib\libg_s.a(lib_a-impure.o)
                0x00008e6c                _global_impure_ptr
 *(.glue_7)
 .glue_7        0x00000000        0x0 linker stubs
 *(.glue_7t)
 .glue_7t       0x00000000        0x0 linker stubs
 *(.eh_frame)
 .eh_frame      0x00008e70        0x0 e:/logiciels/freescale/kinetis design studio v2.0.0/toolchain/bin/../lib/gcc/arm-none-eabi/4.8.0/crtbegin.o
 *(.init)
 .init          0x00008e70        0x4 e:/logiciels/freescale/kinetis design studio v2.0.0/toolchain/bin/../lib/gcc/arm-none-eabi/4.8.0/crti.o
                0x00008e70                _init
 .init          0x00008e74        0x8 e:/logiciels/freescale/kinetis design studio v2.0.0/toolchain/bin/../lib/gcc/arm-none-eabi/4.8.0/crtn.o
 *(.fini)
 .fini          0x00008e7c        0x4 e:/logiciels/freescale/kinetis design studio v2.0.0/toolchain/bin/../lib/gcc/arm-none-eabi/4.8.0/crti.o
                0x00008e7c                _fini
 .fini          0x00008e80        0x8 e:/logiciels/freescale/kinetis design studio v2.0.0/toolchain/bin/../lib/gcc/arm-none-eabi/4.8.0/crtn.o
                0x00008e88                . = ALIGN (0x4)

.vfp11_veneer   0x00008e88        0x0
 .vfp11_veneer  0x00000000        0x0 linker stubs

.v4_bx          0x00008e88        0x0
 .v4_bx         0x00000000        0x0 linker stubs

.iplt           0x00008e88        0x0
 .iplt          0x00000000        0x0 e:/logiciels/freescale/kinetis design studio v2.0.0/toolchain/bin/../lib/gcc/arm-none-eabi/4.8.0/crtbegin.o

.rel.dyn        0x00008e88        0x0
 .rel.iplt      0x00000000        0x0 e:/logiciels/freescale/kinetis design studio v2.0.0/toolchain/bin/../lib/gcc/arm-none-eabi/4.8.0/crtbegin.o

.ARM.extab
 *(.ARM.extab* .gnu.linkonce.armextab.*)

.ARM            0x00008e88        0x0
                0x00008e88                __exidx_start = .
 *(.ARM.exidx*)
                0x00008e88                __exidx_end = .

.ctors          0x00008e88        0x0
                0x00008e88                __CTOR_LIST__ = .
 *crtbegin.o(.ctors)
 *crtbegin?.o(.ctors)
 *(EXCLUDE_FILE(*crtend.o *crtend?.o) .ctors)
 *(SORT(.ctors.*))
 *(.ctors)
                0x00008e88                __CTOR_END__ = .

.dtors          0x00008e88        0x0
                0x00008e88                __DTOR_LIST__ = .
 *crtbegin.o(.dtors)
 *crtbegin?.o(.dtors)
 *(EXCLUDE_FILE(*crtend.o *crtend?.o) .dtors)
 *(SORT(.dtors.*))
 *(.dtors)
                0x00008e88                __DTOR_END__ = .

.preinit_array  0x00008e88        0x0
                0x00008e88                PROVIDE (__preinit_array_start, .)
 *(.preinit_array*)
                0x00008e88                PROVIDE (__preinit_array_end, .)

.init_array     0x00008e88        0x4
                0x00008e88                PROVIDE (__init_array_start, .)
 *(SORT(.init_array.*))
 *(.init_array*)
 .init_array    0x00008e88        0x4 e:/logiciels/freescale/kinetis design studio v2.0.0/toolchain/bin/../lib/gcc/arm-none-eabi/4.8.0/crtbegin.o
                0x00008e8c                PROVIDE (__init_array_end, .)

.fini_array     0x00008e8c        0x4
                0x00008e8c                PROVIDE (__fini_array_start, .)
 *(SORT(.fini_array.*))
 *(.fini_array*)
 .fini_array    0x00008e8c        0x4 e:/logiciels/freescale/kinetis design studio v2.0.0/toolchain/bin/../lib/gcc/arm-none-eabi/4.8.0/crtbegin.o
                0x00008e90                PROVIDE (__fini_array_end, .)
                0x00008e90                __etext = .
                0x00008e90                __DATA_ROM = .

.mtb            0x1fffe000        0x0
                0x1fffe000                . = ALIGN (0x8)
                0x1fffe000                _mtb_start = .
 *(.mtb_buf)
                0x1fffe000                . = ALIGN (0x8)
                0x1fffe000                _mtb_end = .

.data           0x1fffe000      0x2a8 load address 0x00008e90
                0x1fffe000                . = ALIGN (0x4)
                0x1fffe000                __DATA_RAM = .
                0x1fffe000                __data_start__ = .
 *(.data)
 *(.data*)
 .data.PitISRCallBack
                0x1fffe000        0x8 ./DSP/PIT/pit.o
                0x1fffe000                PitISRCallBack
 .data.impure_data
                0x1fffe008      0x298 e:/logiciels/freescale/kinetis design studio v2.0.0/toolchain/bin/../lib/gcc/arm-none-eabi/4.8.0/../../../../arm-none-eabi/lib\libg_s.a(lib_a-impure.o)
 .data._impure_ptr
                0x1fffe2a0        0x4 e:/logiciels/freescale/kinetis design studio v2.0.0/toolchain/bin/../lib/gcc/arm-none-eabi/4.8.0/../../../../arm-none-eabi/lib\libg_s.a(lib_a-impure.o)
                0x1fffe2a0                _impure_ptr
 *(.jcr*)
 .jcr           0x1fffe2a4        0x0 e:/logiciels/freescale/kinetis design studio v2.0.0/toolchain/bin/../lib/gcc/arm-none-eabi/4.8.0/crtbegin.o
 .jcr           0x1fffe2a4        0x4 e:/logiciels/freescale/kinetis design studio v2.0.0/toolchain/bin/../lib/gcc/arm-none-eabi/4.8.0/crtend.o
                0x1fffe2a8                . = ALIGN (0x4)
                0x1fffe2a8                __data_end__ = .
                0x00009138                __DATA_END = (__DATA_ROM + (__data_end__ - __data_start__))

.tm_clone_table
                0x1fffe2a8        0x0 load address 0x00009138
 .tm_clone_table
                0x1fffe2a8        0x0 e:/logiciels/freescale/kinetis design studio v2.0.0/toolchain/bin/../lib/gcc/arm-none-eabi/4.8.0/crtbegin.o
 .tm_clone_table
                0x1fffe2a8        0x0 e:/logiciels/freescale/kinetis design studio v2.0.0/toolchain/bin/../lib/gcc/arm-none-eabi/4.8.0/crtend.o

.igot.plt       0x1fffe2a8        0x0 load address 0x00009138
 .igot.plt      0x00000000        0x0 e:/logiciels/freescale/kinetis design studio v2.0.0/toolchain/bin/../lib/gcc/arm-none-eabi/4.8.0/crtbegin.o

.bss            0x1fffe2a8      0x49c load address 0x00009138
                0x1fffe2a8                . = ALIGN (0x4)
                0x1fffe2a8                __START_BSS = .
                0x1fffe2a8                __bss_start__ = .
 *(.bss)
 *(.bss*)
 .bss.completed.6137
                0x1fffe2a8        0x1 e:/logiciels/freescale/kinetis design studio v2.0.0/toolchain/bin/../lib/gcc/arm-none-eabi/4.8.0/crtbegin.o
 *fill*         0x1fffe2a9        0x3 
 .bss.object.6142
                0x1fffe2ac       0x18 e:/logiciels/freescale/kinetis design studio v2.0.0/toolchain/bin/../lib/gcc/arm-none-eabi/4.8.0/crtbegin.o
 .bss.RtcUpdated
                0x1fffe2c4        0x1 ./DSP/RTC/rtc.o
                0x1fffe2c4                RtcUpdated
 *fill*         0x1fffe2c5        0x3 
 .bss.I2C0Baudrate
                0x1fffe2c8        0x4 ./DSP/I2C/i2c0.o
                0x1fffe2c8                I2C0Baudrate
 .bss.msCounter
                0x1fffe2cc        0x4 ./BSP/Tick/tick.o
                0x1fffe2cc                msCounter
 .bss.tryCounter.4993
                0x1fffe2d0        0x1 ./BSP/RFID_CR95HF/CR95HF.o
 .bss.CR95DeviceSelected
                0x1fffe2d1        0x1 ./BSP/RFID_CR95HF/CR95UartMapper.o
                0x1fffe2d1                CR95DeviceSelected
 .bss.FM25V20_Lpm
                0x1fffe2d2        0x1 ./BSP/FRAM/FM25V20.o
                0x1fffe2d2                FM25V20_Lpm
 *fill*         0x1fffe2d3        0x1 
 .bss.currentDigit
                0x1fffe2d4        0x4 ./BSP/Display/display.o
                0x1fffe2d4                currentDigit
 .bss.displayPower
                0x1fffe2d8        0x1 ./BSP/Display/display.o
                0x1fffe2d8                displayPower
 .bss.RFIDInternalPowerMode
                0x1fffe2d9        0x1 ./Application/RFIDManager/RFIDManager.o
                0x1fffe2d9                RFIDInternalPowerMode
 .bss.RFIDExternalPowerMode
                0x1fffe2da        0x1 ./Application/RFIDManager/RFIDManager.o
                0x1fffe2da                RFIDExternalPowerMode
 *fill*         0x1fffe2db        0x1 
 .bss.msRef.5671
                0x1fffe2dc        0x4 ./Application/RFIDManager/RFIDManager.o
 .bss.addr.5690
                0x1fffe2e0        0x2 ./Application/RFIDManager/RFIDManager.o
 *fill*         0x1fffe2e2        0x2 
 .bss.msRef.5691
                0x1fffe2e4        0x4 ./Application/RFIDManager/RFIDManager.o
 .bss.addr.5708
                0x1fffe2e8        0x2 ./Application/RFIDManager/RFIDManager.o
 *fill*         0x1fffe2ea        0x2 
 .bss.msRef.5709
                0x1fffe2ec        0x4 ./Application/RFIDManager/RFIDManager.o
 .bss.locCounter.5630
                0x1fffe2f0        0x1 ./Application/PowerManager/PowerManager.o
 .bss.lastWriteBpState
                0x1fffe2f1        0x1 ./Application/ButtonManager/ButtonManager.o
                0x1fffe2f1                lastWriteBpState
 .bss.lastReadBpState
                0x1fffe2f2        0x1 ./Application/ButtonManager/ButtonManager.o
                0x1fffe2f2                lastReadBpState
 .bss.waitAllUnpressed
                0x1fffe2f3        0x1 ./Application/ButtonManager/ButtonManager.o
                0x1fffe2f3                waitAllUnpressed
 .bss.writeBpMsRef
                0x1fffe2f4        0x4 ./Application/ButtonManager/ButtonManager.o
                0x1fffe2f4                writeBpMsRef
 .bss.readBpMsRef
                0x1fffe2f8        0x4 ./Application/ButtonManager/ButtonManager.o
                0x1fffe2f8                readBpMsRef
 .bss.msRef.5636
                0x1fffe2fc        0x4 ./Application/ButtonManager/ButtonManager.o
 .bss.state.5691
                0x1fffe300        0x1 ./Application/ButtonManager/ButtonManager.o
 *fill*         0x1fffe301        0x3 
 .bss.msRef.5692
                0x1fffe304        0x4 ./Application/ButtonManager/ButtonManager.o
 .bss.heap_end.5175
                0x1fffe308        0x4 e:/logiciels/freescale/kinetis design studio v2.0.0/toolchain/bin/../lib/gcc/arm-none-eabi/4.8.0/../../../../arm-none-eabi/lib\libg_s.a(lib_a-syscalls.o)
 .bss.__malloc_free_list
                0x1fffe30c        0x4 e:/logiciels/freescale/kinetis design studio v2.0.0/toolchain/bin/../lib/gcc/arm-none-eabi/4.8.0/../../../../arm-none-eabi/lib\libg_s.a(lib_a-mallocr.o)
                0x1fffe30c                __malloc_free_list
 *(COMMON)
 COMMON         0x1fffe310       0x1c ./DSP/UART/uart0.o
                0x1fffe310                Uart0Ctrl
 COMMON         0x1fffe32c      0x11c ./DSP/UART/uart1.o
                0x1fffe32c                txBuf
                0x1fffe3ac                rxBuf
                0x1fffe42c                Uart1Ctrl
 COMMON         0x1fffe448       0x1c ./DSP/UART/uart2.o
                0x1fffe448                Uart2Ctrl
 COMMON         0x1fffe464        0x4 ./DSP/SPI/spi0.o
                0x1fffe464                Spi0Baudrate
 COMMON         0x1fffe468        0x4 ./DSP/SPI/spi1.o
                0x1fffe468                Spi1Baudrate
 COMMON         0x1fffe46c       0x2c ./DSP/DSP/DSP_mkl16z256vlh4.o
                0x1fffe46c                DeviceClock
 COMMON         0x1fffe498       0x14 ./BSP/Tick/tick.o
                0x1fffe498                TickCtrl
 COMMON         0x1fffe4ac      0x128 ./BSP/RFID_CR95HF/CR95HF.o
                0x1fffe4ac                CR95HFCtrl
 COMMON         0x1fffe5d4       0x28 ./BSP/BatteryManagement/BQ27510DRZRG2.o
                0x1fffe5d4                BQBatteryStatus
 COMMON         0x1fffe5fc       0x90 ./Application/UsbManager/UsbManager.o
                0x1fffe5fc                UsbCtrl
 COMMON         0x1fffe68c       0x90 ./Application/RFIDManager/RFIDManager.o
                0x1fffe68c                SRDEeprom
                0x1fffe6cc                RFIDCtrl
 COMMON         0x1fffe71c        0x2 ./Application/PowerManager/PowerManager.o
                0x1fffe71c                PowerManagerCtrl
 *fill*         0x1fffe71e        0x2 
 COMMON         0x1fffe720       0x1c ./Application/MemoryManager/MemoryManager.o
                0x1fffe720                SerialParameters
                0x1fffe730                DivingParameters
                0x1fffe734                MemoryManagerCtrl
 COMMON         0x1fffe73c        0x4 ./Application/ButtonManager/ButtonManager.o
                0x1fffe73c                ButtonManagerCtrl
 COMMON         0x1fffe740        0x4 e:/logiciels/freescale/kinetis design studio v2.0.0/toolchain/bin/../lib/gcc/arm-none-eabi/4.8.0/../../../../arm-none-eabi/lib\libg_s.a(lib_a-reent.o)
                0x1fffe740                errno
                0x1fffe744                . = ALIGN (0x4)
                0x1fffe744                __bss_end__ = .
                0x1fffe744                __END_BSS = .

.heap           0x1fffe744      0x404 load address 0x000095d4
                0x1fffe748                . = ALIGN (0x8)
 *fill*         0x1fffe744        0x4 
                0x1fffe748                __end__ = .
                0x1fffe748                PROVIDE (end, .)
                0x1fffe748                __HeapBase = .
                0x1fffeb48                . = (. + HEAP_SIZE)
 *fill*         0x1fffe748      0x400 
                0x1fffeb48                __HeapLimit = .

.stack          0x1fffeb48      0x400 load address 0x000099d8
                0x1fffeb48                . = ALIGN (0x8)
                0x1fffef48                . = (. + STACK_SIZE)
 *fill*         0x1fffeb48      0x400 
                0x1fffef48                __StackTop = .
                0x1fffeb48                __StackLimit = (__StackTop - STACK_SIZE)
                0x1fffef48                PROVIDE (__stack, __StackTop)

.ARM.attributes
                0x00000000       0x2d
 *(.ARM.attributes)
 .ARM.attributes
                0x00000000       0x23 e:/logiciels/freescale/kinetis design studio v2.0.0/toolchain/bin/../lib/gcc/arm-none-eabi/4.8.0/crti.o
 .ARM.attributes
                0x00000023       0x31 e:/logiciels/freescale/kinetis design studio v2.0.0/toolchain/bin/../lib/gcc/arm-none-eabi/4.8.0/crtbegin.o
 .ARM.attributes
                0x00000054       0x31 e:/logiciels/freescale/kinetis design studio v2.0.0/toolchain/bin/../lib/gcc/arm-none-eabi/4.8.0/../../../../arm-none-eabi/lib/crt0.o
 .ARM.attributes
                0x00000085       0x32 ./Tools/StringTools/StringTools.o
 .ARM.attributes
                0x000000b7       0x32 ./Tools/Decoder7Seg/decoder7Seg.o
 .ARM.attributes
                0x000000e9       0x32 ./Tools/Decoder16Seg/decoder16Seg.o
 .ARM.attributes
                0x0000011b       0x32 ./Tools/Checksum/checksum.o
 .ARM.attributes
                0x0000014d       0x1b ./Project_Settings/Startup_Code/startup_MKL16Z4.o
 .ARM.attributes
                0x00000168       0x32 ./Project_Settings/Startup_Code/system_MKL16Z4.o
 .ARM.attributes
                0x0000019a       0x32 ./DSP/Watchdog/watchdog.o
 .ARM.attributes
                0x000001cc       0x32 ./DSP/UART/uart0.o
 .ARM.attributes
                0x000001fe       0x32 ./DSP/UART/uart1.o
 .ARM.attributes
                0x00000230       0x32 ./DSP/UART/uart2.o
 .ARM.attributes
                0x00000262       0x32 ./DSP/SPI/spi0.o
 .ARM.attributes
                0x00000294       0x32 ./DSP/SPI/spi1.o
 .ARM.attributes
                0x000002c6       0x32 ./DSP/RTC/rtc.o
 .ARM.attributes
                0x000002f8       0x32 ./DSP/PIT/pit.o
 .ARM.attributes
                0x0000032a       0x32 ./DSP/I2C/i2c0.o
 .ARM.attributes
                0x0000035c       0x32 ./DSP/Device/device.o
 .ARM.attributes
                0x0000038e       0x32 ./DSP/DSP/DSP_mkl16z256vlh4.o
 .ARM.attributes
                0x000003c0       0x32 ./BSP/Tick/tick.o
 .ARM.attributes
                0x000003f2       0x32 ./BSP/RFID_CR95HF/CR95HF.o
 .ARM.attributes
                0x00000424       0x32 ./BSP/RFID_CR95HF/CR95UartMapper.o
 .ARM.attributes
                0x00000456       0x32 ./BSP/Led/led.o
 .ARM.attributes
                0x00000488       0x32 ./BSP/FRAM/FM25V20.o
 .ARM.attributes
                0x000004ba       0x32 ./BSP/Display/display.o
 .ARM.attributes
                0x000004ec       0x32 ./BSP/Button/button.o
 .ARM.attributes
                0x0000051e       0x32 ./BSP/BatteryManagement/BQ27510DRZRG2.o
 .ARM.attributes
                0x00000550       0x32 ./BSP/BatteryManagement/LTC4160.o
 .ARM.attributes
                0x00000582       0x32 ./Application/UsbManager/UsbManager.o
 .ARM.attributes
                0x000005b4       0x32 ./Application/RFIDManager/RFIDManager.o
 .ARM.attributes
                0x000005e6       0x32 ./Application/PowerManager/PowerManager.o
 .ARM.attributes
                0x00000618       0x32 ./Application/MemoryManager/MemoryManager.o
 .ARM.attributes
                0x0000064a       0x32 ./Application/ButtonManager/ButtonManager.o
 .ARM.attributes
                0x0000067c       0x32 ./Application/main.o
 .ARM.attributes
                0x000006ae       0x23 e:/logiciels/freescale/kinetis design studio v2.0.0/toolchain/bin/../lib/gcc/arm-none-eabi/4.8.0\libgcc.a(_udivsi3.o)
 .ARM.attributes
                0x000006d1       0x23 e:/logiciels/freescale/kinetis design studio v2.0.0/toolchain/bin/../lib/gcc/arm-none-eabi/4.8.0\libgcc.a(_dvmd_tls.o)
 .ARM.attributes
                0x000006f4       0x31 e:/logiciels/freescale/kinetis design studio v2.0.0/toolchain/bin/../lib/gcc/arm-none-eabi/4.8.0/../../../../arm-none-eabi/lib\libg_s.a(lib_a-atexit.o)
 .ARM.attributes
                0x00000725       0x31 e:/logiciels/freescale/kinetis design studio v2.0.0/toolchain/bin/../lib/gcc/arm-none-eabi/4.8.0/../../../../arm-none-eabi/lib\libg_s.a(lib_a-exit.o)
 .ARM.attributes
                0x00000756       0x31 e:/logiciels/freescale/kinetis design studio v2.0.0/toolchain/bin/../lib/gcc/arm-none-eabi/4.8.0/../../../../arm-none-eabi/lib\libg_s.a(lib_a-fini.o)
 .ARM.attributes
                0x00000787       0x31 e:/logiciels/freescale/kinetis design studio v2.0.0/toolchain/bin/../lib/gcc/arm-none-eabi/4.8.0/../../../../arm-none-eabi/lib\libg_s.a(lib_a-impure.o)
 .ARM.attributes
                0x000007b8       0x31 e:/logiciels/freescale/kinetis design studio v2.0.0/toolchain/bin/../lib/gcc/arm-none-eabi/4.8.0/../../../../arm-none-eabi/lib\libg_s.a(lib_a-memcpy.o)
 .ARM.attributes
                0x000007e9       0x31 e:/logiciels/freescale/kinetis design studio v2.0.0/toolchain/bin/../lib/gcc/arm-none-eabi/4.8.0/../../../../arm-none-eabi/lib\libg_s.a(lib_a-memset.o)
 .ARM.attributes
                0x0000081a       0x31 e:/logiciels/freescale/kinetis design studio v2.0.0/toolchain/bin/../lib/gcc/arm-none-eabi/4.8.0/../../../../arm-none-eabi/lib\libg_s.a(lib_a-syscalls.o)
 .ARM.attributes
                0x0000084b       0x31 e:/logiciels/freescale/kinetis design studio v2.0.0/toolchain/bin/../lib/gcc/arm-none-eabi/4.8.0/../../../../arm-none-eabi/lib\libg_s.a(lib_a-__atexit.o)
 .ARM.attributes
                0x0000087c       0x31 e:/logiciels/freescale/kinetis design studio v2.0.0/toolchain/bin/../lib/gcc/arm-none-eabi/4.8.0/../../../../arm-none-eabi/lib\libg_s.a(lib_a-__call_atexit.o)
 .ARM.attributes
                0x000008ad       0x31 e:/logiciels/freescale/kinetis design studio v2.0.0/toolchain/bin/../lib/gcc/arm-none-eabi/4.8.0/../../../../arm-none-eabi/lib\libg_s.a(lib_a-errno.o)
 .ARM.attributes
                0x000008de       0x31 e:/logiciels/freescale/kinetis design studio v2.0.0/toolchain/bin/../lib/gcc/arm-none-eabi/4.8.0/../../../../arm-none-eabi/lib\libg_s.a(lib_a-malloc.o)
 .ARM.attributes
                0x0000090f       0x31 e:/logiciels/freescale/kinetis design studio v2.0.0/toolchain/bin/../lib/gcc/arm-none-eabi/4.8.0/../../../../arm-none-eabi/lib\libg_s.a(lib_a-mallocr.o)
 .ARM.attributes
                0x00000940       0x31 e:/logiciels/freescale/kinetis design studio v2.0.0/toolchain/bin/../lib/gcc/arm-none-eabi/4.8.0/../../../../arm-none-eabi/lib\libg_s.a(lib_a-sbrkr.o)
 .ARM.attributes
                0x00000971       0x31 e:/logiciels/freescale/kinetis design studio v2.0.0/toolchain/bin/../lib/gcc/arm-none-eabi/4.8.0/../../../../arm-none-eabi/lib\libg_s.a(lib_a-freer.o)
 .ARM.attributes
                0x000009a2       0x31 e:/logiciels/freescale/kinetis design studio v2.0.0/toolchain/bin/../lib/gcc/arm-none-eabi/4.8.0/../../../../arm-none-eabi/lib\libg_s.a(lib_a-reent.o)
 .ARM.attributes
                0x000009d3       0x31 e:/logiciels/freescale/kinetis design studio v2.0.0/toolchain/bin/../lib/gcc/arm-none-eabi/4.8.0/crtend.o
 .ARM.attributes
                0x00000a04       0x23 e:/logiciels/freescale/kinetis design studio v2.0.0/toolchain/bin/../lib/gcc/arm-none-eabi/4.8.0/crtn.o
OUTPUT(BoitierRFID.elf elf32-littlearm)

.comment        0x00000000       0x2a
 .comment       0x00000000       0x2a e:/logiciels/freescale/kinetis design studio v2.0.0/toolchain/bin/../lib/gcc/arm-none-eabi/4.8.0/crtbegin.o
                                 0x2b (size before relaxing)
 .comment       0x00000000       0x2b e:/logiciels/freescale/kinetis design studio v2.0.0/toolchain/bin/../lib/gcc/arm-none-eabi/4.8.0/../../../../arm-none-eabi/lib/crt0.o
 .comment       0x00000000       0x2b ./Tools/StringTools/StringTools.o
 .comment       0x00000000       0x2b ./Tools/Decoder7Seg/decoder7Seg.o
 .comment       0x00000000       0x2b ./Tools/Decoder16Seg/decoder16Seg.o
 .comment       0x00000000       0x2b ./Tools/Checksum/checksum.o
 .comment       0x00000000       0x2b ./Project_Settings/Startup_Code/system_MKL16Z4.o
 .comment       0x00000000       0x2b ./DSP/Watchdog/watchdog.o
 .comment       0x00000000       0x2b ./DSP/UART/uart0.o
 .comment       0x00000000       0x2b ./DSP/UART/uart1.o
 .comment       0x00000000       0x2b ./DSP/UART/uart2.o
 .comment       0x00000000       0x2b ./DSP/SPI/spi0.o
 .comment       0x00000000       0x2b ./DSP/SPI/spi1.o
 .comment       0x00000000       0x2b ./DSP/RTC/rtc.o
 .comment       0x00000000       0x2b ./DSP/PIT/pit.o
 .comment       0x00000000       0x2b ./DSP/I2C/i2c0.o
 .comment       0x00000000       0x2b ./DSP/Device/device.o
 .comment       0x00000000       0x2b ./DSP/DSP/DSP_mkl16z256vlh4.o
 .comment       0x00000000       0x2b ./BSP/Tick/tick.o
 .comment       0x00000000       0x2b ./BSP/RFID_CR95HF/CR95HF.o
 .comment       0x00000000       0x2b ./BSP/RFID_CR95HF/CR95UartMapper.o
 .comment       0x00000000       0x2b ./BSP/Led/led.o
 .comment       0x00000000       0x2b ./BSP/FRAM/FM25V20.o
 .comment       0x00000000       0x2b ./BSP/Display/display.o
 .comment       0x00000000       0x2b ./BSP/Button/button.o
 .comment       0x00000000       0x2b ./BSP/BatteryManagement/BQ27510DRZRG2.o
 .comment       0x00000000       0x2b ./BSP/BatteryManagement/LTC4160.o
 .comment       0x00000000       0x2b ./Application/UsbManager/UsbManager.o
 .comment       0x00000000       0x2b ./Application/RFIDManager/RFIDManager.o
 .comment       0x00000000       0x2b ./Application/PowerManager/PowerManager.o
 .comment       0x00000000       0x2b ./Application/MemoryManager/MemoryManager.o
 .comment       0x00000000       0x2b ./Application/ButtonManager/ButtonManager.o
 .comment       0x00000000       0x2b ./Application/main.o
 .comment       0x00000000       0x2b e:/logiciels/freescale/kinetis design studio v2.0.0/toolchain/bin/../lib/gcc/arm-none-eabi/4.8.0/../../../../arm-none-eabi/lib\libg_s.a(lib_a-atexit.o)
 .comment       0x00000000       0x2b e:/logiciels/freescale/kinetis design studio v2.0.0/toolchain/bin/../lib/gcc/arm-none-eabi/4.8.0/../../../../arm-none-eabi/lib\libg_s.a(lib_a-exit.o)
 .comment       0x00000000       0x2b e:/logiciels/freescale/kinetis design studio v2.0.0/toolchain/bin/../lib/gcc/arm-none-eabi/4.8.0/../../../../arm-none-eabi/lib\libg_s.a(lib_a-fini.o)
 .comment       0x00000000       0x2b e:/logiciels/freescale/kinetis design studio v2.0.0/toolchain/bin/../lib/gcc/arm-none-eabi/4.8.0/../../../../arm-none-eabi/lib\libg_s.a(lib_a-impure.o)
 .comment       0x00000000       0x2b e:/logiciels/freescale/kinetis design studio v2.0.0/toolchain/bin/../lib/gcc/arm-none-eabi/4.8.0/../../../../arm-none-eabi/lib\libg_s.a(lib_a-memcpy.o)
 .comment       0x00000000       0x2b e:/logiciels/freescale/kinetis design studio v2.0.0/toolchain/bin/../lib/gcc/arm-none-eabi/4.8.0/../../../../arm-none-eabi/lib\libg_s.a(lib_a-memset.o)
 .comment       0x00000000       0x2b e:/logiciels/freescale/kinetis design studio v2.0.0/toolchain/bin/../lib/gcc/arm-none-eabi/4.8.0/../../../../arm-none-eabi/lib\libg_s.a(lib_a-syscalls.o)
 .comment       0x00000000       0x2b e:/logiciels/freescale/kinetis design studio v2.0.0/toolchain/bin/../lib/gcc/arm-none-eabi/4.8.0/../../../../arm-none-eabi/lib\libg_s.a(lib_a-__atexit.o)
 .comment       0x00000000       0x2b e:/logiciels/freescale/kinetis design studio v2.0.0/toolchain/bin/../lib/gcc/arm-none-eabi/4.8.0/../../../../arm-none-eabi/lib\libg_s.a(lib_a-__call_atexit.o)
 .comment       0x00000000       0x2b e:/logiciels/freescale/kinetis design studio v2.0.0/toolchain/bin/../lib/gcc/arm-none-eabi/4.8.0/../../../../arm-none-eabi/lib\libg_s.a(lib_a-errno.o)
 .comment       0x00000000       0x2b e:/logiciels/freescale/kinetis design studio v2.0.0/toolchain/bin/../lib/gcc/arm-none-eabi/4.8.0/../../../../arm-none-eabi/lib\libg_s.a(lib_a-malloc.o)
 .comment       0x00000000       0x2b e:/logiciels/freescale/kinetis design studio v2.0.0/toolchain/bin/../lib/gcc/arm-none-eabi/4.8.0/../../../../arm-none-eabi/lib\libg_s.a(lib_a-mallocr.o)
 .comment       0x00000000       0x2b e:/logiciels/freescale/kinetis design studio v2.0.0/toolchain/bin/../lib/gcc/arm-none-eabi/4.8.0/../../../../arm-none-eabi/lib\libg_s.a(lib_a-sbrkr.o)
 .comment       0x00000000       0x2b e:/logiciels/freescale/kinetis design studio v2.0.0/toolchain/bin/../lib/gcc/arm-none-eabi/4.8.0/../../../../arm-none-eabi/lib\libg_s.a(lib_a-freer.o)
 .comment       0x00000000       0x2b e:/logiciels/freescale/kinetis design studio v2.0.0/toolchain/bin/../lib/gcc/arm-none-eabi/4.8.0/../../../../arm-none-eabi/lib\libg_s.a(lib_a-reent.o)
 .comment       0x00000000       0x2b e:/logiciels/freescale/kinetis design studio v2.0.0/toolchain/bin/../lib/gcc/arm-none-eabi/4.8.0/crtend.o

.debug_info     0x00000000     0xb3f5
 .debug_info    0x00000000      0x299 ./Tools/StringTools/StringTools.o
 .debug_info    0x00000299      0x15a ./Tools/Decoder7Seg/decoder7Seg.o
 .debug_info    0x000003f3      0x180 ./Tools/Decoder16Seg/decoder16Seg.o
 .debug_info    0x00000573      0x18d ./Tools/Checksum/checksum.o
 .debug_info    0x00000700       0x9c ./Project_Settings/Startup_Code/startup_MKL16Z4.o
 .debug_info    0x0000079c      0x516 ./Project_Settings/Startup_Code/system_MKL16Z4.o
 .debug_info    0x00000cb2      0x303 ./DSP/Watchdog/watchdog.o
 .debug_info    0x00000fb5      0x53e ./DSP/UART/uart0.o
 .debug_info    0x000014f3      0x51d ./DSP/UART/uart1.o
 .debug_info    0x00001a10      0x51d ./DSP/UART/uart2.o
 .debug_info    0x00001f2d      0x2d9 ./DSP/SPI/spi0.o
 .debug_info    0x00002206      0x2f5 ./DSP/SPI/spi1.o
 .debug_info    0x000024fb      0x373 ./DSP/RTC/rtc.o
 .debug_info    0x0000286e      0x57e ./DSP/PIT/pit.o
 .debug_info    0x00002dec      0x31f ./DSP/I2C/i2c0.o
 .debug_info    0x0000310b      0x684 ./DSP/Device/device.o
 .debug_info    0x0000378f      0x512 ./DSP/DSP/DSP_mkl16z256vlh4.o
 .debug_info    0x00003ca1      0x2e1 ./BSP/Tick/tick.o
 .debug_info    0x00003f82      0x8c4 ./BSP/RFID_CR95HF/CR95HF.o
 .debug_info    0x00004846      0x764 ./BSP/RFID_CR95HF/CR95UartMapper.o
 .debug_info    0x00004faa      0x35a ./BSP/Led/led.o
 .debug_info    0x00005304      0x761 ./BSP/FRAM/FM25V20.o
 .debug_info    0x00005a65      0x7d9 ./BSP/Display/display.o
 .debug_info    0x0000623e      0x35a ./BSP/Button/button.o
 .debug_info    0x00006598      0x93f ./BSP/BatteryManagement/BQ27510DRZRG2.o
 .debug_info    0x00006ed7      0x3a6 ./BSP/BatteryManagement/LTC4160.o
 .debug_info    0x0000727d      0xdd8 ./Application/UsbManager/UsbManager.o
 .debug_info    0x00008055      0xd2d ./Application/RFIDManager/RFIDManager.o
 .debug_info    0x00008d82      0xa9a ./Application/PowerManager/PowerManager.o
 .debug_info    0x0000981c      0xa13 ./Application/MemoryManager/MemoryManager.o
 .debug_info    0x0000a22f      0xde6 ./Application/ButtonManager/ButtonManager.o
 .debug_info    0x0000b015      0x3e0 ./Application/main.o

.debug_abbrev   0x00000000     0x2b58
 .debug_abbrev  0x00000000       0xee ./Tools/StringTools/StringTools.o
 .debug_abbrev  0x000000ee       0xe4 ./Tools/Decoder7Seg/decoder7Seg.o
 .debug_abbrev  0x000001d2       0xbb ./Tools/Decoder16Seg/decoder16Seg.o
 .debug_abbrev  0x0000028d       0x7f ./Tools/Checksum/checksum.o
 .debug_abbrev  0x0000030c       0x14 ./Project_Settings/Startup_Code/startup_MKL16Z4.o
 .debug_abbrev  0x00000320      0x121 ./Project_Settings/Startup_Code/system_MKL16Z4.o
 .debug_abbrev  0x00000441       0xf2 ./DSP/Watchdog/watchdog.o
 .debug_abbrev  0x00000533      0x1dd ./DSP/UART/uart0.o
 .debug_abbrev  0x00000710      0x1e4 ./DSP/UART/uart1.o
 .debug_abbrev  0x000008f4      0x1e4 ./DSP/UART/uart2.o
 .debug_abbrev  0x00000ad8      0x13a ./DSP/SPI/spi0.o
 .debug_abbrev  0x00000c12      0x13a ./DSP/SPI/spi1.o
 .debug_abbrev  0x00000d4c      0x14e ./DSP/RTC/rtc.o
 .debug_abbrev  0x00000e9a      0x14f ./DSP/PIT/pit.o
 .debug_abbrev  0x00000fe9      0x14b ./DSP/I2C/i2c0.o
 .debug_abbrev  0x00001134      0x159 ./DSP/Device/device.o
 .debug_abbrev  0x0000128d      0x121 ./DSP/DSP/DSP_mkl16z256vlh4.o
 .debug_abbrev  0x000013ae      0x1b1 ./BSP/Tick/tick.o
 .debug_abbrev  0x0000155f      0x22e ./BSP/RFID_CR95HF/CR95HF.o
 .debug_abbrev  0x0000178d      0x219 ./BSP/RFID_CR95HF/CR95UartMapper.o
 .debug_abbrev  0x000019a6       0xcf ./BSP/Led/led.o
 .debug_abbrev  0x00001a75      0x1d6 ./BSP/FRAM/FM25V20.o
 .debug_abbrev  0x00001c4b      0x1c5 ./BSP/Display/display.o
 .debug_abbrev  0x00001e10       0xcf ./BSP/Button/button.o
 .debug_abbrev  0x00001edf      0x149 ./BSP/BatteryManagement/BQ27510DRZRG2.o
 .debug_abbrev  0x00002028      0x10c ./BSP/BatteryManagement/LTC4160.o
 .debug_abbrev  0x00002134      0x1c7 ./Application/UsbManager/UsbManager.o
 .debug_abbrev  0x000022fb      0x1e3 ./Application/RFIDManager/RFIDManager.o
 .debug_abbrev  0x000024de      0x1d6 ./Application/PowerManager/PowerManager.o
 .debug_abbrev  0x000026b4      0x189 ./Application/MemoryManager/MemoryManager.o
 .debug_abbrev  0x0000283d      0x1be ./Application/ButtonManager/ButtonManager.o
 .debug_abbrev  0x000029fb      0x15d ./Application/main.o

.debug_aranges  0x00000000      0x998
 .debug_aranges
                0x00000000       0x50 ./Tools/StringTools/StringTools.o
 .debug_aranges
                0x00000050       0x28 ./Tools/Decoder7Seg/decoder7Seg.o
 .debug_aranges
                0x00000078       0x20 ./Tools/Decoder16Seg/decoder16Seg.o
 .debug_aranges
                0x00000098       0x38 ./Tools/Checksum/checksum.o
 .debug_aranges
                0x000000d0       0x20 ./Project_Settings/Startup_Code/startup_MKL16Z4.o
 .debug_aranges
                0x000000f0       0x28 ./Project_Settings/Startup_Code/system_MKL16Z4.o
 .debug_aranges
                0x00000118       0x30 ./DSP/Watchdog/watchdog.o
 .debug_aranges
                0x00000148       0x40 ./DSP/UART/uart0.o
 .debug_aranges
                0x00000188       0x40 ./DSP/UART/uart1.o
 .debug_aranges
                0x000001c8       0x40 ./DSP/UART/uart2.o
 .debug_aranges
                0x00000208       0x38 ./DSP/SPI/spi0.o
 .debug_aranges
                0x00000240       0x38 ./DSP/SPI/spi1.o
 .debug_aranges
                0x00000278       0x38 ./DSP/RTC/rtc.o
 .debug_aranges
                0x000002b0       0x28 ./DSP/PIT/pit.o
 .debug_aranges
                0x000002d8       0x38 ./DSP/I2C/i2c0.o
 .debug_aranges
                0x00000310       0x48 ./DSP/Device/device.o
 .debug_aranges
                0x00000358       0x88 ./DSP/DSP/DSP_mkl16z256vlh4.o
 .debug_aranges
                0x000003e0       0x38 ./BSP/Tick/tick.o
 .debug_aranges
                0x00000418       0xc0 ./BSP/RFID_CR95HF/CR95HF.o
 .debug_aranges
                0x000004d8       0x80 ./BSP/RFID_CR95HF/CR95UartMapper.o
 .debug_aranges
                0x00000558       0x20 ./BSP/Led/led.o
 .debug_aranges
                0x00000578       0x68 ./BSP/FRAM/FM25V20.o
 .debug_aranges
                0x000005e0       0x48 ./BSP/Display/display.o
 .debug_aranges
                0x00000628       0x20 ./BSP/Button/button.o
 .debug_aranges
                0x00000648       0xc0 ./BSP/BatteryManagement/BQ27510DRZRG2.o
 .debug_aranges
                0x00000708       0x28 ./BSP/BatteryManagement/LTC4160.o
 .debug_aranges
                0x00000730       0x40 ./Application/UsbManager/UsbManager.o
 .debug_aranges
                0x00000770       0x60 ./Application/RFIDManager/RFIDManager.o
 .debug_aranges
                0x000007d0       0x80 ./Application/PowerManager/PowerManager.o
 .debug_aranges
                0x00000850       0x70 ./Application/MemoryManager/MemoryManager.o
 .debug_aranges
                0x000008c0       0x70 ./Application/ButtonManager/ButtonManager.o
 .debug_aranges
                0x00000930       0x68 ./Application/main.o

.debug_ranges   0x00000000      0x788
 .debug_ranges  0x00000000       0x40 ./Tools/StringTools/StringTools.o
 .debug_ranges  0x00000040       0x18 ./Tools/Decoder7Seg/decoder7Seg.o
 .debug_ranges  0x00000058       0x10 ./Tools/Decoder16Seg/decoder16Seg.o
 .debug_ranges  0x00000068       0x28 ./Tools/Checksum/checksum.o
 .debug_ranges  0x00000090       0x18 ./Project_Settings/Startup_Code/system_MKL16Z4.o
 .debug_ranges  0x000000a8       0x20 ./DSP/Watchdog/watchdog.o
 .debug_ranges  0x000000c8       0x30 ./DSP/UART/uart0.o
 .debug_ranges  0x000000f8       0x30 ./DSP/UART/uart1.o
 .debug_ranges  0x00000128       0x30 ./DSP/UART/uart2.o
 .debug_ranges  0x00000158       0x28 ./DSP/SPI/spi0.o
 .debug_ranges  0x00000180       0x28 ./DSP/SPI/spi1.o
 .debug_ranges  0x000001a8       0x28 ./DSP/RTC/rtc.o
 .debug_ranges  0x000001d0       0x18 ./DSP/PIT/pit.o
 .debug_ranges  0x000001e8       0x28 ./DSP/I2C/i2c0.o
 .debug_ranges  0x00000210       0x38 ./DSP/Device/device.o
 .debug_ranges  0x00000248       0x78 ./DSP/DSP/DSP_mkl16z256vlh4.o
 .debug_ranges  0x000002c0       0x28 ./BSP/Tick/tick.o
 .debug_ranges  0x000002e8       0xb0 ./BSP/RFID_CR95HF/CR95HF.o
 .debug_ranges  0x00000398       0x70 ./BSP/RFID_CR95HF/CR95UartMapper.o
 .debug_ranges  0x00000408       0x10 ./BSP/Led/led.o
 .debug_ranges  0x00000418       0x58 ./BSP/FRAM/FM25V20.o
 .debug_ranges  0x00000470       0x38 ./BSP/Display/display.o
 .debug_ranges  0x000004a8       0x10 ./BSP/Button/button.o
 .debug_ranges  0x000004b8       0xb0 ./BSP/BatteryManagement/BQ27510DRZRG2.o
 .debug_ranges  0x00000568       0x18 ./BSP/BatteryManagement/LTC4160.o
 .debug_ranges  0x00000580       0x30 ./Application/UsbManager/UsbManager.o
 .debug_ranges  0x000005b0       0x50 ./Application/RFIDManager/RFIDManager.o
 .debug_ranges  0x00000600       0x70 ./Application/PowerManager/PowerManager.o
 .debug_ranges  0x00000670       0x60 ./Application/MemoryManager/MemoryManager.o
 .debug_ranges  0x000006d0       0x60 ./Application/ButtonManager/ButtonManager.o
 .debug_ranges  0x00000730       0x58 ./Application/main.o

.debug_macro    0x00000000     0x8d0a
 .debug_macro   0x00000000       0x1b ./Tools/StringTools/StringTools.o
 .debug_macro   0x0000001b      0x802 ./Tools/StringTools/StringTools.o
 .debug_macro   0x0000081d       0x1a ./Tools/Decoder7Seg/decoder7Seg.o
 .debug_macro   0x00000837       0x6a ./Tools/Decoder7Seg/decoder7Seg.o
 .debug_macro   0x000008a1       0x1a ./Tools/Decoder16Seg/decoder16Seg.o
 .debug_macro   0x000008bb       0xca ./Tools/Decoder16Seg/decoder16Seg.o
 .debug_macro   0x00000985       0x1b ./Tools/Checksum/checksum.o
 .debug_macro   0x000009a0       0x60 ./Project_Settings/Startup_Code/system_MKL16Z4.o
 .debug_macro   0x00000a00      0x214 ./Project_Settings/Startup_Code/system_MKL16Z4.o
 .debug_macro   0x00000c14       0x4b ./Project_Settings/Startup_Code/system_MKL16Z4.o
 .debug_macro   0x00000c5f       0x3a ./Project_Settings/Startup_Code/system_MKL16Z4.o
 .debug_macro   0x00000c99       0x1f ./Project_Settings/Startup_Code/system_MKL16Z4.o
 .debug_macro   0x00000cb8      0x250 ./Project_Settings/Startup_Code/system_MKL16Z4.o
 .debug_macro   0x00000f08       0xc5 ./Project_Settings/Startup_Code/system_MKL16Z4.o
 .debug_macro   0x00000fcd     0x5642 ./Project_Settings/Startup_Code/system_MKL16Z4.o
 .debug_macro   0x0000660f       0x88 ./DSP/Watchdog/watchdog.o
 .debug_macro   0x00006697       0x16 ./DSP/Watchdog/watchdog.o
 .debug_macro   0x000066ad       0x39 ./DSP/Watchdog/watchdog.o
 .debug_macro   0x000066e6      0x1fb ./DSP/Watchdog/watchdog.o
 .debug_macro   0x000068e1       0x97 ./DSP/UART/uart0.o
 .debug_macro   0x00006978       0x65 ./DSP/UART/uart0.o
 .debug_macro   0x000069dd       0x97 ./DSP/UART/uart1.o
 .debug_macro   0x00006a74       0x57 ./DSP/UART/uart1.o
 .debug_macro   0x00006acb       0x97 ./DSP/UART/uart2.o
 .debug_macro   0x00006b62       0x57 ./DSP/UART/uart2.o
 .debug_macro   0x00006bb9       0x8d ./DSP/SPI/spi0.o
 .debug_macro   0x00006c46       0x44 ./DSP/SPI/spi0.o
 .debug_macro   0x00006c8a       0x8d ./DSP/SPI/spi1.o
 .debug_macro   0x00006d17       0x44 ./DSP/SPI/spi1.o
 .debug_macro   0x00006d5b       0x8d ./DSP/RTC/rtc.o
 .debug_macro   0x00006de8       0x10 ./DSP/RTC/rtc.o
 .debug_macro   0x00006df8       0x8d ./DSP/PIT/pit.o
 .debug_macro   0x00006e85       0x2e ./DSP/PIT/pit.o
 .debug_macro   0x00006eb3       0xd9 ./DSP/I2C/i2c0.o
 .debug_macro   0x00006f8c       0x3a ./DSP/I2C/i2c0.o
 .debug_macro   0x00006fc6       0x8d ./DSP/Device/device.o
 .debug_macro   0x00007053       0x22 ./DSP/Device/device.o
 .debug_macro   0x00007075       0x74 ./DSP/DSP/DSP_mkl16z256vlh4.o
 .debug_macro   0x000070e9       0x9c ./BSP/Tick/tick.o
 .debug_macro   0x00007185       0x48 ./BSP/Tick/tick.o
 .debug_macro   0x000071cd      0x102 ./BSP/RFID_CR95HF/CR95HF.o
 .debug_macro   0x000072cf       0x65 ./BSP/RFID_CR95HF/CR95HF.o
 .debug_macro   0x00007334       0x5d ./BSP/RFID_CR95HF/CR95HF.o
 .debug_macro   0x00007391       0x10 ./BSP/RFID_CR95HF/CR95HF.o
 .debug_macro   0x000073a1       0x34 ./BSP/RFID_CR95HF/CR95HF.o
 .debug_macro   0x000073d5       0x48 ./BSP/RFID_CR95HF/CR95HF.o
 .debug_macro   0x0000741d       0x1c ./BSP/RFID_CR95HF/CR95HF.o
 .debug_macro   0x00007439       0xb9 ./BSP/RFID_CR95HF/CR95UartMapper.o
 .debug_macro   0x000074f2       0x8d ./BSP/Led/led.o
 .debug_macro   0x0000757f       0x34 ./BSP/Led/led.o
 .debug_macro   0x000075b3       0xa8 ./BSP/FRAM/FM25V20.o
 .debug_macro   0x0000765b       0x84 ./BSP/FRAM/FM25V20.o
 .debug_macro   0x000076df       0xae ./BSP/Display/display.o
 .debug_macro   0x0000778d       0x3b ./BSP/Display/display.o
 .debug_macro   0x000077c8       0x8d ./BSP/Button/button.o
 .debug_macro   0x00007855       0x28 ./BSP/Button/button.o
 .debug_macro   0x0000787d       0xa6 ./BSP/BatteryManagement/BQ27510DRZRG2.o
 .debug_macro   0x00007923       0x8e ./BSP/BatteryManagement/BQ27510DRZRG2.o
 .debug_macro   0x000079b1       0x8d ./BSP/BatteryManagement/LTC4160.o
 .debug_macro   0x00007a3e       0x7b ./BSP/BatteryManagement/LTC4160.o
 .debug_macro   0x00007ab9      0x21a ./Application/UsbManager/UsbManager.o
 .debug_macro   0x00007cd3       0x57 ./Application/UsbManager/UsbManager.o
 .debug_macro   0x00007d2a       0x52 ./Application/UsbManager/UsbManager.o
 .debug_macro   0x00007d7c       0x16 ./Application/UsbManager/UsbManager.o
 .debug_macro   0x00007d92       0x4a ./Application/UsbManager/UsbManager.o
 .debug_macro   0x00007ddc      0x196 ./Application/UsbManager/UsbManager.o
 .debug_macro   0x00007f72       0x7c ./Application/UsbManager/UsbManager.o
 .debug_macro   0x00007fee       0x16 ./Application/UsbManager/UsbManager.o
 .debug_macro   0x00008004       0x6b ./Application/UsbManager/UsbManager.o
 .debug_macro   0x0000806f       0x81 ./Application/UsbManager/UsbManager.o
 .debug_macro   0x000080f0       0x4a ./Application/UsbManager/UsbManager.o
 .debug_macro   0x0000813a       0x28 ./Application/UsbManager/UsbManager.o
 .debug_macro   0x00008162       0x2e ./Application/UsbManager/UsbManager.o
 .debug_macro   0x00008190       0x3a ./Application/UsbManager/UsbManager.o
 .debug_macro   0x000081ca       0x10 ./Application/UsbManager/UsbManager.o
 .debug_macro   0x000081da       0x8e ./Application/UsbManager/UsbManager.o
 .debug_macro   0x00008268      0x216 ./Application/RFIDManager/RFIDManager.o
 .debug_macro   0x0000847e       0x5d ./Application/RFIDManager/RFIDManager.o
 .debug_macro   0x000084db      0x216 ./Application/PowerManager/PowerManager.o
 .debug_macro   0x000086f1       0xcc ./Application/MemoryManager/MemoryManager.o
 .debug_macro   0x000087bd      0x21c ./Application/ButtonManager/ButtonManager.o
 .debug_macro   0x000089d9       0x28 ./Application/ButtonManager/ButtonManager.o
 .debug_macro   0x00008a01      0x244 ./Application/main.o
 .debug_macro   0x00008c45       0x5d ./Application/main.o
 .debug_macro   0x00008ca2       0x3a ./Application/main.o
 .debug_macro   0x00008cdc       0x2e ./Application/main.o

.debug_line     0x00000000     0x633f
 .debug_line    0x00000000      0x144 ./Tools/StringTools/StringTools.o
 .debug_line    0x00000144       0xae ./Tools/Decoder7Seg/decoder7Seg.o
 .debug_line    0x000001f2       0xc2 ./Tools/Decoder16Seg/decoder16Seg.o
 .debug_line    0x000002b4       0xdf ./Tools/Checksum/checksum.o
 .debug_line    0x00000393       0x83 ./Project_Settings/Startup_Code/startup_MKL16Z4.o
 .debug_line    0x00000416      0x21c ./Project_Settings/Startup_Code/system_MKL16Z4.o
 .debug_line    0x00000632      0x1e0 ./DSP/Watchdog/watchdog.o
 .debug_line    0x00000812      0x2bf ./DSP/UART/uart0.o
 .debug_line    0x00000ad1      0x2b8 ./DSP/UART/uart1.o
 .debug_line    0x00000d89      0x2b8 ./DSP/UART/uart2.o
 .debug_line    0x00001041      0x284 ./DSP/SPI/spi0.o
 .debug_line    0x000012c5      0x288 ./DSP/SPI/spi1.o
 .debug_line    0x0000154d      0x1f6 ./DSP/RTC/rtc.o
 .debug_line    0x00001743      0x1d9 ./DSP/PIT/pit.o
 .debug_line    0x0000191c      0x280 ./DSP/I2C/i2c0.o
 .debug_line    0x00001b9c      0x29a ./DSP/Device/device.o
 .debug_line    0x00001e36      0x2d5 ./DSP/DSP/DSP_mkl16z256vlh4.o
 .debug_line    0x0000210b      0x21a ./BSP/Tick/tick.o
 .debug_line    0x00002325      0x560 ./BSP/RFID_CR95HF/CR95HF.o
 .debug_line    0x00002885      0x322 ./BSP/RFID_CR95HF/CR95UartMapper.o
 .debug_line    0x00002ba7      0x1b0 ./BSP/Led/led.o
 .debug_line    0x00002d57      0x324 ./BSP/FRAM/FM25V20.o
 .debug_line    0x0000307b      0x2ea ./BSP/Display/display.o
 .debug_line    0x00003365      0x1b8 ./BSP/Button/button.o
 .debug_line    0x0000351d      0x401 ./BSP/BatteryManagement/BQ27510DRZRG2.o
 .debug_line    0x0000391e      0x1e1 ./BSP/BatteryManagement/LTC4160.o
 .debug_line    0x00003aff      0x778 ./Application/UsbManager/UsbManager.o
 .debug_line    0x00004277      0x7a6 ./Application/RFIDManager/RFIDManager.o
 .debug_line    0x00004a1d      0x6eb ./Application/PowerManager/PowerManager.o
 .debug_line    0x00005108      0x3fc ./Application/MemoryManager/MemoryManager.o
 .debug_line    0x00005504      0x79e ./Application/ButtonManager/ButtonManager.o
 .debug_line    0x00005ca2      0x69d ./Application/main.o

.debug_str      0x00000000    0x25bb7
 .debug_str     0x00000000     0x237f ./Tools/StringTools/StringTools.o
                               0x23c0 (size before relaxing)
 .debug_str     0x0000237f      0x2a5 ./Tools/Decoder7Seg/decoder7Seg.o
                               0x24ff (size before relaxing)
 .debug_str     0x00002624      0x4d3 ./Tools/Decoder16Seg/decoder16Seg.o
                               0x2739 (size before relaxing)
 .debug_str     0x00002af7       0x90 ./Tools/Checksum/checksum.o
                               0x2302 (size before relaxing)
 .debug_str     0x00002b87    0x1be13 ./Project_Settings/Startup_Code/system_MKL16Z4.o
                              0x1e325 (size before relaxing)
 .debug_str     0x0001e99a      0x9d8 ./DSP/Watchdog/watchdog.o
                              0x1ea9b (size before relaxing)
 .debug_str     0x0001f372      0x479 ./DSP/UART/uart0.o
                              0x1ed66 (size before relaxing)
 .debug_str     0x0001f7eb      0x224 ./DSP/UART/uart1.o
                              0x1ecfa (size before relaxing)
 .debug_str     0x0001fa0f      0x222 ./DSP/UART/uart2.o
                              0x1ecf8 (size before relaxing)
 .debug_str     0x0001fc31      0x1d7 ./DSP/SPI/spi0.o
                              0x1eb8c (size before relaxing)
 .debug_str     0x0001fe08      0x1a9 ./DSP/SPI/spi1.o
                              0x1eb97 (size before relaxing)
 .debug_str     0x0001ffb1       0xdb ./DSP/RTC/rtc.o
                              0x1ea6f (size before relaxing)
 .debug_str     0x0002008c      0x21a ./DSP/PIT/pit.o
                              0x1ece5 (size before relaxing)
 .debug_str     0x000202a6      0x4e6 ./DSP/I2C/i2c0.o
                              0x1ee9d (size before relaxing)
 .debug_str     0x0002078c      0x18e ./DSP/Device/device.o
                              0x1ec43 (size before relaxing)
 .debug_str     0x0002091a      0x13b ./DSP/DSP/DSP_mkl16z256vlh4.o
                              0x1ebbb (size before relaxing)
 .debug_str     0x00020a55      0x264 ./BSP/Tick/tick.o
                              0x1ed22 (size before relaxing)
 .debug_str     0x00020cb9      0x99a ./BSP/RFID_CR95HF/CR95HF.o
                              0x1fa1f (size before relaxing)
 .debug_str     0x00021653      0x20a ./BSP/RFID_CR95HF/CR95UartMapper.o
                              0x1f116 (size before relaxing)
 .debug_str     0x0002185d      0x183 ./BSP/Led/led.o
                              0x1eb5a (size before relaxing)
 .debug_str     0x000219e0      0x5aa ./BSP/FRAM/FM25V20.o
                              0x1f107 (size before relaxing)
 .debug_str     0x00021f8a      0x2f6 ./BSP/Display/display.o
                              0x1f524 (size before relaxing)
 .debug_str     0x00022280      0x148 ./BSP/Button/button.o
                              0x1eb1f (size before relaxing)
 .debug_str     0x000223c8      0x5ef ./BSP/BatteryManagement/BQ27510DRZRG2.o
                              0x1f010 (size before relaxing)
 .debug_str     0x000229b7      0x420 ./BSP/BatteryManagement/LTC4160.o
                              0x1edf7 (size before relaxing)
 .debug_str     0x00022dd7     0x1c80 ./Application/UsbManager/UsbManager.o
                              0x22ad7 (size before relaxing)
 .debug_str     0x00024a57      0x8d7 ./Application/RFIDManager/RFIDManager.o
                              0x2337f (size before relaxing)
 .debug_str     0x0002532e      0x457 ./Application/PowerManager/PowerManager.o
                              0x22cba (size before relaxing)
 .debug_str     0x00025785      0x1cc ./Application/MemoryManager/MemoryManager.o
                              0x204b1 (size before relaxing)
 .debug_str     0x00025951      0x1a6 ./Application/ButtonManager/ButtonManager.o
                              0x22f10 (size before relaxing)
 .debug_str     0x00025af7       0xc0 ./Application/main.o
                              0x22574 (size before relaxing)

.debug_frame    0x00000000     0x1bbc
 .debug_frame   0x00000000       0xf0 ./Tools/StringTools/StringTools.o
 .debug_frame   0x000000f0       0x50 ./Tools/Decoder7Seg/decoder7Seg.o
 .debug_frame   0x00000140       0x30 ./Tools/Decoder16Seg/decoder16Seg.o
 .debug_frame   0x00000170       0x90 ./Tools/Checksum/checksum.o
 .debug_frame   0x00000200       0x4c ./Project_Settings/Startup_Code/system_MKL16Z4.o
 .debug_frame   0x0000024c       0x68 ./DSP/Watchdog/watchdog.o
 .debug_frame   0x000002b4       0xb0 ./DSP/UART/uart0.o
 .debug_frame   0x00000364       0xb0 ./DSP/UART/uart1.o
 .debug_frame   0x00000414       0xb0 ./DSP/UART/uart2.o
 .debug_frame   0x000004c4       0x8c ./DSP/SPI/spi0.o
 .debug_frame   0x00000550       0x8c ./DSP/SPI/spi1.o
 .debug_frame   0x000005dc       0x88 ./DSP/RTC/rtc.o
 .debug_frame   0x00000664       0x54 ./DSP/PIT/pit.o
 .debug_frame   0x000006b8       0x8c ./DSP/I2C/i2c0.o
 .debug_frame   0x00000744       0xbc ./DSP/Device/device.o
 .debug_frame   0x00000800      0x1b4 ./DSP/DSP/DSP_mkl16z256vlh4.o
 .debug_frame   0x000009b4       0x84 ./BSP/Tick/tick.o
 .debug_frame   0x00000a38      0x298 ./BSP/RFID_CR95HF/CR95HF.o
 .debug_frame   0x00000cd0      0x190 ./BSP/RFID_CR95HF/CR95UartMapper.o
 .debug_frame   0x00000e60       0x2c ./BSP/Led/led.o
 .debug_frame   0x00000e8c      0x14c ./BSP/FRAM/FM25V20.o
 .debug_frame   0x00000fd8       0xd4 ./BSP/Display/display.o
 .debug_frame   0x000010ac       0x2c ./BSP/Button/button.o
 .debug_frame   0x000010d8      0x2f4 ./BSP/BatteryManagement/BQ27510DRZRG2.o
 .debug_frame   0x000013cc       0x4c ./BSP/BatteryManagement/LTC4160.o
 .debug_frame   0x00001418       0xb4 ./Application/UsbManager/UsbManager.o
 .debug_frame   0x000014cc      0x120 ./Application/RFIDManager/RFIDManager.o
 .debug_frame   0x000015ec      0x194 ./Application/PowerManager/PowerManager.o
 .debug_frame   0x00001780      0x19c ./Application/MemoryManager/MemoryManager.o
 .debug_frame   0x0000191c      0x178 ./Application/ButtonManager/ButtonManager.o
 .debug_frame   0x00001a94      0x128 ./Application/main.o
